:100000000C94EA0B0C94250C0C9499940C94250CEC
:100010000C94250C0C94333E0C94250C0C94250C5C
:100020000C94250C0C94250C0C94250C0C94250C8C
:100030000C94250C0C94A8940C94250C0C94250C71
:100040000C94250C0C94250C0C94250C0C94250C6C
:100050000C94250C0C94250C0C94250C0C94250C5C
:100060000C94250C0C944FDF0C94250C0C947BDF26
:100070000C94250C0C94250C0C94250C0C94250C3C
:100080000C941E910C94250C0C94250C0C94250CAE
:100090000C94B4DF0C94250C0C94ECDF0C94250C20
:1000A0000C94250C0C94250C0C946F940C94250C3A
:1000B0000C94250C0C94250C0C94250C0C94250CFC
:1000C0000C94250C0C94250C0C94250C0C94250CEC
:1000D0000C94250C0C94250C0C94250C0C94250CDC
:1000E0000C94250C543B9B3B9E3B803BAB3B5B3CC9
:1000F0005B3C803BEE3B5B3CFD3B023C173C1C3CCD
:10010000B53BBE3BCC3B803BE93B5B3C673BB03BFC
:10011000213C2F3C363C5B3C5B3C3A3C7CAC7FACAE
:1001200082AC85AC88AC8BAC8EAC91AC94AC97AC0B
:100130009AAC9DACA0ACA3ACA6ACA9ACACAC48D37B
:100140004AD34CD356D359D35CD35FD362D365D350
:1001500068D36BD36ED371D374D377D37AD37DD373
:1001600080D383D386D389D35468696E672D4F2D8E
:100170004D617469630024F404D9201BC40C5C0E27
:100180009804C4095F0265077101F405F900FB04D6
:10019000B30048048700C1036900580355000303F6
:1001A0004500BE023A008402310053022A002902AF
:1001B000250004022000E4011C00C8011900AF0161
:1001C00017009801140084011300710110006101EF
:1001D000100051010E0043010D0036010B002B01F0
:1001E0000B0020010B00150109000C01090003019F
:1001F0000800FB000800F3000800EB000700E40023
:100200000600DE000600D8000600D2000600CC0082
:100210000500C7000500C2000500BD000400B900CC
:100220000400B5000400B1000400AD000400A90002
:100230000400A5000300A20003009F0004009B002F
:100240000300980003009500020093000300900053
:1002500003008D0002008B0003008800020086006E
:10026000020084000300810002007F0002007D0084
:1002700002007B0002007900020077000100760096
:1002800002007400020072000100710002006F00A1
:1002900002006D0001006C0002006A0001006900AC
:1002A00002006700010066000100650001006400B3
:1002B00002006200010061000100600001005F00B7
:1002C00002005D0001005C0001005B0001005A00BB
:1002D00001005900010058000100570001005600BC
:1002E00001005500010054000100530000005300BC
:1002F00001005200010051000100500001004F00B8
:1003000001004E0000004E0001004D0001004C00B5
:1003100001004B0000004B0001004A0001004900B1
:1003200001004800000048000100470001004600AD
:1003300000004600010045000000450001004400A7
:1003400001004300000043000100420000004200A1
:1003500001004100000041000100400001003F0099
:1003600000003F0001003E0000003E0001003D0093
:1003700000003D0001003C0000003C0000003C008B
:1003800001003B0000003B0001003A0000003A0081
:100390000100390000003900010038000000380079
:1003A000000038000100370000003700010036006F
:1003B0000000360000003600010035000000350066
:1003C000000035000100340000003400000034005B
:1003D0000100330000003300000033000100320050
:1003E0000000320000003200010031000000310046
:1003F000000031000100300000003000000030003B
:1004000001002F0000002F0000002F0000002F002F
:1004100001002E0000002E0000002E0001002D0023
:1004200000002D0000002D0000002D0001002C0018
:1004300000002C0000002C0000002C0001002B000C
:1004400000002B0000002B0000002B0001002A0000
:1004500000002A0000002A0000002A0001002900F4
:1004600000002900000029000000290000002900E8
:1004700001002800000028000000280000002800DB
:1004800000002800010027000000270000002700CE
:1004900000002700000027000100260000002600C1
:1004A00000002600000026000000260001002500B4
:1004B00000002500000025000000250000002500A8
:1004C000000025000100240000002400000024009A
:1004D000000024000000240001002300000023008D
:1004E0000000230000002300000023000000230080
:1004F0000000230001002200000022000000220072
:100500000000220000002200000022000100210063
:100510000000210000002100000021000000210057
:100520000000210000002100010020000000200048
:10053000000020000000200000002000000020003B
:10054000000020000000200001001F0000001F002C
:1005500000001F0000001F0000001F0000001F001F
:1005600000001F0001001E0000001E0000001E0011
:1005700000001E00000024F4D43050C38E20C2A21C
:100580004017828B7011127A910D816CD90AA86183
:10059000E108C7586607615143061E4B5D05C1451A
:1005A000A7041A411104093D9803713931034036FB
:1005B000DB0265339102D4305402802E1D02632C7D
:1005C000EE01752AC501B028A001102781018F25F1
:1005D00064012B244B01E0223401AC211F018D204A
:1005E0000D01801FFC00841EED00971DDF00B81C6C
:1005F000D200E61BC600201BBC00641AB200B21970
:10060000A8000A19A0006A189900D1179100401794
:100610008B00B516840031167E00B31579003A15AB
:100620007300C7146F0058146A00EE136600881335
:10063000630025135E00C7125B006C125700151291
:100640005400C111510070114F0021114B00D61000
:1006500049008D1047004610440002104200C00FB0
:100660004000800F3E00420F3C00060F3B00CB0EC7
:100670003800930E37005C0E3500270E3400F30D62
:100680003200C10D3100900D3000600D2E00320D92
:100690002D00050D2C00D90C2B00AE0C2900850C6B
:1006A00029005C0C2700350C27000E0C2600E80BF7
:1006B0002400C40B2400A00B23007D0B23005A0B45
:1006C0002100390B2100180B2000F80A1F00D90A5D
:1006D0001E00BB0A1E009D0A1D00800A1D00630A41
:1006E0001C00470A1B002C0A1B00110A1A00F709FC
:1006F0001A00DD091900C4091900AB091900920993
:1007000017007B091800630917004C091600360909
:100710001600200916000A091500F5081500E00862
:100720001400CC081400B8081400A40814009008A1
:1007300013007D0812006B081300580812004608C9
:1007400012003408110023081100120811000108DA
:100750001100F0071000E0071000D0071000C007DC
:100760001000B0070F00A107100091070E008307CB
:100770000F0074070F0065070E0057070E004907AA
:100780000E003B070D002E070E0020070D0013077B
:100790000D0006070D00F9060C00ED060D00E00641
:1007A0000C00D4060C00C8060C00BC060C00B006F9
:1007B0000C00A4060B0099060C008D060B008206A7
:1007C0000B0077060B006C060B0061060A0057064B
:1007D0000B004C060A0042060A0038060A002E06E4
:1007E0000A0024060A001A060A0010060900070675
:1007F0000A00FD050900F4050900EB050900E20502
:100800000900D9050900D0050900C7050900BE0582
:100810000900B5050800AD050800A50509009C05FF
:100820000800940508008C050800840508007C0574
:100830000800740508006C050700650508005D05E3
:100840000700560508004E0507004705070040054C
:10085000080038050700310507002A0507002305B1
:1008600007001C050600160507000F050700080510
:10087000060002050700FB040600F5040700EE046D
:100880000600E8040600E2040700DB040600D504C5
:100890000600CF040600C9040600C3040600BD0418
:1008A0000600B7040600B1040500AC040600A60467
:1008B0000600A00405009B040600950405009004B2
:1008C00006008A04050085040500800406007A04F9
:1008D000050075040500700405006B04050066043E
:1008E0000500610405005C0405005704050052047E
:1008F00005004D04050048040500430405003E04BE
:1009000004003A04050035040500300404002C04FA
:10091000050027040400230405001E0404001A0433
:10092000040016040500110404000D040400090469
:1009300005000404040000040400FC030400F803A0
:100940000400F4030400F0030400EC030400E803D3
:100950000400E4030400E0030400DC030400D80303
:100960000400D4030400D0030400CC030400C80333
:100970000300C503030020205361696C6669736836
:1009800020465720202000202D2D2D2D2D2D2D2DC2
:100990002D2D2D2D2D2D20005468696E67203332AA
:1009A00030383420342E317A0020526576697369EC
:1009B0006F6E2030303836362000582F5920446969
:1009C00072656374696F6E3A004D6F64656C205692
:1009D00069657700557365722056696577004A6FBF
:1009E00067206D6F64653A20002E316D6D00316DAA
:1009F0006D00436F6E742E2E002020592020202081
:100A0000202020202020205A2B00202020592B207D
:100A100020202020202020205A2B0058205620580B
:100A20002020202020286D6F64652900582D205635
:100A30002020582B2020286D6F6465290020205924
:100A400020202020202020202020205A2D0020207F
:100A500020592D2020202020202020205A2D004504
:100A60007874727564653A200028736574206D6D22
:100A70002F732920202046776400202873746F701C
:100A800029202020202864757229002D2D2D2F2D3E
:100A90002D2D43202020202052657600202020206C
:100AA00020202000534543530045787472756465D7
:100AB000722073706565643A00206D6D2F7320009D
:100AC000546F6F6C3020746F6F20636F6C64210003
:100AD00043616E63656C004F766572726964650090
:100AE0004D6F6F64204C69676874206E6F7400707E
:100AF000726573656E7421210053656520546869C1
:100B00006E67697665727365002020207468696E6F
:100B1000673A3135333437004D6F6F643A200055F2
:100B2000702F446E2F456E7420746F2053657400CF
:100B300020202020202020202020002873657420E1
:100B400052474229005265643A00477265656E3A21
:100B500000426C75653A0055702F446E2F456E74D7
:100B600020746F2053657400436F6D706C657465FD
:100B7000643A202020302520006572726F722100B7
:100B8000546F6F6C2020202D2D2D2F2D2D2D010029
:100B9000426564202020202D2D2D2F2D2D2D01008C
:100BA000456C61707365643A202020306830306D88
:100BB0000054696D654C6566743A202030683030A9
:100BC0006D0073656373002020206E6F6E65005AA0
:100BD000506F733A20202020202020202020200049
:100BE0006D6D0046696C616D656E743A302E303003
:100BF0006D202000436F70793A2020202020202093
:100C00002020202000206F6620004163633A2020CE
:100C100020202020202020202020004D6F74686597
:100C200072626F61726420205F2E5F002020204579
:100C30007874727564657220205F2E5F00205265A3
:100C4000766973696F6E2030303836362000467210
:100C50006565205352414D2000506C6561736520DD
:100C600043686F6F73653A0041626F72742050720F
:100C7000696E74202020005072696E7420416E6F7E
:100C80007468657220005061757365206174205A24
:100C9000506F732000506175736520202020202044
:100CA0002020200050617573652C20484250206F31
:100CB0006E200050617573652C204E6F2048656171
:100CC000740052657475726E20746F204D656E7578
:100CD00000436F6E74696E7565204275696C6400BF
:100CE00053442063617264206572726F72004E6FAC
:100CF0002066696C657320666F756E64004E6F20A8
:100D000053442063617264005772697465204661C0
:100D1000696C656421004572726F720046696C658A
:100D2000206578697374732100526561642046619F
:100D3000696C65642100454550524F4D206D6179C5
:100D400020626500636F72727570740046696C652D
:100D5000206E6F7420666F756E642100457261733A
:100D6000696E672E2E2E0030303A30300055702FCD
:100D7000446E2F456E7420746F2053657400436F6A
:100D80006F6C200048656174200042656400536503
:100D90007420546F6F6C302054656D70005365740F
:100DA000204265642054656D7000546F6F6C300094
:100DB000546F6F6C3020546172672054656D703AC7
:100DC00000426564205461726765742054656D70DB
:100DD0003A00486F6D6520417869733A2000202001
:100DE000592020202020202020202020205A005878
:100DF000202020582028656E6473746F707329005A
:100E00002020592020202020202020202020205A6F
:100E10000044697361626C6500456E61626C6500D7
:100E200053746570706572204D6F746F72733A0001
:100E3000005465737420456E642053746F70733A68
:100E40002000584D696E3A4E20202020584D617880
:100E50003A4E00594D696E3A4E20202020594D617E
:100E6000783A4E005A4D696E3A4E202020205A4D55
:100E700061783A4E0059004E00456E746572696E95
:100E8000672070617573652E2E0052657472616300
:100E9000742066696C616D656E7400436C65617287
:100EA000696E67206275696C642E2E0050617573DF
:100EB00065642800293A00202020592B202020207A
:100EC00020202020205A2B00582D205265762058B3
:100ED0002B2020284677642900202020592D20200F
:100EE000202020202020205A2D0048656174696E42
:100EF000672E2E2E202020202020004C6561766950
:100F00006E672070617573652E2E2E0050617573AB
:100F100065206174205A506F733A0055702F446EEB
:100F20002F456E7420746F20536574006D6D202002
:100F30002000416476616E6365204142503A00684A
:100F40006F6C64206B65792E2E2E002020202020CF
:100F500020202020202028667764290043616C69C6
:100F600062726174653A204D6F7665200062756922
:100F70006C6420706C6174666F726D00756E74695C
:100F80006C206E6F7A7A6C652E2E2E002020202029
:100F900020202020202028636F6E7429006C696552
:100FA0007320696E2063656E7465722C00747572AF
:100FB0006E20746872656164656400726F64207588
:100FC0006E74696C2E2E2E006E6F7A7A6C65206AB4
:100FD00075737400746F75636865732E00486F6D68
:100FE000696E67205A2E2E2E00486F6D696E67203D
:100FF000592E2E2E00486F6D696E6720582E2E2EAA
:1010000000212043616C6962726174656420210073
:10101000526567656E65726174652067636F6465AC
:101020000020202020202020202028726573657455
:10103000290058204F66667365743A0059204F6640
:10104000667365743A005A204F66667365743A0099
:1010500055702F446E2F456E7420746F2053657445
:10106000005265706561742042757A7A65723A0043
:1010700028303D42757A7A6572204F6666290055A0
:10108000702F446E2F456E7420746F20536574006A
:101090002074696D6573200045787472756465729B
:1010A0002046616E3A0000526573657420546F20CB
:1010B0005A65726F3F004E6F00596573004C696648
:1010C0006574696D65204F646F2E3A0054726970C3
:1010D000204F646F6D657465723A00287472697090
:1010E000292020202872657365742900286C6966A0
:1010F000652920202028726573657429004F766564
:1011000072726964652054656D7000446974746F0F
:10111000205072696E7400416363656C2E204F6EBF
:101120002F4F666600416363656C2E2053657474AF
:10113000696E677300457874727564657220486FD4
:101140006C6400546F6F6C686561642053797374CC
:10115000656D0041425020436F70696573202853CC
:1011600044290041425020436F7069657320285321
:1011700044293A0055702F446E2F456E7420746FC9
:1011800020536574004F7665727269646520474329
:101190006F64650054656D70657261747572653A4F
:1011A00000416363656C65726174656400507269C7
:1011B0006E74696E673A004F6666004F6E00457840
:1011C00074727564657200486F6C643A004F6666AD
:1011D000004F6E00546F6F6C68656164206F6666C7
:1011E0007365740073797374656D3A004F6C6400B5
:1011F0004E657700446974746F205072696E74692B
:101200006E673A000050726F66696C653F00526508
:1012100073746F726500446973706C617920436FF9
:101220006E666967004368616E6765204E616D6533
:10123000005361766520546F2050726F66696C654B
:101240000050726F66696C65204E616D653A00559D
:10125000702F446E2F456E7420746F205365740098
:101260002000584F66663A2000594F66663A2000C3
:101270005A4F66663A20004842502054656D703AD5
:1012800020202000546F6F6C302054656D703A2020
:10129000004578747264724D4D2F733A2000466198
:1012A000696C656420746F206F70656E0066696C90
:1012B00065206F7220666F6C6465722E004E616DE2
:1012C0006520746F6F206C6F6E673F00436F6E74A4
:1012D000696E75650058204D617820416363656CC7
:1012E0003A0059204D617820416363656C3A005A99
:1012F000204D617820416363656C3A0052696768EC
:1013000074204D617820416363656C3A004C6566DA
:1013100074204D617820416363656C3A004D6178BB
:1013200020416363656C3A004D61782041636365D9
:101330006C2045787464723A004A4B4E20416476C2
:10134000616E6365204B3A004A4B4E2041647661E2
:101350006E6365204B323A0045787464722E4465A2
:101360007072696D65523A0045787464722E4465F6
:101370007072696D654C3A00536C6F77646F776E6D
:10138000456E61626C65643A004D617853706565C5
:10139000644368616E6765583A004D6178537065C3
:1013A00065644368616E6765593A004D61785370B2
:1013B0006565644368616E67655A3A004D617853AC
:1013C000706565644368616E6765523A004D617887
:1013D00053706565644368616E67654C3A0055708B
:1013E0002F446E2F456E7420746F20536574002057
:1013F00020202000456E6473746F707350726573A3
:10140000656E743A0055702F446E2F456E742074CB
:101410006F205365740020005820486F6D6520468A
:10142000656564726174653A005920486F6D652086
:1014300046656564726174653A005A20486F6D654F
:101440002046656564726174653A0055702F446E7C
:101450002F456E7420746F20536574006D6D2F6D71
:10146000696E200054686973206D656E7520636134
:101470006E006D616B6520796F757220626F74000C
:10148000696E6F70657261626C652E005072657373
:101490007320592B20746F20636F6E740053617634
:1014A000696E672E2E2E00526573746F72696E67B7
:1014B0002E2E2E002A205072657373200078206D26
:1014C0006F72652100202020202020202020202055
:1014D000202020202000454550524F4D202D3E20F9
:1014E0005344005344202D3E20454550524F4D005B
:1014F000457261736520454550524F4D004D6F6EEA
:1015000069746F72004275696C642066726F6D2039
:101510005344005072656865617400457874727553
:101520006465004275696C642053657474696E6704
:101530007300486F6D652041786973004A6F6700DA
:1015400046696C616D656E74205573656400416415
:1015500076616E636520414250005374657070651A
:101560007273004D6F6F64204C6967687400427538
:101570007A7A65720050726F66696C6573004361B8
:101580006C69627261746500486F6D65204F6666B4
:101590007365747300486F6D696E6720526174657E
:1015A000730045787472756465722046616E0054EC
:1015B00065737420456E642053746F707300506FB0
:1015C000736974696F6E0056657273696F6E00455A
:1015D0006570726F6D00554E4B4E4F574E000000B8
:1015E00000FFFFFFFF000000FF000000FF00FFFF03
:1015F000FF00FFFFFF00A020F0FFA500FFC3A5FF35
:10160000B291CDFFD2D2D0FFB4B4FFFFD0CD708A5B
:1016100090BEBEBED3D3D319197000BFFF55892F1A
:10162000228B22FFD700FF69B4F0F0E6426F7420EE
:1016300053746174757300437573746F6D205247F2
:1016400042004F6666005768697465005265640021
:10165000477265656E00426C7565004379616E0086
:101660004D6167656E74610059656C6C6F770050F1
:101670007572706C65004F72616E676500416C6DCC
:101680006F6E640050656163682050756666004D3A
:10169000696E7420437265616D00416C69636520F9
:1016A000426C7565004C6176656E646572004D69CB
:1016B00073747920526F736500536C6174652047B1
:1016C0007261790047726179004C696768742047DC
:1016D000726179004D69646E676874426C7500448C
:1016E000656570536B79426C75004F6C6976654720
:1016F0007265656E00466F727374477265656E0041
:10170000476F6C6400486F742050696E6B004C69C1
:101710006E656E0057524742005247420057686953
:101720007465466C6173680052656420466C617331
:101730006800477265656E466C61736800426C753F
:101740006520466C617368004379616E20466C6168
:101750007368004D676E7461466C6173680059650B
:101760006C6C20466C61736800426C61636B00486E
:101770007565204379636C65004D6F6F64204C691B
:101780006768740043616E646C65005761746572CC
:10179000004F6C64204E656F6E00536561736F6E11
:1017A00073005468756E64727374726D0053746F55
:1017B00070204C6967687400532E204F2E20532EE2
:1017C0000000AE32DB32673DC979877CAE95FA9571
:1017D0005FD930E0EEE2FCE185EC91E201C081935B
:1017E000EF3FF907E0F3D9F311241FBECFEFD1E2A9
:1017F000DEBFCDBF00E00CBF18E0A0E0B2E0E6EF36
:10180000FBEC01E00BBF02C007900D92AE34B107B4
:10181000D9F71CE1AEE4B8E001C01D92AE32B107C9
:10182000E1F717E1C4EDD7E100E006C02297010916
:10183000FE010BBF0E9470E5C23CD10780E00807A3
:10184000A9F70E94003E0C94F9E50C940000A0E377
:10185000B0E0EDE2FCE00C943BE5298F3A8F4B8F32
:101860005C8F6D8F7E8F8F8F98A3A98ABA8ACB8A5F
:10187000DC8AED8AFE8A0F8B188F098D1A8D2B8DCD
:101880003C8D09A31AA32BA33CA3680179018FEF18
:101890009FEFA0E0B0E0C822D922EA22FB22890112
:1018A0002227332709A71AA72BA73CA709891A893A
:1018B0002B893C890DA31EA32FA338A748015901EA
:1018C00088229922AA22BB22290166247724C501F5
:1018D000B401A70196010E94AAE46DA77EA78FA775
:1018E00098ABC301B2010E94AAE46B017C01C5015F
:1018F000B40129A53AA54BA55CA50E94AAE44B0119
:101900005C01C301B2010E94AAE4AB01BC01C80C96
:10191000D91CEA1CFB1C0DA51EA52FA538A9C901C1
:10192000AA27BB27C80ED91EEA1EFB1EC814D9045D
:10193000EA04FB0420F4405050406F4F7F4FC70132
:10194000AA27BB27840F951FA61FB71F8D839E83D1
:10195000AF83B8877601DD24CC244DA55EA56FA5A5
:1019600078A960707070C40ED51EE61EF71EC9827D
:10197000DA82EB82FC821C2D0A818B804C808D8761
:101980008E818E878F818F878885888B2D893E8970
:101990004F89588D69A17AA18BA19CA10E94AAE4CC
:1019A0006B017C012D8D3E8D4F8D58A16DA17EA1C7
:1019B0008FA198A50E94AAE4DC01CB01C80ED91E14
:1019C000EA1EFB1E8D859E85AF85B8898C0D9D1DF9
:1019D000AE1DBF1D8D879E87AF87B88B682F7E8514
:1019E000212F302F482D542D8F859889E096E0E1E6
:1019F0000C9457E50F93CF93DF93CDB7DEB7609785
:101A00000FB6F894DEBF0FBECDBF002309F456C059
:101A100029873A874B875C876D877E878F87988B6E
:101A200020E2201B8D859E85AF85B889AC01BD0164
:101A30001216B4F0770F440B542FBA014D835E8316
:101A40006F837887332727FD3095309521953F4F59
:101A500004C0B595A795979587952A95D2F722C08A
:101A6000002E04C075956795579547950A94D2F74F
:101A70004D835E836F83788704C0880F991FAA1FE8
:101A8000BB1F2A95D2F749855A856B857C8504C092
:101A900076956795579547950A95D2F7842B952BA0
:101AA000A62BB72B89839A83AB83BC8329813A8188
:101AB0004B815C816D817E818F81988560960FB6A8
:101AC000F894DEBF0FBECDBFDF91CF910F91089587
:101AD000A8E4B0E0EEE6FDE00C943AE5F50129A3B8
:101AE0003AA34BA35CA36DA37EA38FA398A7A98E53
:101AF000FA8FCB8EDC8EED8EFE8E0F8F18A38DA00D
:101B00009EA0AFA0B8A4B7FE67C02195B1E01216A1
:101B100008F0B0E03195A1E0131608F0A0E0B32E74
:101B2000BB1ABB2D882483943B1508F08824A82970
:101B3000419531E0141608F030E0B42EBA1AAB2DFE
:101B4000882483944B1508F088243829519541E066
:101B5000151608F040E0452E431A31E0541508F000
:101B600030E0432B619531E0161608F030E0862E08
:101B7000841A41E0681508F040E0342B719541E08B
:101B8000171608F040E0572F531B31E0751708F087
:101B900030E0432B819531E0181608F030E0682FD3
:101BA000641B462F61E0841708F060E0362B9195A6
:101BB000931B29A3BAA3ABA34CA28DA25EA34FA3F0
:101BC00098A78FEF9FEFAFEFBFEF25968CAF9DAF3C
:101BD000AEAFBFAF259706C025961CAE1DAE1EAE9C
:101BE0001FAE25978D8D9E8DAF8DB8A1B7FF68C0B4
:101BF00025962CAD3DAD4EAD5FAD2597209530952A
:101C00004095509525962CAF3DAF4EAF5FAF2597D1
:101C1000E19581E01E1608F080E0F19591E01F1635
:101C200008F090E04F2F481B81E0F41708F080E0A7
:101C3000982BC19481E01C1408F080E06C2D691B86
:101C400091E0C61608F090E0892BD19491E01D1424
:101C500008F090E05D2D581B81E0D51608F080E07B
:101C6000982BE19481E01E1408F080E03E2D391B92
:101C700091E0E31608F090E0892BF19491E01F14B5
:101C800008F090E02F2D281B81E0F21608F080E08C
:101C9000982B019581E0101608F080E0702F791BD9
:101CA000972F71E0091708F070E0872B1195181B2A
:101CB000E98F4A8F6B8F5C8F3D8F2E8F9F8F18A37C
:101CC000798D6A8D5B8D4C8D3D8D2E8D9F8D88A17C
:101CD000E9A1E98BEAA1EA8BEBA1EB8BECA1EC8B00
:101CE000EDA1ED8BEEA1EE8BEFA1EF8BE8A5E88FD8
:101CF00079876A875B874C873D872E879F87888B8C
:101D000089849A84AB84BC848D859E85AF85B8898F
:101D1000E988FA880B891C89EDAAFEAA0FAB18AFD7
:101D2000CD88DE88EF88F88C0097A105B10509F011
:101D3000BFC3C814D904EA04FB0408F04EC100E094
:101D4000801600E0900601E0A00600E0B00660F416
:101D50001FEF81169104A104B10409F098F480E00A
:101D600090E0A0E0B0E017C020E0821620E09206EC
:101D700020E0A20621E0B20650F480E190E0A0E06D
:101D8000B0E009C088E090E0A0E0B0E004C088E1E5
:101D900090E0A0E0B0E0B501A401082E04C0769563
:101DA0006795579547950A94D2F7FA01E45BFD4F82
:101DB000208140E250E060E070E0481B590B6A0B64
:101DC0007B0B421B510961097109411551056105E0
:101DD0007105A1F1042E04C0880C991CAA1CBB1C1F
:101DE0000A94D2F797018601042E04C0000F111F38
:101DF000221F331F0A94D2F780E290E0841B950BD8
:101E0000CDA8DEA8EFA8F8AC04C0F694E794D79468
:101E1000C7948A95D2F7C02AD12AE22AF32A0DA9BB
:101E20001EA92FA938AD04C0000F111F221F331F98
:101E30004A95D2F70DAB1EAB2FAB38AF2501662408
:101E40007724950184012070307009AB1AAB2BAB5D
:101E50003CABC701B601A30192010E94FCE42DA78F
:101E60003EA74FA758AB69A77AA78BA79CA7C70126
:101E7000B601A30192010E94FCE4CA01B90129A99B
:101E80003AA94BA95CA90E94AAE4AB01BC0109A52F
:101E90001AA52BA53CA57801DD24CC240DA91EA9EB
:101EA0002FA938ADC901AA27BB27C82AD92AEA2AEF
:101EB000FB2A0DA51EA52FA538A9C416D506E60632
:101EC000F70638F5015010402040304009A71AA706
:101ED0002BA73CA7C80CD91CEA1CFB1CC814D904AE
:101EE000EA04FB04D0F0C416D506E606F706A8F40B
:101EF0000DA51EA52FA538A9025010402040304046
:101F000009A71AA72BA73CA7C80CD91CEA1CFB1CC5
:101F100004C009A71AA72BA73CA7C41AD50AE60A2A
:101F2000F70AC701B601A30192010E94FCE42DA7A4
:101F30003EA74FA758AB69AF7AAF8BAF9CAFC70135
:101F4000B601A30192010E94FCE4CA01B90129A9CA
:101F50003AA94BA95CA90E94AAE46B017C0149AD96
:101F60005AAD6BAD7CAD9A01112700274DA95EA932
:101F70006FA978AD60707070042B152B262B372B52
:101F80008DA59EA5AFA5B8A90C151D052E053F056D
:101F9000C0F40197A109B109080D191D2A1D3B1DA7
:101FA000081519052A053B0560F00C151D052E05C1
:101FB0003F0538F48DA59EA5AFA5B8A90297A10944
:101FC000B10909A51AA52BA53CA57801DD24CC24CF
:101FD000C82AD92AEA2AFB2AB9C481149104A10487
:101FE000B10451F461E070E080E090E0A50194015B
:101FF0000E94FCE449015A0110E0811610E09106AC
:1020000011E0A10610E0B10660F42FEF82169104F2
:10201000A104B10409F098F480E090E0A0E0B0E001
:1020200017C030E0831630E0930630E0A30631E0BD
:10203000B30650F480E190E0A0E0B0E009C088E091
:1020400090E0A0E0B0E004C088E190E0A0E0B0E063
:10205000B501A401082E04C076956795579547955C
:102060000A94D2F7FA01E45BFD4F2081AC01BD0177
:10207000420F511D611D711D80E290E0A0E0B0E0B3
:10208000841B950BA60BB70B51F4C818D908EA08A6
:10209000FB08F1E04F2E512C612C712C28C1082E29
:1020A00004C0880C991CAA1CBB1C0A94D2F7970187
:1020B0008601042E04C036952795179507950A9436
:1020C000D2F709AB1AAB2BAB3CAB97018601082EBC
:1020D00004C0000F111F221F331F0A94D2F70DA74F
:1020E0001EA72FA738ABEDA8FEA80FA918AD04C0F6
:1020F00016950795F794E7944A95D2F7B801A7018A
:102100000DA51EA52FA538A9042B152B262B372B83
:102110000DA71EA72FA738ABEDA8FEA80FA918ADD5
:1021200004C0EE0CFF1C001F111F8A95D2F7EDAA08
:10213000FEAA0FAB18AF2501662477249501840110
:102140002070307009AF1AAF2BAF3CAF69A97AA9E4
:102150008BA99CA9A30192010E94FCE429A73AA79C
:102160004BA75CA76B017C0169A97AA98BA99CA9E3
:10217000A30192010E94FCE4CA01B90129AD3AAD64
:102180004BAD5CAD0E94AAE4AB01BC017601DD243D
:10219000CC240DA51EA52FA538A9C901AA27BB27A8
:1021A000C82AD92AEA2AFB2A09A51AA52BA53CA5E3
:1021B000C416D506E606F70638F501501040204053
:1021C000304009AB1AAB2BAB3CABC80CD91CEA1C9A
:1021D000FB1CC814D904EA04FB04D0F0C416D506CD
:1021E000E606F706A8F409A51AA52BA53CA50250FA
:1021F00010402040304009AB1AAB2BAB3CABC80CB5
:10220000D91CEA1CFB1C04C009AB1AAB2BAB3CABC2
:10221000C41AD50AE60AF70AC701B601A30192015A
:102220000E94FCE429A73AA74BA75CA721966CAFB4
:102230007DAF8EAF9FAF2197C701B601A301920179
:102240000E94FCE4CA01B90129AD3AAD4BAD5CADC9
:102250000E94AAE48B019C0121964CAD5DAD6EAD50
:102260007FAD2197DA01992788274DA55EA56FA537
:1022700078A960707070842B952BA62BB72B49A57D
:102280005AA56BA57CA580179107A207B307F0F4A8
:102290004150504060407040880D991DAA1DBB1DE3
:1022A00088159905AA05BB0588F080179107A20734
:1022B000B30760F449A55AA56BA57CA542505040D0
:1022C00060407040880D991DAA1DBB1D6C017D01E9
:1022D000C01AD10AE20AF30A09A91AA92BA93CA932
:1022E000380155244424442A552A662A772A850130
:1022F000222733270DA71EA72FA738AB95018401EE
:102300002070307009AF1AAF2BAF3CAFC701B601D8
:102310002DA53EA54FA558A90E94FCE429A73AA7E0
:102320004BA75CA769AB7AAB8BAB9CABC701B60183
:102330002DA53EA54FA558A90E94FCE4CA01B901EC
:1023400029AD3AAD4BAD5CAD0E94AAE4AB01BC0136
:1023500009A91AA92BA93CA97801DD24CC240DA92F
:102360001EA92FA938ADC901AA27BB27C82AD92A77
:10237000EA2AFB2A09A51AA52BA53CA5C416D50651
:10238000E606F70638F5015010402040304009AB12
:102390001AAB2BAB3CABC80CD91CEA1CFB1CC814F9
:1023A000D904EA04FB04D0F0C416D506E606F70605
:1023B000A8F409A51AA52BA53CA502501040204061
:1023C000304009AB1AAB2BAB3CABC80CD91CEA1C98
:1023D000FB1C04C009AB1AAB2BAB3CABC41AD50A2F
:1023E000E60AF70AC701B6012DA53EA54FA558A9D3
:1023F0000E94FCE429A73AA74BA75CA721966CAFE3
:102400007DAF8EAF9FAF2197C701B6012DA53EA529
:102410004FA558A90E94FCE4CA01B90129AD3AAD03
:102420004BAD5CAD0E94AAE48B019C0121964CADA2
:102430005DAD6EAD7FAD2197DA01992788274DA953
:102440005EA96FA978AD60707070842B952BA62B58
:10245000B72B49A55AA56BA57CA580179107A207A4
:10246000B307D0F44150504060407040880D991D32
:10247000AA1DBB1D88159905AA05BB0568F0801724
:102480009107A207B30740F449A55AA56BA57CA5FF
:10249000425050406040704009A91AA92BA93CA99C
:1024A0007801DD24CC24C42AD52AE62AF72A51C291
:1024B000C816D906EA06FB0608F438C2803010E0D8
:1024C000910711E0A10710E0B10758F48F3F910583
:1024D000A105B10509F090F400E010E020E030E043
:1024E00016C0803020E0920720E0A20721E0B2076A
:1024F00050F400E110E020E030E009C008E010E016
:1025000020E030E004C008E110E020E030E0AC0161
:10251000BD01002E04C076956795579547950A949E
:10252000D2F7FA01E45BFD4F4081040F111D211D1C
:10253000311D40E250E060E070E0401B510B620B47
:10254000730BA1F48C159D05AE05BF0508F4F5C10C
:10255000EDA8FEA80FA918AD442455243201E814B3
:10256000F9040A051B0508F0EBC1E3C1342E2C0168
:102570003D0104C0440C551C661C771C4A95D2F7DB
:10258000D501C401002E04C0B695A79597958795EF
:102590000A94D2F7482A592A6A2A7B2AA50194016B
:1025A000032C04C0220F331F441F551F0A94D2F777
:1025B00029AF3AAF4BAF5CAFB701A601002E04C004
:1025C00076956795579547950A94D2F749AB5AABDC
:1025D0006BAB7CABC701B601032C04C0660F771F41
:1025E000881F991F0A94D2F76DA77EA78FA798AB73
:1025F0008DA99EA9AFA9B8AD04C0B695A79597952A
:1026000087950A95D2F74DA55EA56FA578A9482BA9
:10261000592B6A2B7B2B4DA75EA76FA778AB430185
:10262000AA24BB24930182012070307021960CAF44
:102630001DAF2EAF3FAF219769A97AA98BA99CA99D
:10264000A50194010E94FCE429A73AA74BA75CA727
:102650006B017C0169A97AA98BA99CA9A5019401A8
:102660000E94FCE4CA01B90121962CAD3DAD4EADEE
:102670005FAD21970E94AAE4DC01CB017601DD2445
:10268000CC240DA51EA52FA538A9A901662777275B
:10269000C42AD52AE62AF72A09A51AA52BA53CA5FE
:1026A000C816D906EA06FB0638F50150104020404E
:1026B000304009AB1AAB2BAB3CABC40CD51CE61CB1
:1026C000F71CC414D504E604F704D0F0C816D906E4
:1026D000EA06FB06A8F409A51AA52BA53CA50250FD
:1026E00010402040304009AB1AAB2BAB3CABC40CC4
:1026F000D51CE61CF71C04C009AB1AAB2BAB3CABDA
:10270000C81AD90AEA0AFB0AC701B601A501940151
:102710000E94FCE429A73AA74BA75CA729966CAFB7
:102720007DAF8EAF9FAF2997C701B601A501940178
:102730000E94FCE4CA01B90121962CAD3DAD4EAD1D
:102740005FAD21970E94AAE44B015C0129964CAD34
:102750005DAD6EAD7FAD29979A01112700278DA53C
:102760009EA5AFA5B8A9A070B070082B192B2A2B75
:102770003B2B89A59AA5ABA5BCA5081519052A056B
:102780003B05E0F40197A109B109040D151D261DB3
:10279000371D041515052605370580F008151905A0
:1027A0002A053B0558F489A59AA5ABA5BCA50297B7
:1027B000A109B109040D151D261D371DB901A80178
:1027C000481959096A097B094DA75EA76FA778AB1D
:1027D00009A91AA92BA93CA97801DD24CC24C82A6F
:1027E000D92AEA2AFB2AFFEF8F2EFFEF9F2EA12C7A
:1027F000B12C8C209D20AE20BF20870122273327BB
:1028000009A71AA72BA73CA749AC5AAC6BAC7CAC68
:102810002FEF3FEF40E050E0422253226422752226
:1028200029AD3AAD4BAD5CAD8A012227332709AB08
:102830001AAB2BAB3CABC501B401A30192010E94C2
:10284000AAE469AF7AAF8BAF9CAFC501B40129A9E7
:102850003AA94BA95CA90E94AAE44B015C0169A5B5
:102860007AA58BA59CA5A30192010E94AAE42B0145
:102870003C0169A57AA58BA59CA529A93AA94BA9D4
:102880005CA90E94AAE4AB01BC01840C951CA61CA7
:10289000B71C09AD1AAD2BAD3CADC901AA27BB27AA
:1028A000880E991EAA1EBB1E84149504A604B704A4
:1028B00020F4405050406F4F7F4FC501AA27BB27DF
:1028C000840F951FA61FB71F0DA51EA52FA538A9FC
:1028D000081719072A073B0718F180179107A20765
:1028E000B307A1F554019924882489AD9AADABAD05
:1028F000BCADA070B070880E991EAA1EBB1E4DA95B
:102900005EA96FA978AD032C04C0440F551F661F44
:10291000771F0A94D2F7481559056A057B05B0F46C
:102920000894C108D108E108F10810C044245524D6
:102930003201CC24DD2476010CC04424552432011C
:1029400081E0C82ED12CE12CF12C03C04424552465
:102950003201FE01319688E0DF011D928A95E9F788
:10296000C982DA82EB82FC824D825E826F82788637
:102970002C2D3A814B815C81642D7E818F819885DD
:102980002596ECACFDAC0EAD1FAD2597E114F1041E
:102990000105110509F456C02195E1E0121608F071
:1029A000E0E03195F1E0131608F0F0E0032F0E1B84
:1029B000E1E0301708F0E0E0FE2B4195E1E014166D
:1029C00008F0E0E0142F1F1B31E0411708F030E061
:1029D000E32B5195F1E0151608F0F0E0B52FBE1B82
:1029E00031E05B1708F030E0F32B6195E1E016165B
:1029F00008F0E0E0462E4F1A31E0641508F030E0B0
:102A0000E32B7195F1E0171608F0F0E0A72FAE1B4D
:102A100031E07A1708F030E0F32B8195E1E01816E9
:102A200008F0E0E0F82EFF1AFF2D31E08F1508F0D6
:102A300030E0E32B9195302F412F5B2F642D7A2FBF
:102A40008F2F9E1BC85BDF4FE1E10C9456E5F89495
:102A50002091DD083091DE088091DB089091DC0840
:102A6000821B930B7894089580914D0308958823D9
:102A700029F06093990880E490E002C080E890E03B
:102A80009093D5088093D40808952091D40830916C
:102A9000D5082115310529F081E027FF03C080E02A
:102AA000089580E008958091D4089091D508089504
:102AB00081E02091D4083091D5082230310508F406
:102AC00080E00895FC01A5EEBAE024E10D900192AA
:102AD0002150E1F70895CF93DF93CDB7DEB7649728
:102AE0000FB6F894DEBF0FBECDBFDC01CB018093E3
:102AF000C2089093C308A093C408B093C508CE0140
:102B000001960E94EC6FCE01019662E070E00E9497
:102B1000B03E4091C2085091C3086091C4087091C2
:102B2000C508FC0180819181A281B381841795073A
:102B3000A607B7071CF01092C10803C081E080937C
:102B4000C10864960FB6F894DEBF0FBECDBFDF910B
:102B5000CF9108950F931F930091C2081091C3085D
:102B60002091C4083091C508B801C9011F910F9187
:102B70000895CF92DF92EF92FF920F931F93CF931E
:102B8000DF93C0914D03CC2309F478C0C53609F416
:102B900075C0D0919408CD1709F470C06091950864
:102BA00070919608809197089091980820E030E005
:102BB00040E050E00E94DFE1882309F45FC0DD239C
:102BC00009F45CC0C0909008D0909108E090920801
:102BD000F0909308C701B60120E030E040E050E0FB
:102BE0000E94DFE1882309F449C06C2F70E06D1B5F
:102BF0007109882777FD8095982F0E94BCE29B0180
:102C0000AC01C701B6010E94E3E16B017C016C2FAE
:102C100070E080E090E00E94BAE29B01AC0160E0CD
:102C200070E088EC92E40E9467E19B01AC01C7016F
:102C3000B6010E94FEE3C62E072FD82FC92F9E0192
:102C4000862F902FA32FB22FBC01CD0120E030E0C2
:102C500040E050E00E94DFE187FF04C0CC2400E0A8
:102C6000D0E0C0E09E018C2D902FA32FBC2FBC0183
:102C7000CD010E9485E28B019C0104C000E010E0C0
:102C800020E030E0B801C901DF91CF911F910F9191
:102C9000FF90EF90DF90CF9008952091DD08309164
:102CA000DE0881E02115310509F080E00895482F04
:102CB0008091DD089091DE086091DB087091DC085E
:102CC00086179707E8F42091DD083091DE0880919F
:102CD000DF089091E008820F931F0E94D5E4E091F5
:102CE000E108F091E208E80FF91F40838091DD08C8
:102CF0009091DE0801969093DE088093DD08089598
:102D000081E0EBEDF8E080870895CF9385E680932E
:102D10004D0380E090E0A0E0B0E0809395089093B0
:102D20009608A0939708B093980810929408C1E071
:102D3000C0934C038093900890939108A0939208BD
:102D4000B093930860E070E080E090E00E946B1523
:102D50001092C1081092DE081092DD081092E0086F
:102D60001092DF081092E3081092E4081092D6083F
:102D70001092D7081092D8081092D9081092D5084E
:102D80001092D4081092D0081092D1081092D20854
:102D90001092D3081092B9081092BA081092BB088A
:102DA0001092BC081092BD081092BE081092BF0885
:102DB0001092C008E1EBF8E01092B1081182128283
:102DC000138214821582168217821092A90810921B
:102DD000AA081092AB081092AC081092AD0810929D
:102DE000AE081092AF081092B008E1EAF8E0109235
:102DF000A108118212821382148215821682178210
:102E00001092FD0A1092FE0A1092FF0A1092000B17
:102E10001092F90A1092FA0A1092FB0A1092FC0A18
:102E20008EEA91E061E00E94DA99823099F48CEDAB
:102E300091E060E00E94DA99882361F0C0938F08E6
:102E40008091B4188093010B10928E0810928D0817
:102E5000CF91089510928F08F3CF6091D6087091AA
:102E6000D7088091D8089091D90808951092D60873
:102E70001092D7081092D8081092D90808956F922E
:102E80007F928F929F92AF92BF92CF92DF92EF92FA
:102E9000FF920F931F93CF93DF93CDB7DEB7649765
:102EA0000FB6F894DEBF0FBECDBF182F882321F0D8
:102EB00081E08093A00805C08091A008882309F4D0
:102EC000BFC0CE0101960E94EC6FCE01019663E077
:102ED00070E00E94B83E3C01FC0180809180A2809D
:102EE000B380113029F0CC24CA94DC2C760105C0C3
:102EF00091E0C92ED12CE12CF12C60E070E080E053
:102F000090E443E00E94786D9B01AC01C701B601DB
:102F10000E94AAE4DC01CB01880D991DAA1DBB1DEE
:102F2000F30180839183A283B383CE01019664E091
:102F300070E00E94B83E3C01FC0180809180A2803C
:102F4000B380113029F0CC24CA94DC2C760105C062
:102F500081E0C82ED12CE12CF12C60E070E080E003
:102F600090E444E00E94786D9B01AC01C701B6017A
:102F70000E94AAE4DC01CB01880D991DAA1DBB1D8E
:102F8000F30180839183A283B3838EE991E04CE2C5
:102F900051E060E070E00E943C9A0E94BAE220E0BA
:102FA00030E040E251E40E94E3E12091E2143091EC
:102FB000E3144091E4145091E5140E94FEE39B0158
:102FC000AC0160E074E284E799E40E94E3E10E94CE
:102FD00085E2162F072F882E692E80918F0888236F
:102FE00039F18091DA08882361F4CE01019664E01A
:102FF00070E00E94B83E6C01CE01019663E070E083
:103000000BC0CE01019663E070E00E94B83E6C01F7
:10301000CE01019664E070E00E94B83EFC01808120
:103020009181A281B381F60180839183A283B383CE
:10303000CE010196412F502F682D762D0E943071C0
:1030400064960FB6F894DEBF0FBECDBFDF91CF916F
:103050001F910F91FF90EF90DF90CF90BF90AF90B6
:103060009F908F907F906F9008952F923F924F92F4
:103070005F926F927F928F929F92AF92BF92CF9208
:10308000DF92EF92FF920F931F93CF93DF93CDB711
:10309000DEB7C855D0400FB6F894DEBF0FBECDBF27
:1030A000182FCE0189960E947B3ECE0145960E9444
:1030B0007B3E112309F440C0E0E7F4E180E0908119
:1030C000992309F401C2DF0111979C91992309F416
:1030D000FBC18F5FB996833091F7DE015596E5EE1F
:1030E000FAE084E101900D928150E1F7CE0145961E
:1030F00062E070E00E94B83E6C018090C71490902E
:10310000C814A090C914B090CA1482E00E942D6D1A
:1031100020E030E040EA50E40E94FEE30E9485E2B5
:10312000DC01CB01881A990AAA0ABB0AF60180823F
:103130009182A282B38270C0DE015596E5EEFAE07C
:1031400084E101900D928150E1F7CE01CD960E946D
:10315000EC6FDE019996FE01FD9684E101900D92DF
:103160008150E1F7CE01899660E070E00E94B83EA0
:10317000FC014080518062807380CE01899661E0BD
:1031800070E00E94B83EFC010081118122813381F0
:10319000CE01899662E070E068962FAF68976996D5
:1031A0003FAF69970E94B83EFC01C080D180E280A9
:1031B000F380CE01459663E070E00E94B83EFC01CA
:1031C00080809180A280B380CE01459664E070E05B
:1031D0000E94B83E00D00F92FC0180819181A281B3
:1031E000B381EDB7FEB781839283A383B483CE010D
:1031F0000196B301A20168962FAD689769963FAD1D
:1032000069970E947C3E0F900F900F900F90CE0117
:10321000019660E00E945A6F6091BD147091BE14D7
:103220008091BF149091C0140E94BCE220E030E075
:1032300040E857E30E94FEE32091B9143091BA149C
:103240004091BB145091BC140E94FEE30E9485E2A1
:1032500064966FAF649765967FAF659766968FAFFC
:10326000669767969FAF6797CE01CD960E94EC6FE9
:10327000DE019996FE01FD9684E101900D92815048
:10328000E1F7CE01899660E070E00E94B83EFC0153
:1032900080809180A280B380CE01459660E070E08E
:1032A0000E94B83EFC0180819181A281B381A50179
:1032B0009401281B390B4A0B5B0BCA01B9010E9410
:1032C000BCE22091671430916814409169145091C8
:1032D0006A140E94E3E1C62E172F482EF92ECE0164
:1032E000899661E070E00E94B83EFC018080918088
:1032F000A280B380CE01459661E070E00E94B83EA6
:10330000FC0180819181A281B381A5019401281BD8
:10331000390B4A0B5B0BCA01B9010E94BCE2209138
:1033200090143091911440919214509193140E94F2
:10333000E3E1362E272E62968FAF629763969FAF9A
:103340006397CE01899662E070E00E94B83EFC016E
:1033500080809180A280B380CE01459662E070E0CB
:103360000E94B83EFC0180819181A281B381A501B8
:103370009401281B390B4A0B5B0BCA01B9010E944F
:10338000BCE22091B9143091BA144091BB14509111
:10339000BC140E94E3E1062F872EB82EA92E8C2D97
:1033A000912FA42DBF2DBC01CD01D12EE42CA7015E
:1033B00096010E94FEE32B013C01A10162963FAD04
:1033C000629763962FAD6397852F942FA32FB22F0B
:1033D000BC01CD01C52ED42EE32EF22EA7019601FD
:1033E0000E94FEE39B01AC01C301B2010E9468E1AF
:1033F0006B017C019501802F982DA32FB22FBC016A
:10340000CD01A501182D252F342FA90198010E9467
:10341000FEE39B01AC01C701B6010E9468E10E9476
:1034200065E47B018C0180918F08882339F18091BC
:10343000DA08882361F4CE01459664E070E00E94CA
:10344000B83E4C01CE01459663E070E00BC0CE0162
:10345000459663E070E00E94B83E4C01CE0145966F
:1034600064E070E00E94B83EFC0180819181A281FD
:10347000B381F40180839183A283B3838090BD14D0
:103480009090BE14A090BF14B090C01426E0880C99
:10349000991CAA1CBB1C2A95D1F74501BB2497FC9B
:1034A000B094AB2CCE01459664964FAD649765966B
:1034B0005FAD659766966FAD669767967FAD6797C8
:1034C00020E064010E94FA72C85ADF4F0FB6F894E8
:1034D000DEBF0FBECDBFDF91CF911F910F91FF9047
:1034E000EF90DF90CF90BF90AF909F908F907F90A4
:1034F0006F905F904F903F902F9008951F93CF93C0
:10350000DF93E82FF0E043E0EE0FFF1F4A95E1F76D
:10351000EF54F74F2081318142815381648175815D
:103520008681978197FF56C02195E1E0121608F039
:10353000E0E03195F1E0131608F0F0E0132F1E1BC8
:10354000E1E0311708F0E0E0FE2B4195E1E01416D0
:1035500008F0E0E0D42FDF1B31E04D1708F030E039
:10356000E32B5195F1E0151608F0F0E0C52FCE1BC6
:1035700031E05C1708F030E0F32B6195E1E01616BE
:1035800008F0E0E0B62FBF1B31E06B1708F030E029
:10359000E32B7195F1E0171608F0F0E0A72FAE1BB2
:1035A00031E07A1708F030E0F32B8195E1E018164E
:1035B00008F0E0E0382F3F1BF32F31E08F1708F0C1
:1035C00030E0E32B9195312F4D2F5C2F6B2F7A2F0D
:1035D0008F2F9E1BDF91CF911F9108957F928F9225
:1035E0009F92AF92BF92CF92DF92EF92FF920F9392
:1035F0001F93CF93DF93E82E0E947E1AD22EC32E04
:10360000B42EA52E962E872E782EF92E191694F00C
:10361000992309F0A0C0882369F4772359F466231D
:1036200049F4552339F4442329F4332319F422238C
:1036300009F491C0EE2019F4C3EBD0E002C0C4ED50
:10364000D1E0CE0100E010E020E030E040E050E0CA
:1036500060E070E00E94E399022F0D0D11E0021767
:1036600008F010E0C30E21E0C31608F020E01C0DA6
:1036700031E01C1508F030E0232BB40E31E0B41615
:1036800008F030E02B0D41E02B1508F040E0342B22
:10369000A50E41E0A51608F040E03A0D51E03A15BC
:1036A00008F050E0452B960E51E0961608F050E0D9
:1036B000490D61E0491508F060E0562B870E61E086
:1036C000871608F060E0580D71E0581508F070E0BA
:1036D000672B780E71E0781608F070E0670D81E0D6
:1036E000671508F080E0782BF90E7F0DCE010E945F
:1036F0006E9AEE2DF0E0A3E0EE0FFF1FAA95E1F722
:10370000DF01AF55B74FEF54F74F80818C93818124
:1037100011968C931197828112968C9312978381C4
:1037200013968C931397848114968C9314978581A8
:1037300015968C931597868116968C93169787818C
:1037400017968C931797108211821282138214821B
:10375000158216821782DF91CF911F910F91FF90F2
:10376000EF90DF90CF90BF90AF909F908F907F9021
:10377000089580E00E94EE1A81E00E94EE1A0895FA
:103780001F93CF93DF93E82FF0E0B3E0EE0FFF1F1E
:10379000BA95E1F7EF55F74F20813181428153818E
:1037A000648175818681978197FF56C02195E1E0FC
:1037B000121608F0E0E03195F1E0131608F0F0E0A1
:1037C000132F1E1BE1E0311708F0E0E0FE2B4195BE
:1037D000E1E0141608F0E0E0D42FDF1B31E04D17D4
:1037E00008F030E0E32B5195F1E0151608F0F0E019
:1037F000C52FCE1B31E05C1708F030E0F32B61954C
:10380000E1E0161608F0E0E0B62FBF1B31E06B17C1
:1038100008F030E0E32B7195F1E0171608F0F0E0C6
:10382000A72FAE1B31E07A1708F030E0F32B81951B
:10383000E1E0181608F0E0E0382F3F1BF32F31E0ED
:103840008F1708F030E0E32B9195312F4D2F5C2F2F
:103850006B2F7A2F8F2F9E1BDF91CF911F91089591
:103860000F931F93CF93DF93CDB7DEB7A6970FB615
:10387000F894DEBF0FBECDBFCE0101960E9485DB5E
:1038800080918F088823C9F081E09091DA08913007
:1038900009F480E064E240E050E09E012F5F3F4F7A
:1038A00000E010E00E94F234882339F0CE01019646
:1038B00061E00E946DDB80FF15C08091DA0864E250
:1038C00040E050E09E012F5F3F4F00E010E00E947B
:1038D000F234882339F0CE01019661E00E946DDB5D
:1038E00091E080FF90E0892FA6960FB6F894DEBF96
:1038F0000FBECDBFDF91CF911F910F9108950F9310
:103900001F93CF93DF93CDB7DEB7A6970FB6F8948A
:10391000DEBF0FBECDBFCE0101960E9485DB80E0E9
:1039200063E240E050E09E012F5F3F4F00E010E077
:103930000E94F234882341F0CE01019661E00E949A
:103940006DDB91E0882309F490E0892FA6960FB6ED
:10395000F894DEBF0FBECDBFDF91CF911F910F91C5
:1039600008951092CA081092CB081092CC081092B9
:10397000CD081092C6081092C7081092C80810927D
:10398000C9081092DE081092DD081092E00810922B
:10399000DF081092E3081092E4080E942E400E9473
:1039A000B91B1092A1081092A2081092A3081092BD
:1039B000A4081092A5081092A6081092A7081092C9
:1039C000A808E9EAF8E01092A9081182128213828D
:1039D000148215821682178208950F931F93CF9336
:1039E000DF93CDB7DEB7A6970FB6F894DEBF0FBE54
:1039F000CDBFCE0101960E9485DB10929B081092EC
:103A00009A0880E060E240E050E09E012F5F3F4F67
:103A100000E010E00E94F234882349F0CE010196C4
:103A200061E00E9472DB90939B0880939A08109249
:103A30009D0810929C088EEA91E061E00E94DA995C
:103A40008230B1F481E060E240E050E09E012F5FFF
:103A50003F4F00E010E00E94F234882349F0CE018D
:103A6000019661E00E9472DB90939D0880939C0810
:103A700010929F0810929E0880E061E240E050E0C2
:103A80009E012F5F3F4F00E010E00E94F234CE0114
:103A9000019661E00E9472DB90939F0880939E08DC
:103AA000A6960FB6F894DEBF0FBECDBFDF91CF91C3
:103AB0001F910F910895FF920F931F93CF93DF9360
:103AC000CDB7DEB7A6970FB6F894DEBF0FBECDBF59
:103AD000F82ECE0101960E9485DBF0FE1BC080E02F
:103AE00063E041E050E09E012F5F3F4F00E010E0B7
:103AF0000E94F2348EEA91E061E00E94DA9982300D
:103B000049F481E063E041E050E09E012F5F3F4FC8
:103B10000E94F234F1FE0BC080E06FE141E050E022
:103B20009E012F5F3F4F00E010E00E94F234A69606
:103B30000FB6F894DEBF0FBECDBFDF91CF911F91BE
:103B40000F91FF9008950F931F93CF93DF93CDB7FD
:103B5000DEB7A6970FB6F894DEBF0FBECDBFCE017D
:103B600001960E9485DB00919A0810919B0810161F
:103B700011064CF480E063E041E050E09E012F5FCD
:103B80003F4F0E94F2348EEA91E061E00E94DA99A0
:103B9000823081F400919C0810919D081016110646
:103BA0004CF481E063E041E050E09E012F5F3F4F25
:103BB0000E94F23400919E0810919F081016110681
:103BC0004CF480E06FE141E050E09E012F5F3F4FF9
:103BD0000E94F234A6960FB6F894DEBF0FBECDBF9A
:103BE000DF91CF911F910F9108950F931F93CF9362
:103BF000DF93CDB7DEB7A6970FB6F894DEBF0FBE42
:103C0000CDBFCE0101960E9485DB80919A089091EC
:103C10009B0818161906A4F480E066E140E050E025
:103C20009E012F5F3F4F00E010E00E94F234882396
:103C300039F0CE01019661E00E946DDB8823F1F13D
:103C40008EEA91E061E00E94DA998230D9F48091A5
:103C50009C0890919D0818161906A4F481E066E16D
:103C600040E050E09E012F5F3F4F00E010E00E94D7
:103C7000F234882339F0CE01019661E00E946DDBB9
:103C80008823E1F080919E0890919F0818161906EC
:103C9000BCF480E063E240E050E09E012F5F3F4FC4
:103CA00000E010E00E94F234882351F0CE0101962A
:103CB00061E00E946DDB91E0882319F490E001C07F
:103CC00091E0892FA6960FB6F894DEBF0FBECDBF48
:103CD000DF91CF911F910F9108950F931F93CF9371
:103CE000DF93CDB7DEB7EA970FB6F894DEBF0FBE0D
:103CF000CDBFCE0101960E9485DB8091D4089091C2
:103D0000D5088534910509F496C086349105C4F42C
:103D10008234910509F43FC08334910544F4803422
:103D2000910559F18134910509F0D9C029C0833436
:103D3000910509F443C08434910509F0D0C049C00D
:103D40008238910509F4A3C0833891054CF480387A
:103D5000910509F47BC08138910509F0C0C08EC07F
:103D60008438910509F4A3C0843891050CF495C0FA
:103D70008538910509F0B3C0A0C081E490E0ABC0E4
:103D80008091F10B9091F00B891B8F7009F0A7C007
:103D900082E490E0A0C0CE0187960E94EC6FA5EE71
:103DA000BAE0FE01B79684E101900D928150E1F7EF
:103DB00081E00E943F1783E490E08DC08091F10B79
:103DC0009091F00B891B8F7009F089C084E490E01A
:103DD00082C081E00E94351885E490E09093D50878
:103DE0008093D4080E943F398530910529F00E94C4
:103DF0003F398430910511F411E001C010E0809149
:103E00009908882311F00E94ED1C112341F4809140
:103E10009908882321F0809199080E945B1D80E019
:103E20006CE041E050E09E012F5F3F4F00E010E06A
:103E30000E94F23454C08091F10B9091F00B891BD9
:103E40008F7009F04CC081E090E045C080919908E6
:103E5000882311F00E94A31D80919908882359F0AE
:103E600080E06CE041E050E09E012F5F3F4F01E0B9
:103E700010E00E94F23481E890E02DC08091990812
:103E8000882339F10E94F51D882349F122C080E082
:103E90000E94351883E890E01EC08091F10B90914C
:103EA000F00B891B8F70D9F484E890E014C080E097
:103EB0000E943F1785E890E00EC08091F10B909131
:103EC000F00B891B8F7059F41092D5081092D4080A
:103ED00006C082E890E09093D5088093D408EA96D3
:103EE0000FB6F894DEBF0FBECDBFDF91CF911F910B
:103EF0000F9108952F923F924F925F926F927F920F
:103F00008F929F92AF92BF92CF92DF92EF92FF92E9
:103F10000F931F93CF93DF93CDB7DEB7CC54D04030
:103F20000FB6F894DEBF0FBECDBF8091CE08909142
:103F3000CF0801969093CF088093CE082FE0803A67
:103F4000920708F499C21092CF081092CE08CE01C1
:103F500042966DE678E10E941491CE0142960E944D
:103F6000EEDA882309F088C2CE0142960E94E9DA8F
:103F70002D969FAF8EAF2D978430910509F047C2E3
:103F80004091C6085091C7086091C8087091C9084F
:103F90008091CA089091CB08A091CC08B091CD082F
:103FA00080509543AC40B040481759076A077B07DB
:103FB00008F062C22CC2CE01839661E00E9472DBDF
:103FC0007C0180E060E240E050E09E012D5D3F4FCB
:103FD00000E010E00E94F234882339F0CE0183968D
:103FE00061E00E9472DB1C0102C02224332480E0C5
:103FF0006EE140E050E09E012D5D3F4F00E010E09B
:104000000E94F234882339F0CE01839661E00E9449
:1040100072DB2C0102C04424552480E061E240E0C0
:1040200050E09E012D5D3F4F00E010E00E94F23411
:10403000882351F0CE01839661E00E9472DB2B96BB
:104040009FAF8EAF2B9704C02B961FAE1EAE2B9743
:10405000B70180E090E021143104C9F50E94BAE272
:1040600020E030E040E452E40E9467E120E030E0EC
:1040700040E453E40E94E3E120E030E048EC52E405
:104080000E94FEE34B016C01862F992DAC2DBD2DB6
:10409000BC01CD0120E030E048EC52E40E94FAE39C
:1040A000181634F488249924F8ECCF2EA2E4DA2EE2
:1040B000882D992DAC2DBD2DBC01CD0120E030E027
:1040C00040E050E00E94DFE187FD5BC06AC00E94D3
:1040D000BAE220E030E040E951E40E9467E16B0180
:1040E0007C01B10180E090E00E94BAE220E030E083
:1040F00040E951E40E9467E19B01AC01C701B601B0
:104100000E94E3E120E030E048EC52E40E94FEE34C
:104110004B016C01862F992DAC2DBD2DBC01CD011D
:1041200020E030E048EC52E40E94FAE3181634F440
:104130008824992478ECC72EE2E4DE2E882D992D70
:10414000AC2DBD2DBC01CD0120E030E040E050E0C1
:104150000E94DFE187FF04C088249924CC24DD2459
:10416000AA20A1F4882D992DAC2DBD2DBC01CD0127
:1041700020E030E048EC52E40E94FAE387FF0BC0F5
:1041800010C088249924CC24DD240BC088249924D1
:1041900068ECC62E04C08824992456ECC52E42E44F
:1041A000D42EB20180E090E02B962EAD3FAD2B9740
:1041B00021153105B9F50E94BAE220E030E040E473
:1041C00052E40E9467E120E030E040E952E40E94BE
:1041D000E3E120E030E048EC52E40E94FEE37B01A2
:1041E0008C01862F9F2DA02FB12FBC01CD0120E087
:1041F00030E048EC52E40E94FAE3181624F4EE246E
:10420000FF2408EC12E48E2D9F2DA02FB12FBC01AE
:10421000CD0120E030E040E050E00E94DFE187FD8A
:104220005DC069C00E94BAE220E030E040E951E49C
:104230000E9467E12B013C012B962EAD3FAD2B97E1
:10424000B90180E090E00E94BAE220E030E040E96D
:1042500051E40E9467E19B01AC01C301B2010E94DD
:10426000E3E120E030E048EC52E40E94FEE37B0111
:104270008C01862F9F2DA02FB12FBC01CD0120E0F6
:1042800030E048EC52E40E94FAE3181624F4EE24DD
:10429000FF2408EC12E48E2D9F2DA02FB12FBC011E
:1042A000CD0120E030E040E050E00E94DFE187FFF8
:1042B00004C0EE24FF2400E010E0BB20A1F48E2D0A
:1042C0009F2DA02FB12FBC01CD0120E030E048ECA4
:1042D00052E40E94FAE387FF0AC00DC0EE24FF24D7
:1042E00000E010E008C0EE24FF2408EC03C0EE2438
:1042F000FF2406EC12E4582D492D3C2D2D2D2114C0
:10430000310409F09FC02B968EAD9FAD2B9700977F
:1043100009F098C0882D992DAC2DBD2DBC01CD0183
:1043200020E030E040E050E00E94DFE118164CF55C
:1043300036C08E2D9F2DA02FB12FBC01CD0120E0C6
:1043400030E048EC52E40E94FAE387FD89C04091D6
:10435000C6085091C7086091C8087091C90880913B
:10436000CA089091CB08A091CC08B091CD0880509C
:104370009543AC40B040481759076A077B07F0F4F3
:104380006FC08E2D9F2DA02FB12FBC01CD0120E03D
:1043900030E040E050E00E94DFE118165CF42D961A
:1043A0002EAD3FAD2D972130310521F033E0A32E06
:1043B000B12C07C021E0A22EB12C03C094E0A92E9D
:1043C000B12C882D992DAC2DBD2DBC01CD014E2CCD
:1043D0005F2C602E712EA30192010E94FAE387FDEB
:1043E00002C074018601CE0101966DE678E10E945B
:1043F0001491CE010196B501502F412F0E2D1F2D86
:10440000252F342FA90198010E949CDA35C00E9403
:10441000301CA82E0E947F1CB82ECE0183960E94CD
:1044200085DB80E062E040E050E09E012D5D3F4F83
:1044300000E010E00E94F234882309F0BCCDEE24A5
:10444000FF24BFCD852F942FA32FB22FBC01CD0108
:1044500020E030E048EC52E40E94FAE387FF69CFA5
:104460002D968EAD9FAD2D978430910509F4A6CF82
:1044700082E0A82EB12CA5CFC45BDF4F0FB6F89415
:10448000DEBF0FBECDBFDF91CF911F910F91FF9087
:10449000EF90DF90CF90BF90AF909F908F907F90E4
:1044A0006F905F904F903F902F900895CF93DF9340
:1044B000FC0182819381009721F481E0818780E073
:1044C00019C08481958120813181B9010E94D5E490
:1044D000C681D781C80FD91F848195810196B90102
:1044E0000E94D5E49583848382819381019793838D
:1044F00082838881DF91CF910895EF92FF921F937D
:10450000CF93DF930F920F92CDB7DEB7BBEDEB2EBB
:10451000B8E0FB2EC7010E945622682FC7016A83AC
:104520000E945622782FC70179830E945622182FA5
:10453000C7010E945622982F6A817981812F0F909E
:104540000F90DF91CF911F91FF90EF9008951F93EF
:10455000CF93DF93CBEDD8E0CE010E945622182FE7
:10456000CE010E945622982F812FDF91CF911F916B
:1045700008958BED98E00E9456220895CF92DF9225
:10458000EF92FF920F931F93CF93DF93E82EC62FE6
:104590000E94D879882309F408C10E94D5796C015A
:1045A0000E948DDB8091DF089091E0080196609178
:1045B000DB087091DC080E94D5E4E091E108F091FD
:1045C000E208E80FF91FD081CF3F09F0DC2FC601C8
:1045D0006D2F0E94D3DB8091DF089091E008029656
:1045E0006091DB087091DC080E94D5E4E091E1085D
:1045F000F091E208E80FF91FC081C6016C2F0E94FC
:10460000D3DB8091DF089091E00803966091DB088E
:104610007091DC080E94D5E4E091E108F091E20895
:10462000E80FF91FF080EE2099F08091D608909164
:10463000D708A091D808B091D9080196A11DB11D45
:104640008093D6089093D708A093D808B093D90840
:104650008C2F8A50823080F0C43071F0C53061F008
:10466000C83051F0C93041F0C63031F0C73021F0C8
:10467000CE3011F0CF3089F4EE2029F492C00E94A0
:10468000B9220F5F04C000E0CF2DD0E02496802F28
:1046900090E08C179D0798F384C0C33009F08FC059
:1046A0000E94A33F8823B9F48091DF089091E0082D
:1046B00004966091DB087091DC080E94D5E4E091DB
:1046C000E108F091E208E80FF91F808191810097DD
:1046D00011F40E94B91B8091DF089091E0080496C4
:1046E0006091DB087091DC080E94D5E40091E1083C
:1046F0001091E208080F191FF8018081918100973D
:1047000009F185EC90E060E00E94DA998823D1F00D
:10471000C33019F0CF3189F409C0DD2319F480E8E2
:1047200090E002C081E890E06CED03C082E890E088
:104730006EE60E94DA9990E002C080E090E0F80115
:1047400091838083C0E0D0E018C08091DF08909111
:10475000E00804968C0F9D1F6091DB087091DC08C7
:104760000E94D5E4E091E108F091E208E80FF91F1A
:10477000C60160810E94D3DB2196CF1530F30E94E1
:10478000EB79EE2029F40DC00E94B9220F5F04C01E
:1047900000E0CF2DD0E02496802F90E08C179D076D
:1047A00098F30E94E87981E001C080E0DF91CF9129
:1047B0001F910F91FF90EF90DF90CF900895CF3130
:1047C00009F689CF2F923F924F925F926F927F921C
:1047D0008F929F92AF92BF92CF92DF92EF92FF9211
:1047E0000F931F93CF93DF93CDB7DEB7C95FD04050
:1047F0000FB6F894DEBF0FBECDBF8091CA0890916E
:10480000CB08A091CC08B091CD080196A11DB11D97
:104810008093CA089093CB08A093CC08B093CD089E
:104820000E947A1F0E94A33F882309F55DC0209152
:10483000DD083091DE088091DF089091E008820F5A
:10484000931F0E94D5E4E091E108F091E208E80F9F
:10485000F91F40838091DD089091DE0801969093C6
:10486000DE088093DD0804C01093E30801C011E066
:104870008091DD089091DE082091DB083091DC0802
:104880002817390711F40C9461320E941C408823C8
:1048900011F40C9461328091D0089091D108A091CC
:1048A000D208B091D3080196A11DB11D8093D00804
:1048B0009093D108A093D208B093D3080E941F40D0
:1048C000482F8091DD089091DE086091DB0870919F
:1048D000DC088617970708F4AACFC6CF8091010B92
:1048E000882311F40E94C1408091C2089091C308AE
:1048F000A091C408B091C5080097A105B10529F1A0
:104900008091C108882309F5CE0189549F4F0E94E8
:10491000EC6FCE0189549F4F62E070E00E94B03E80
:104920004091C2085091C3086091C4087091C508B5
:10493000FC0180819181A281B38184179507A6072C
:10494000B7071CF481E08093C1088091C208909160
:10495000C308A091C408B091C5080097A105B1058E
:1049600011F40C9469328091C108882311F40C94DD
:1049700069320E944515882311F00C946932CE01EA
:104980008D559F4F0E94EC6FCE018D559F4F62E079
:1049900070E00E94B03E4091C2085091C3086091FF
:1049A000C4087091C508FC0180819181A281B38106
:1049B00084179507A607B70714F40C94693260E0D2
:1049C00070E080E090E00E946B1581E00E947A39EF
:1049D0008AE890E063E00E94DA99282F8DE698E15A
:1049E00064E043E00E9462920C9494320E946D1E37
:1049F0000C9494328130910511F40C94943280918E
:104A00008D0890918E088330910581F40E94D86DB5
:104A1000882341F08FE698E00E94CBDD882331F0B7
:104A20000E94017610928E0810928D0880918D0858
:104A300090918E088130910541F40E94D86D8823B1
:104A400021F410928E0810928D0880918D0890911B
:104A50008E088230910551F48EE798E00E94CBDDFC
:104A6000882321F010928E0810928D0880918D0875
:104A700090918E088430910571F480E698E00E9450
:104A8000CBDD882321F40E94301C882321F0109272
:104A90008E0810928D0880918D0890918E08853037
:104AA000910571F480E698E00E94CBDD882321F423
:104AB0000E947F1C882321F010928E0810928D088E
:104AC00080918D0890918E088630910511F581E5D1
:104AD00098E00E94CBDD882351F080914E0881FF41
:104AE00014C08DE698E160E00E947D9112C08EE4D2
:104AF00099E10E942F9D882361F080914E0882FFEA
:104B000004C08EE499E10E94519D10928E0810928B
:104B10008D0880918D0890918E08009711F00C946B
:104B200043328091DD089091DE08009711F40C94D7
:104B300043328091DF089091E0086091DB0870912A
:104B4000DC080E94D5E4E091E108F091E208E80F6A
:104B5000F91F10811B38A1F11E3811F40C94783222
:104B60001B3911F40C948132193811F40C947432FD
:104B7000163811F40C948B321C3811F40C947432E6
:104B80001C3911F40C947432103911F40C947432F1
:104B9000133811F40C947432143811F40C947432E8
:104BA000183811F40C947432143911F40C947432D2
:104BB0000E94E655882311F00C9474320C949432C0
:104BC0008091DD089091DE088931910510F40C94F4
:104BD00043320E94B92281E090E090938E08809346
:104BE0008D080E947D22C553DF4F688379838A83B5
:104BF0009B83CB5CD0400E947D22C153DF4F6883F2
:104C000079838A839B83CF5CD0400E947D22CD52E2
:104C1000DF4F688379838A839B83C35DD0400E9482
:104C20007D224B015C010E947D226B017C010E9470
:104C30007D22C952DF4F688379838A839B83C75D56
:104C4000D04080918F08882349F08091DA0888232A
:104C500019F47501640102C0460157018091F90AF7
:104C60009091FA0AA091FB0AB091FC0AA501940167
:104C7000281B390B4A0B5B0BDA01C901192FFA2FDC
:104C8000EB2FBB0F880B982FDC01782F682F582F44
:104C90009091B1083091B2084090B3085090B40898
:104CA0006090B5087090B6080091B708B091B80848
:104CB000920F41E0921708F040E0310F21E03117E8
:104CC00008F020E0430FA1E0431708F0A0E02A2BF2
:104CD0004F0E31E04F1608F030E0240DF1E02415BE
:104CE00008F0F0E03F2B5E0EF1E05E1608F0F0E019
:104CF000A32FA50D31E0A51508F030E0F32B670ECA
:104D0000E1E0671608F0E0E0F60D31E0F61508F096
:104D100030E0E32B760E31E0761608F030E0E70D58
:104D200061E0E71508F060E0362B050F61E005173C
:104D300008F060E0300F51E0301708F050E0562BDB
:104D40008B0F580F9093B1084093B2082093B3088B
:104D5000A093B408F093B508E093B6083093B70871
:104D60005093B8088091FD0A9091FE0AA091FF0A25
:104D7000B091000BA7019601281B390B4A0B5B0B66
:104D8000DA01C901192FFA2FEB2FBB0F880B982FCF
:104D9000DC01782F682F582F9091B9083091BA080C
:104DA0004090BB085090BC086090BD087090BE0851
:104DB0000091BF08B091C008920F41E0921708F02F
:104DC00040E0310F21E0311708F020E0430FA1E06F
:104DD000431708F0A0E02A2B4F0E31E04F1608F0E1
:104DE00030E0240DF1E0241508F0F0E03F2B5E0EDA
:104DF000F1E05E1608F0F0E0A32FA50D31E0A51557
:104E000008F030E0F32B670EE1E0671608F0E0E011
:104E1000F60D31E0F61508F030E0E32B760E31E0C8
:104E2000761608F030E0E70D61E0E71508F060E085
:104E3000362B050F61E0051708F060E0300F51E0F8
:104E4000301708F050E0562B8B0F580F9093B9088D
:104E50004093BA082093BB08A093BC08F093BD0808
:104E6000E093BE083093BF085093C0088092F90ABF
:104E70009092FA0AA092FB0AB092FC0AC092FD0A34
:104E8000D092FE0AE092FF0AF092000B8091D608C1
:104E90009091D708A091D808B091D9080196A11D8A
:104EA000B11D8093D6089093D708A093D808B093EB
:104EB000D90800D00F92ADB7BEB71196CD92DD9252
:104EC000ED92FC921497CE018D5A9F4FC553DF4F40
:104ED000488159816A817B81CB5CD040C153DF4FCF
:104EE000088119812A813B81CF5CD040CD52DF4FB0
:104EF000C880D980EA80FB80C35DD0400E947C3EA0
:104F00000F900F900F900F90CE018D5A9F4FC95266
:104F1000DF4F488159816A817B81C75DD0400E9403
:104F200030710C9443320E94B92281E090E090935A
:104F30008E0880938D080E947D22C952DF4F6883BE
:104F400079838A839B83C75DD0400E947D22C352B0
:104F5000DF4F688379838A839B83CD5DD0400E9435
:104F60007D22CF51DF4F688379838A839B83C15E23
:104F7000D0400E947D224B015C010E947D22062FC1
:104F8000D72E682E592E0E947D22CB51DF4F688389
:104F900079838A839B83C55ED0400E94B922782E94
:104FA00080918F088823D9F08091DA08882339F41A
:104FB000BFEE7B2273FE0AC0E0E17E2A07C0F7EF56
:104FC0007F2274FE08C028E0722A05C0082DD92C63
:104FD0006A2C5B2C04C0802E9D2CA62CB52C8D82B7
:104FE0009E82AF82B8860987DA866B865C86E1EBA3
:104FF000F8E0AE014B5F5F4FCD52DF4F59834883DE
:10500000C35DD04089EF9AE0C553DF4F9983888311
:10501000CB5CD040A3E0B0E0C153DF4FB983A8839D
:10502000CF5CD040272D30E0C552DF4F3983288335
:10503000CB5DD040C151DF4F7882CF5ED040C051B0
:10504000DF4F8882C05FD040CF50DF4F9882C15F72
:10505000D040CD50DF4FA882C35FD0402B2C302EE4
:105060004D2CCC50DF4F6882C45FD040C552DF4F1B
:1050700088819981CB5DD040C153DF4F0880CF5CE0
:10508000D04002C0959587950A94E2F7CD52DF4F44
:10509000A881B981C35DD04080FF7DC04D915D91F5
:1050A0006D917C91152FD62EC72EDB01CA01BB0F47
:1050B000880B982FDC01B82EA82E982E782E808190
:1050C000E1800281B381A481358126818780982F78
:1050D000940FFF24F394981708F0FF241E0D81E02D
:1050E0001E1508F080E0F10EEE24E394F11608F0AE
:1050F000EE248E29D00E11E0D01608F010E08D0DB0
:1051000001E08D1508F000E0102BCB0E01E0CB166E
:1051100008F000E01C0DB1E01C1508F0B0E00B2B0E
:10512000BA0EB1E0BA1608F0B0E00B0DA1E00B1515
:1051300008F0A0E0BA2BA30EA1E0A31608F0A0E0AF
:10514000BA0D31E0BA1508F030E0A32B920E31E031
:10515000921608F030E0A90D21E0A91508F020E032
:10516000322B870C380D9083F18282831383048362
:10517000B583A6833783C553DF4FA881B981CB5C44
:10518000D0400D911D912D913C911397040F151F47
:10519000261F371F97C00D911D912D913C91C5532E
:1051A000DF4FA881B981CB5CD0404D915D916D916D
:1051B0007C91D901C801841B950BA60BB70BAC01E0
:1051C000BD01C52EB62EA72EBB0F880B982FDC0174
:1051D000982E882E782EC751DF4F8883C95ED04025
:1051E000D080E180F280B381A4819581868167803F
:1051F000C351DF4F6882CD5ED0404D0D51E04D155B
:1052000008F050E0CE0C61E0CE1408F060E05C0DD8
:1052100071E05C1508F070E0672BBF0C71E0BF1403
:1052200008F070E06B0DFF24F3946B1508F0FF2479
:105230007F29AB0EFF24F394AB1608F0FF247A0D00
:10524000B1E07A1508F0B0E0FB2A9A0EB1E09A16A8
:1052500008F0B0E0F90CA1E0F91408F0A0E0BA2BD6
:10526000890EA1E0891608F0A0E0B80D91E0B8150C
:1052700008F090E0A92B982F970DEE24E39498174F
:1052800008F0EE24A90F81E0A91708F080E0E82AD1
:10529000C351DF4F8881CD5ED040C751DF4F78804A
:1052A000C95ED040870DE80E4083518362837383CB
:1052B000F482B583A683E782C553DF4FA881B98105
:1052C000CB5CD0400D931D932D933C931397C1530A
:1052D000DF4F28813981CF5CD0402F5F3F4FC153D2
:1052E000DF4F39832883CF5CD0403896CD52DF4FD3
:1052F00048815981C35DD0404C5F5F4FCD52DF4F35
:1053000059834883C35DD040C553DF4F888199815D
:10531000CB5CD0400496C553DF4F99838883CB5C28
:10532000D0402530310509F0A1CEC151DF4F788042
:10533000CF5ED040C051DF4F8880C05FD040CF509B
:10534000DF4F9880C15FD040CD50DF4FA880C35F52
:10535000D040B22CCC50DF4F6880C45FD0408091E9
:10536000D6089091D708A091D808B091D908019695
:10537000A11DB11D8093D6089093D708A093D8089B
:10538000B093D90800D00F92EDB7FEB73196ADB704
:10539000BEB711963C92418262825382CE01CF9673
:1053A000C952DF4F488159816A817B81C75DD040F6
:1053B000C352DF4F088119812A813B81CD5DD040E6
:1053C000CF51DF4FC880D980EA80FB80C15ED040DA
:1053D0000E947C3E0F900F900F900F90CE01CF96C1
:1053E000CB51DF4F488159816A817B81C55ED040B6
:1053F000272D0E94FC710C9443320E94B92281E057
:1054000090E090938E0880938D080E947D22C9526F
:10541000DF4F688379838A839B83C75DD0400E9476
:105420007D22C352DF4F688379838A839B83CD5D5E
:10543000D0400E947D22CF51DF4F688379838A83D9
:105440009B83C15ED0400E947D224B015C010E9483
:105450007D22062F672E582E492E0E947D22CB5189
:10546000DF4F688379838A839B83C55ED0400E9427
:10547000B922182F2FE7722E78220E947D22C75161
:10548000DF4F688379838A839B83C95ED0400E9403
:10549000A722C351DF4F99838883CD5ED04080918E
:1054A0008F088823E9F08091DA08882341F49FE689
:1054B000792E712273FE0BC0B0E17B2A08C087E70A
:1054C000782E712274FE08C0E8E07E2A05C0082DFF
:1054D000692C5A2C4B2C04C0802E962CA52CB42C55
:1054E0008D829E82AF82B88609876A865B864C86EB
:1054F000E1EBF8E09E012B5F3F4FCD52DF4F398348
:105500002883C35DD04049EF5AE0C553DF4F59832C
:105510004883CB5CD04083E090E0C153DF4F998358
:105520008883CF5CD040A72DB0E0CF50DF4FB98348
:10553000A883C15FD040CD50DF4F7882C35FD04099
:10554000CC50DF4F8882C45FD040CB50DF4F988271
:10555000C55FD0401501C750DF4F0883C95FD040F9
:10556000CF50DF4F88819981C15FD040C153DF4F59
:105570000880CF5CD04002C0959587950A94E2F7E9
:10558000CD52DF4FA881B981C35DD04080FF83C079
:105590004D915D916D917C91152FD62EC72EDB011B
:1055A000CA01BB0F880B982FDC01B82EA82E982EAD
:1055B000782E8081E1800281B381A48135812681AA
:1055C0008780982F940FFF24F394981708F0FF24F6
:1055D0001E0D81E01E1508F080E0F10EEE24E3942C
:1055E000F11608F0EE248E29D00E11E0D01608F046
:1055F00010E08D0D01E08D1508F000E0102BCB0EB2
:1056000001E0CB1608F000E01C0DB1E01C1508F01D
:10561000B0E00B2BBA0EB1E0BA1608F0B0E00B0DFB
:10562000A1E00B1508F0A0E0BA2BA30EA1E0A31691
:1056300008F0A0E0BA0D31E0BA1508F030E0A32B75
:10564000920E31E0921608F030E0A90D21E0A91584
:1056500008F020E0322B272D280D320F9083F182A5
:10566000828313830483B583A6833783C553DF4FB7
:10567000A881B981CB5CD0400D911D912D913C91B9
:105680001397040F151F261F371F0D931D932D937E
:105690003C931397A1C0CD90DD90ED90FC90C55345
:1056A000DF4FA881B981CB5CD0404D915D916D9168
:1056B0007C91D701C601841B950BA60BB70BAC01DF
:1056C000BD01052FB62EA72EBB0F880B982FDC012E
:1056D000982E882EC552DF4F8883CB5DD040C151B4
:1056E000DF4F8883CF5ED0401081B181A2813381AA
:1056F0002481958186817780C051DF4F7882C05F99
:10570000D040410F51E0411708F050E00B0F61E02D
:105710000B1708F060E0500F71E0501708F070E0D0
:10572000672BBA0E71E0BA1608F070E06B0DA1E0BD
:105730006B1508F0A0E07A2BA30EA1E0A31608F0E9
:10574000A0E07A0D31E07A1508F030E0A32B920E3C
:1057500031E0921608F030E0A90D21E0A91508F01B
:1057600020E0322B890E21E0891608F020E0380D68
:1057700091E0381508F090E0292BC552DF4F988151
:10578000CB5DD040980FB1E0981708F0B0E0290F3A
:1057900081E0291708F080E0B82BC051DF4F8881E5
:1057A000C05FD040C151DF4F9881CF5ED040890F9C
:1057B000B80F4083518362837383A4833583268328
:1057C000B783C553DF4FA881B981CB5CD040CD9260
:1057D000DD92ED92FC921397C153DF4F28813981FE
:1057E000CF5CD0402F5F3F4FC153DF4F39832883B9
:1057F000CF5CD0403896CD52DF4F48815981C35D90
:10580000D0404C5F5F4FCD52DF4F59834883C35D1B
:10581000D040C553DF4F88819981CB5CD04004963E
:10582000C553DF4F99838883CB5CD0402530310549
:1058300009F096CECC50DF4F8880C45FD040CB506B
:10584000DF4F9880C55FD0405101C750DF4F0881BE
:10585000C95FD040CD50DF4F7880C35FD04080918A
:10586000D6089091D708A091D808B091D908019690
:10587000A11DB11D8093D6089093D708A093D80896
:10588000B093D90800D00F92EDB7FEB73196ADB7FF
:10589000BEB711960C93618252824382CE018B96E1
:1058A000C952DF4F488159816A817B81C75DD040F1
:1058B000C352DF4F088119812A813B81CD5DD040E1
:1058C000CF51DF4FC880D980EA80FB80C15ED040D5
:1058D0000E947C3E0F900F900F900F90CE018B9600
:1058E000CB51DF4F488159816A817B81C55ED040B1
:1058F000272DC751DF4FE880F9800A811B81C95EDF
:10590000D040C351DF4FC880D980CD5ED0400E94C7
:10591000FA72B9C50E94B9220E94B9228093DA08AE
:105920004091D6085091D7086091D8087091D90855
:105930004F5F5F4F6F4F7F4F4093D6085093D7080C
:105940006093D8087093D9080E9435758091DA0861
:105950000E94817C98C58091CA089091CB08A09143
:10596000CC08B091CD088093C6089093C708A09347
:10597000C808B093C9088091DD089091DE08823094
:10598000910508F480C50E94B9220E94B922409175
:10599000D6085091D7086091D8087091D9084F5F08
:1059A0005F4F6F4F7F4F4093D6085093D708609357
:1059B000D8087093D90890918F08992361F090913D
:1059C000DA08992329F48F7E83FF05C0806103C024
:1059D000877F84FD8860F82EFF1CFF24FF1CCC24E9
:1059E000DD24082F10E0C8010C2C02C09595879586
:1059F0000A94E2F780FF04C08C2D6F2D0E941C7565
:105A00000894C11CD11CB5E0CB16D10461F73BC58D
:105A10001C3809F077C08091DD089091DE0885314F
:105A2000910508F430C50E94B9220E947D222B0105
:105A30003C010E947D22C553DF4F688379838A83AE
:105A40009B83CB5CD0400E947D226B017C010E9435
:105A50007D224B015C010E947D229B0140918F08B9
:105A6000442349F04091DA08442319F49401C50114
:105A700002C04B015C018092F90A9092FA0AA0924E
:105A8000FB0AB092FC0AEDEFFAE02093FD0A3183A5
:105A9000828393834091D6085091D7086091D808AB
:105AA0007091D9084F5F5F4F6F4F7F4F4093D6087B
:105AB0005093D7086093D8087093D90800D00F92FC
:105AC000EDB7FEB73196ADB7BEB711962C933183C3
:105AD00082839383CE0181579F4FB301A201C553A7
:105AE000DF4F088119812A813B81CB5CD0400E9425
:105AF0007C3E0F900F900F900F90CE0181579F4FDB
:105B000060E06DC21538A1F58091DD089091DE0846
:105B10008530910508F4B7C482E090E090938E0838
:105B200080938D080E94B9220E947D22AB01BC01A6
:105B30008091D6089091D708A091D808B091D90843
:105B40000196A11DB11D8093D6089093D708A0930C
:105B5000D808B093D908CB01BA0128EE33E040E071
:105B600050E00E94AAE4AB01BC018EE798E048C176
:105B7000143909F03EC08091DD089091DE0885302F
:105B8000910508F480C40E94B9220E94B922809332
:105B90004F08109250080E94A7228C010E94B9223F
:105BA00080934E080115110581F0B80180E090E066
:105BB00020E432E44FE050E00E94AAE4AB01BC01D3
:105BC00081E598E00E94A5DD0DC0CE014C960E94B3
:105BD000A1DDA1E5B8E0FE017C968FE001900D9279
:105BE0008150E1F760914F08709150088EE499E17F
:105BF00078C0153909F07EC08091DD089091DE08EB
:105C00008630910508F43FC40E94B9220E94B9224F
:105C1000082F0E94B922D82E0E94B922E82E0E9495
:105C2000B922F82E10E000FD04C087EB98E10E9435
:105C30003BCDD092B918E092BA1887EB98E16BEDA2
:105C400078E00E94C4CC01FF08C28EE499E10E9472
:105C5000399D882329F48EE499E10E943C9D04C07B
:105C600087EB98E10E9486CD04701070FF2041F010
:105C70000115110529F487EB98E16F2D0E9470CD75
:105C80000115110509F4E9C1FF2089F06F2D70E0BD
:105C900080E090E020E432E44FE050E00E94AAE48B
:105CA000AB01BC0181E598E00E94A5DD0DC0CE01ED
:105CB0000D960E94A1DDA1E5B8E0FE013D968FE0C2
:105CC00001900D928150E1F780E090E190935008AF
:105CD00080934F0884E080934E088EE499E160E061
:105CE00070E10E942B9D86E090E090938E08809357
:105CF0008D08B3C1812F8358823008F046C080914F
:105D0000DD089091DE088830910508F4BCC30E943C
:105D1000B9220E94B922082F0E947D226B017C01CA
:105D20000E94A7224091D6085091D7086091D808C8
:105D30007091D9084F5F5F4F6F4F7F4F4093D608E8
:105D40005093D7086093D8087093D90823E030E0C7
:105D500030938E0820938D08BC0180E090E020E411
:105D600032E44FE050E00E94AAE4AB01BC018FE6B0
:105D700098E00E94A5DD81E0143809F080E0602FF2
:105D8000A70196010E9490747EC31738E1F58091B7
:105D9000DD089091DE088630910508F474C384E034
:105DA00090E090938E0880938D080E94B9220E9403
:105DB000B9228093DA080E94A7220E94A72240916C
:105DC000D6085091D7086091D8087091D9084F5FD4
:105DD0005F4F6F4F7F4F4093D6085093D708609323
:105DE000D8087093D908BC0180E090E020E432E448
:105DF0004FE050E00E94AAE4AB01BC0180E698E0CD
:105E00000E94A5DD40C31D3899F48091DD08909172
:105E1000DE088630910508F436C385E090E0909363
:105E20008E0880938D080E94B9220E94B922C3CFA8
:105E30001F3809F056C08091DD089091DE0882304D
:105E4000910508F420C30E94B9220E94B922409112
:105E5000D6085091D7086091D8087091D9084F5F43
:105E60005F4F6F4F7F4F4093D6085093D708609392
:105E7000D8087093D90800E610E0CC24DD24E82E81
:105E8000FF24C7010C2C02C0959587950A94E2F770
:105E900080FF1DC0CE0185589F4F0E94EC6FCE0140
:105EA00085589F4FB6010E94B03EFC0180819181D0
:105EB000A281B38189839A83AB83BC83F894CE019A
:105EC0000196B80144E050E00E94E1E5789408941E
:105ED000C11CD11C0C5F1F4FF5E0CF16D10489F611
:105EE000D2C2103909F07EC08091DD089091DE08A1
:105EF0008230910508F4C7C20E94B9220E94B922DB
:105F0000E82E8091D6089091D708A091D808B0913A
:105F1000D9080196A11DB11D8093D6089093D7088A
:105F2000A093D808B093D9088E0109591F4FC80112
:105F30000E94EC6F20E6A22EB12CCC24DD24FF249D
:105F4000212FC5015701E02E8C01F22EC5010C2C2A
:105F500002C0959587950A94E2F780FF0BC0F894EC
:105F6000C701B6010E94B83EB80144E050E00E946B
:105F7000C9E578940894C11CD11C0C5F1F4F25E023
:105F8000C216D10419F7CE0189599F4F63E070E022
:105F90000E94B83EFC0180819181A281B3818093EF
:105FA000F90A9093FA0AA093FB0AB093FC0ACE0177
:105FB00089599F4F64E070E00E94B83EFC018081E7
:105FC0009181A281B3818093FD0A9093FE0AA093F0
:105FD000FF0AB093000BCE0189599F4F61E00E94E8
:105FE0005A6F51C2123909F04CC08091DD0890916E
:105FF000DE088630910508F446C20E94B9220E944C
:10600000B922C850DF4F8883C85FD0400E94B922B0
:10601000C950DF4F8883C75FD0400E94B922CA5061
:10602000DF4F8883C65FD0400E94B922082F0E94AC
:10603000B9228DE698E1C850DF4F6881C85FD04033
:10604000C950DF4F4881C75FD040CA50DF4F288119
:10605000C65FD040EE240E9427928091D60890918E
:10606000D708A091D808B091D9080196A11DB11DFB
:106070008093D6089093D708A093D808B093D908F6
:1060800002C2133969F58091DD089091DE088630EF
:10609000910508F4F8C10E94B9220E94A722C850B5
:1060A000DF4F8883C85FD0400E94A722C950DF4FCE
:1060B0008883C75FD0400E94B922282FC850DF4F85
:1060C0006881C85FD040C950DF4F4881C75FD0406A
:1060D0008DE698E1662309F003C10E94BA92BDCF14
:1060E000183809F074C08091DD089091DE08843082
:1060F000910508F4C8C18091DF089091E0082091D3
:10610000DB083091DC08C090E108D090E208E09113
:10611000DD08F091DE080396B9010E94D5E48C0DEC
:106120009D1DDC018C918C5F90E0E817F90708F465
:10613000AAC110914C0380918F08882329F0112364
:1061400019F010924C0303C081E080934C038091BE
:10615000DF089091E0080296B9010E94D5E48C0D09
:106160009D1DFC018081833089F08091DF08909132
:10617000E0080296B9010E94D5E48C0D9D1DDC015A
:106180008C918C3019F081E080934C03E0914C03AA
:10619000EE2399F44091DF085091E0084F5F5F4F84
:1061A000CA01B9010E94D5E48C0D9D1D61E0DC019E
:1061B0008C91882319F060E001C06FEF8E2F0E9450
:1061C000BE22882309F05FC110934C035CC11639CD
:1061D00009F055C08091DD089091DE08833091056B
:1061E00008F451C10E94B9220E94B92280934D0344
:1061F000882331F1609195087091960880919708F5
:106200009091980820E030E040E050E00E94DFE10B
:106210008823B1F480919408882391F48DE698E165
:106220000E946890DC01CB018093950890939608BA
:10623000A0939708B093980880914D038093940899
:1062400080914D038823C1F08DE698E10E9468900B
:1062500020919508309196084091970850919808A0
:106260000E9467E1DC01CB01809390089093910834
:10627000A0939208B09393080E94B922EECE1739EA
:1062800091F58091DD089091DE088230910508F447
:10629000FAC00E94B9220E94B922882351F48AE8E8
:1062A00090E063E00E94DA99282F8DE698E166E09D
:1062B00016C0813059F48AE890E063E00E94DA99D0
:1062C000282F8DE698E164E043E00AC08AE890E078
:1062D00063E00E94DA99282F8DE698E168E041E0BA
:1062E0000E946292BACE183951F58091DD089091E2
:1062F000DE088230910508F4C6C00E94B9220E94CF
:10630000B9228091D6089091D708A091D808B09171
:10631000D9080196A11DB11D8093D6089093D70886
:10632000A093D808B093D908F89481E00E94A334D0
:1063300078948DE698E160E00E947D91A4C01939BF
:1063400021F58091DD089091DE088530910508F4F3
:106350009AC00E94B9220E947D228091D608909115
:10636000D708A091D808B091D9080196A11DB11DF8
:106370008093D6089093D708A093D808B093D908F3
:106380008BED98E00E94AC397EC01A3919F58091E6
:10639000DD089091DE088230910508F474C00E94F7
:1063A000B9220E94B9224091D6085091D708609135
:1063B000D8087091D9084F5F5F4F6F4F7F4F409360
:1063C000D6085093D7086093D8087093D9080E94D4
:1063D000C93A59C01C3939F58091DD089091DE0821
:1063E0008230910508F44FC00E94B9228091D608EE
:1063F0009091D708A091D808B091D9080196A11D15
:10640000B11D8093D6089093D708A093D808B09375
:10641000D9080E94B92291E0813009F090E0892FDB
:106420000E94327530C01D3971F58091DD08909160
:10643000DE088531910538F10E94B9228091D60895
:106440009091D708A091D808B091D9080196A11DC4
:10645000B11D8093D6089093D708A093D808B09325
:10646000D9080E94B9220E94B9220E94B9220E9432
:106470007D220E94A7220E94A7220E947D220E94C4
:106480007D220E94B9228091D6089091D708A091D0
:10649000D808B091D9088130EAEC9E07EAE9AE0746
:1064A000EBE3BE0708F440C081E09AECAAE9BBE345
:1064B0008093D6089093D708A093D808B093D908B2
:1064C00033C00E941C40882311F40C946E240C9459
:1064D00074248091D4089091D5088230910510F4ED
:1064E0000C94FA240C94F624193809F091CA33CA92
:1064F0008091DD089091DE088A31910520F20C949C
:1065000093278091DD089091DE088032910508F490
:10651000BACF0C94FD298091DD089091DE0882307D
:10652000910508F0F7C9AFCFC750DF4F0FB6F89409
:10653000DEBF0FBECDBFDF91CF911F910F91FF90B6
:10654000EF90DF90CF90BF90AF909F908F907F9013
:106550006F905F904F903F902F90089580E092E071
:106560009093DC088093DB081092DE081092DD081F
:106570001092E0081092DF0885EE98E09093E20810
:106580008093E1081092E3081092E40885EE9AE007
:106590000E947B3E8EE798E00E94A1DD8FE698E0A6
:1065A0000E94A1DD80E698E00E94A1DD81E598E0EF
:1065B0000E94A1DD089582E09BE00E9485DB0895A2
:1065C000CF93DF93CDB7DEB72C970FB6F894DEBF2D
:1065D0000FBECDBF19821A821B821C821D821E82B1
:1065E0001F82188619861A861B861C86CE01019684
:1065F00060EB71E04CE050E00E94E1E52C960FB6B4
:10660000F894DEBF0FBECDBFDF91CF910895CF9339
:10661000DF93CDB7DEB728970FB6F894DEBF0FBE75
:10662000CDBF81EC93E29E838D838CED9CEA9887AD
:106630008F83CE01019665EE71E044E050E00E9448
:10664000C9E529813A818D819E812817390739F45E
:106650002B813C818F8198852817390741F0CE0125
:10666000059665EE71E044E050E00E94E1E5289671
:106670000FB6F894DEBF0FBECDBFDF91CF91089566
:106680000F931F9380E890E06CED0E94EBE581E8AA
:1066900090E06CED0E94EBE582E890E06EE60E94EF
:1066A000EBE583E890E061E00E94EBE584E890E0B0
:1066B00061E00E94EBE585E890E060E00E94EBE598
:1066C00086E890E06FEF0E94EBE587E890E06FEFDF
:1066D0000E94EBE588E890E06FEF0E94EBE589E827
:1066E00090E060E00E94EBE58AE890E063E00E94C1
:1066F000EBE58BE890E000EC1DE621ED37E94DE697
:1067000050E060E070E00E946E9A83E990E021ED35
:1067100037E94DE650E060E070E00E946E9A8BE948
:1067200090E000E010E22AE439EA41ED51E060E057
:1067300070E00E946E9A83EA90E005EE1EEB2DEA6F
:1067400036EF44E750E060E070E00E946E9A8BEA1A
:1067500090E02DEA36EF44E750E060E070E00E9400
:106760006E9A83EC90E061E00E94EBE585EC90E0AE
:1067700060E00E94EBE586E291E061E00E94EBE5DB
:1067800087E291E040E757E160E070E00E94959A6F
:106790008BE291E040E757E160E070E00E94959A5B
:1067A0008FE291E040EC53E060E070E00E94959A47
:1067B00083E391E040E757E160E070E00E94959A42
:1067C00087E391E040E757E160E070E00E94959A2E
:1067D0008BE391E044EF51E060E070E00E94959A15
:1067E0008FE391E044EF51E060E070E00E94959A01
:1067F00083E491E046E950E060E070E00E94959A01
:1068000087E491E040E157E260E070E00E94959AF1
:1068100086EA91E040E157E260E070E00E94959ADC
:106820008BE491E040ED57E060E070E00E94959AC3
:106830008FE491E040EA5FE060E070E00E94959AAA
:106840008FE591E040E951E060E070E00E94959AA8
:1068500087E691E04CEB52E060E070E00E94959A90
:1068600083E791E060E00E94EBE584E791E065E278
:106870000E94EBE585E791E044EF51E060E070E0D5
:106880000E94959A89E791E044EF51E060E070E062
:106890000E94959A8DE791E044EF51E060E070E04E
:1068A0000E94959A85E891E048E050E060E070E051
:1068B0000E94959A8AEA91E048E050E060E070E03A
:1068C0000E94959A89E891E061E00E94EBE582E9F7
:1068D00091E04CE251E060E070E00E94959A86E918
:1068E00091E04CE251E060E070E00E94959A8AE904
:1068F00091E044E650E060E070E00E94959A8EE9F5
:1069000091E04CE251E060E070E00E94959A82EAEA
:1069100091E04CE251E060E070E00E94959A8CEDCD
:1069200091E060E00E94EBE589EE91E060E00E947A
:10693000EBE58AEE91E061E00E94EBE50E9407330F
:106940001F910F9108950F931F93CF93C82F82E04B
:1069500090E062E00E94EBE583E090E06FE10E944E
:10696000EBE580E290E060E00E94EBE584E790E0F8
:1069700060E00E94EBE58EEA91E061E00E94EBE5C9
:106980000E944033CC2351F583EB90E000E010E00F
:1069900020E030E040E050E060E070E00E946E9A5D
:1069A00084ED91E020E030E040E050E060E070E015
:1069B0000E946E9A8BEB90E020E030E040E050E0E7
:1069C00060E070E00E946E9A8DED91E020E030E092
:1069D00040E050E060E070E00E946E9ACF911F911D
:1069E0000F9108956F927F928F929F92AF92BF9274
:1069F000CF92DF92EF92FF920F931F93CF93DF938B
:106A0000CDB7DEB72F970FB6F894DEBF0FBECDBF60
:106A1000782E662E4A015901F02EE12E8E010F5F6D
:106A20001F4FC8010E94A1DDC80142E350E060E0B1
:106A300070E00E94A5DDC02E012F07C08C2D902F85
:106A40000E94CBDD882309F058C00E94D8798823A2
:106A5000A9F30E94D5798C010E94D2796C01C801FA
:106A60000E948DDBC5010E948DDBC801672D0E944D
:106A7000D3DBC801662D0E94D3DB81E08816910428
:106A800031F4C8016F2D7E2D0E94D6DB08C0E2E0F4
:106A90008E16910421F4C8016F2D0E94D3DB0E9451
:106AA000EB790E94E87902C00E94477A0E94427AFC
:106AB0008823D1F3F60182A18430F9F000E009C007
:106AC000C601602F0E946DDB682FC5010E94D3DBD9
:106AD0000F5FF6018081081798F3C50160E00E94FE
:106AE0006DDB282F30E081E890E0282739272F77C9
:106AF000307081E02115310509F080E02F960FB646
:106B0000F894DEBF0FBECDBFDF91CF911F910F91E3
:106B1000FF90EF90DF90CF90BF90AF909F908F90BD
:106B20007F906F900895CF92DF92EF92FF920F9334
:106B30001F93CF93DF93EC018B0188818823E1F1D0
:106B40006E01CE0160E00E946DDB87FF35C00E94C0
:106B5000A63F882331F0CE010E94A93FC80161E819
:106B600006C00E94A33F882329F0C8016AE80E945A
:106B7000D3DB20C0F894C8810E9427152C2F30E069
:106B80008217930748F411C0C6016C2F0E946DDB79
:106B90000E945716219603C0C0E0D0E07901CE15BF
:106BA000DF0594F3C80161E802C0C80162E80E94F1
:106BB000D3DB789481E001C080E0DF91CF911F9119
:106BC0000F91FF90EF90DF90CF9008950F931F9358
:106BD000CF93DF93CDB7DEB764970FB6F894DEBFDF
:106BE0000FBECDBF8B01F894CE01019660E070E03E
:106BF0000E948A70C80161E80E94D3DBCE01019631
:106C000060E070E00E94B03EFC01408151816281F1
:106C10007381C8010E94ECDBCE01019661E070E057
:106C20000E94B03EFC014081518162817381C801A4
:106C30000E94ECDBCE01019662E070E00E94B03E63
:106C4000FC014081518162817381C8010E94ECDBAB
:106C50000E944475682FC8010E94D3DB7894649623
:106C60000FB6F894DEBF0FBECDBFDF91CF911F915D
:106C70000F9108950F931F93CF93DF93CDB7DEB796
:106C800064970FB6F894DEBF0FBECDBF8B01F894AA
:106C9000CE01019660E070E00E948A70C80161E850
:106CA0000E94D3DBCE01019660E070E00E94B03E0E
:106CB000FC014081518162817381C8010E94ECDB3B
:106CC000CE01019661E070E00E94B03EFC0140817F
:106CD000518162817381C8010E94ECDBCE01019673
:106CE00062E070E00E94B03EFC014081518162810F
:106CF0007381C8010E94ECDBCE01019663E070E075
:106D00000E94B03EFC014081518162817381C801C3
:106D10000E94ECDBCE01019664E070E00E94B03E80
:106D2000FC014081518162817381C8010E94ECDBCA
:106D30000E944475682FC80170E00E94D6DB7894E9
:106D400064960FB6F894DEBF0FBECDBFDF91CF9132
:106D50001F910F910895DF92EF92FF920F931F936F
:106D6000CF93DF93CDB7DEB7A0970FB6F894DEBF11
:106D70000FBECDBF8C017B01CB0161E80E94D3DB4C
:106D8000C80161E00E946DDB882361F00E94974298
:106D9000BC01009739F08630910521F0C7010E94AF
:106DA000D3DB27C0CE0102966FE1AE014F5F5F4F8C
:106DB0000E942E428A818E3249F48981882391F380
:106DC0008B818E3279F78C81882361F7C70160E06F
:106DD0000E94D3DB8E010E5F1F4F2FE1D22EF801F0
:106DE00061918F01662329F0C7010E94D3DBDA94F9
:106DF000B1F7C70160E00E94D3DBA0960FB6F8940C
:106E0000DEBF0FBECDBFDF91CF911F910F91FF90DD
:106E1000EF90DF900895CF92DF92EF92FF920F9361
:106E20001F93CF93DF93CDB7DEB72F970FB6F894AC
:106E3000DEBF0FBECDBF6C018E010F5F1F4FC801BB
:106E40000E94A1DDC80140E553EC60E070E00E94C3
:106E5000A5DDE02E012F11C08E2D902F0E94CBDDDD
:106E6000882359F0C60167E80E94D3DB8DE698E1DC
:106E700062E070E00E9448913EC00E94D879882369
:106E800059F30E94D5798C010E94D2797C01C80106
:106E90000E948DDB0E94847C682FC8010E94D3DB96
:106EA000C80167E10E94D3DB0E94EB790E94E87978
:106EB00002C00E94477A0E94427A8823D1F3F701E8
:106EC00082A1843081F4C60167E80E94D3DB13C03D
:106ED000C701602F0E946DDB682FC6010E94D3DBC3
:106EE0000F5F1F4F02C000E010E0F701808190E0CB
:106EF000081719076CF32F960FB6F894DEBF0FBE74
:106F0000CDBFDF91CF911F910F91FF90EF90DF9058
:106F1000CF9008958F929F92AF92BF92CF92DF92BF
:106F2000EF92FF920F931F93CF93DF93CDB7DEB70E
:106F30002F970FB6F894DEBF0FBECDBF7C016B015B
:106F4000FC018081823048F4CB0160E80E94D3DBF1
:106F50008DE698E168E070E01EC08E010F5F1F4F64
:106F6000C8010E94A1DDC80140E553EC60E070E07B
:106F70000E94A5DDA02E012F11C08A2D902F0E9406
:106F8000CBDD882359F0C60167E80E94D3DB8DE68C
:106F900098E162E070E00E94489147C00E94D87971
:106FA000882359F30E94D5794C010E94D2795C0163
:106FB000C4010E948DDB01E010E00AC0C701602F10
:106FC0000E946DDB682FC4010E94D3DB0F5F1F4F4F
:106FD000F701808190E00817190784F30E94EB798C
:106FE0000E94E87902C00E94477A0E94427A882370
:106FF000D1F3F50182A1843081F4C60167E80E94D3
:10700000D3DB13C0C501602F0E946DDB682FC60162
:107010000E94D3DB0F5F1F4F02C000E010E0F501BC
:10702000808190E0081719076CF32F960FB6F8943B
:10703000DEBF0FBECDBFDF91CF911F910F91FF90AB
:10704000EF90DF90CF90BF90AF909F908F9008957A
:107050006F927F928F929F92AF92BF92CF92DF9268
:10706000EF92FF920F931F93CF93DF93CDB7DEB7CD
:10707000A82EE92E6B016DB67EB661E00E9472DB30
:107080008C018A2D9E2D63E00E946DDB482F882E97
:1070900099248DB79EB7881999090FB6F8949EBFA9
:1070A0000FBE8DBFADB6BEB60894A11CB11CC50104
:1070B000B80150E00E94C9E5C60161E80E94D3DB37
:1070C000750100E010E008C0F70161917F01C60181
:1070D0000E94D3DB0F5F1F4F08151905ACF30FB6E5
:1070E000F8947EBE0FBE6DBEDF91CF911F910F91C0
:1070F000FF90EF90DF90CF90BF90AF909F908F90D8
:107100007F906F9008952F923F925F926F927F923F
:107110008F929F92AF92BF92CF92DF92EF92FF92A7
:107120000F931F93CF93DF930F920F92CDB7DEB7DC
:10713000E82ED92E3B018DB79EB79A8389838E2D79
:107140009D2D61E00E9472DBC82EB92E8E2D9D2DE3
:1071500063E00E946DDBF82E282E3324EDB7FEB7D6
:10716000E219F3090FB6F894FEBF0FBEEDBF0DB7DD
:107170001EB70F5F1F4FA02E512EC8016C2D7B2D07
:107180004F2D50E00E94C9E5480100E010E00BC01F
:10719000602F6C5F8E2D9D2D0E946DDBF40181931D
:1071A0004F010F5F1F4F0215130594F30FB7F894AB
:1071B0008A2D952D6C2D7B2D4F2D50E00E94E1E501
:1071C0000FBFC30161E80E94D3DBC3016F2D0E9492
:1071D000D3DB89819A810FB6F8949EBF0FBE8DBF15
:1071E0000F900F90DF91CF911F910F91FF90EF9033
:1071F000DF90CF90BF90AF909F908F907F906F90D7
:107200005F903F902F9008950F931F93CF93DF933C
:107210008091640B882389F404E61BE0C0E2D0E08F
:10722000CE0160E00E94DA99F80181938F012196E6
:10723000C033D105A9F71092740B8091640B882399
:1072400079F4A4E6BBE080E090E0FC01E859FE4F51
:10725000E491ED9301968D309105B9F71092710B81
:1072600084E69BE0DF91CF911F910F91089585E413
:107270009BE008958091430B9091440B0895809179
:10728000410B9091420B0895CF93DF930097A9F0A3
:107290002BE08534920799F0EC01A5E4BBE0E0E037
:1072A00004C02D93EF5FEE3119F029912223C9F725
:1072B000F0E0EB5BF44F108202C085E49BE00E949B
:1072C0005F41EC018930910579F0009779F40E94D3
:1072D00085160E9412760E94017682E090E09093DB
:1072E000440B8093430B02C0C0E0D0E0CE01DF919D
:1072F000CF910895CF93C82F0E944515C817F9F074
:107300000E9458158823D9F48C2F60E00E9437150D
:10731000CC2351F083E090E09093420B8093410B9B
:107320008BE29BE061E009C081E090E09093420B2A
:107330008093410B8BE29BE060E00E94F8DDCF91EF
:1073400008958BE29BE040E054EA63E976ED0E9409
:10735000A5DD10923A0B0895FF920F931F93CF93E0
:10736000DF93FC018091430B9091440B8130910598
:1073700079F18230910519F0009721F155C0828191
:107380009381009719F481E081874EC084819581B3
:1073900020813181B9010E94D5E4C681D781C80F0F
:1073A000D91F848195810196B9010E94D5E4958306
:1073B0008483828193810197938382838881882348
:1073C000F1F632C081E090E09093440B8093430B40
:1073D00005E41BE04FE1FF24F39482819381009741
:1073E00019F4F18680E019C0848195812081318172
:1073F000B9010E94D5E4C681D781C80FD91F848105
:1074000095810196B9010E94D5E495838483828198
:1074100093810197938382838881D8018D938D0115
:10742000882311F04150C9F68DE698E10E949F90A3
:107430000E94A1390E94361781E090E09093420BA0
:107440008093410BDF91CF911F910F91FF90089591
:107450008BE29BE00E94CBDD882369F08BE29BE00E
:1074600040E054EA63E976ED0E94A5DD80913A0B95
:107470008F5F80933A0B0895CF93DF93EB012091B8
:107480003A0BFC0120838BE29BE00E9427DE20E088
:1074900037E843E953E00E94FCE42883DF91CF9171
:1074A0000895CF93DF93CDB7DEB72F970FB6F8943B
:1074B000DEBF0FBECDBF80E49BE06FE37BE00E94A8
:1074C0003C3ACE0101960E94A1DDABE2BBE0FE0199
:1074D00031968FE001900D928150E1F710923A0BB6
:1074E0002F960FB6F894DEBF0FBECDBFDF91CF91C0
:1074F00008958091430B9091440B8130910589F45C
:1075000084E090E09093440B8093430B84E89BE0ED
:1075100040E452E46FE070E00E94A5DD81E08093DA
:10752000280B0E942D17DC01CB0180933B0B90931D
:107530003C0BA0933D0BB0933E0B0E94513A81E06F
:1075400080932A0B85E79BE040E45DE063E070E018
:107550000E94A5DD84E090E09093420B8093410B64
:10756000089585E090E09093420B8093410B0E9438
:1075700001760E944515882321F40E94581588231E
:1075800019F00E94793A089581E060E00E94371571
:1075900008950E94513A0E942D17DC01CB0180937F
:1075A0003B0B90933C0BA0933D0BB0933E0B82E0C2
:1075B00090E09093420B8093410B1092440B1092F9
:1075C000430B08950F931F93CF93DF930F920F9266
:1075D000CDB7DEB78C0161E80E94D3DBCE01029605
:1075E000BE016F5F7F4F0E943C3AC8016091410B22
:1075F0000E94D3DBC8016A810E94D3DBC801698184
:107600000E94D3DB8091410B9091420B8130910518
:1076100019F08330910529F40E942D17AB01BC01AC
:1076200008C040913B0B50913C0B60913D0B709119
:107630003E0BC8010E94ECDBC80140E050E060E076
:1076400070E00E94ECDB0F900F90DF91CF911F91C3
:107650000F910895AF92BF92CF92DF92EF92FF9277
:107660000F931F93CF93DF930F92CDB7DEB75C01DB
:107670008B01FC018081882309F41DC1FA2CEB2CBD
:10768000C50160E00E946DDB87FD15C1E82FF0E0C9
:10769000EC31F10508F00FC1EE58FF4FEE0FFF1F60
:1076A0000590F491E02D19948A2D9B2D61E00E94A4
:1076B00072DB8732910518F4C80161E8F4C0C80193
:1076C00061E80E94D3DBC80162E971E0F1C0C80142
:1076D00061E80E94D3DB45E4E42E4BE0F42E5FE149
:1076E000C52E5701C801F70161917F010E94D3DBCC
:1076F000F5018081882309F4E0C0CA9491F7DDC0C8
:107700000E94B91B8091430B9091440B01978230EA
:10771000910530F48DE698E16BE070E00E944891AD
:1077200081E080932A0B85E79BE040E45DE063E025
:1077300070E00E94A5DDC80161E8D4C0C80161E81D
:107740000E94D3DB0E942715AC0160E070E0C80105
:107750000E94ECDBB2C0C501B8010E94E635ADC0A5
:10776000C501B8010E943A36A8C0C80161E80E946C
:10777000D3DBC50103960E94CA41B2C0C80161E8CB
:107780000E94D3DB0E94E63FAB01BC01C8010E940E
:10779000ECDB0E94CC4091C0C80161E80E94D3DBC1
:1077A00035E4C32E3BE0D32E21E0F501808128177C
:1077B00008F090C02F3109F48DC08F2D9E2D622FBF
:1077C00029830E946DDBF60181936F0129812F5F70
:1077D000ECCFC501B8010E94AB366FC00E945815AE
:1077E000882309F0A8CF0E94451591E089270E94BF
:1077F0007A39C8010E940B379ECFC501B8010E949B
:107800008A375BC0C80161E80E94D3DBF8940E940C
:10781000D86D882321F40E944D16882311F460E06E
:1078200001C061E0C8010E94D3DB789446C0C50165
:10783000B8010E94283841C0C501B8010E948338B0
:107840003CC08A2D9B2D61E00E946DDBE82E80FFFD
:1078500002C00E940176E1FE02C00E948516C801A6
:1078600061E80E94D3DBC80160E03CC0C8010E940F
:10787000E23A23C08A2D9B2D61E00E9472DBC80191
:1078800061E80E94D3DBC80162E971E00E94D6DBA7
:10789000C80160E070E00E94D6DBC80160E80E9489
:1078A000D3DBC80160E00E94D3DBC80160E070E078
:1078B0000E94D6DB02C080E001C081E00F90DF9122
:1078C000CF911F910F91FF90EF90DF90CF90BF90DD
:1078D000AF9008951092630B80E090E00E944439CD
:1078E000682FC8010E94D3DBE8CF8091410B9091B3
:1078F000420B8530910539F40E9453158130910572
:1079000011F40E94793A8091291C90912A1C0097C9
:1079100009F4BAC08091291C90912A1C84309105E9
:1079200009F4B2C080912A0B882309F4BAC085E714
:107930009BE00E94CBDD882309F4B3C0A5C08091F1
:10794000280B882339F084E89BE00E94CBDD882354
:1079500009F49FC08091410B9091420B81309105B9
:1079600019F08330910511F40E94B13A10922A0B5C
:107970008091290B0E94883D1092290B83E99BE09E
:107980000E94F5DD1092640B1092450B1092440B8F
:107990001092430B08958091031C9091041C843035
:1079A0009105D1F08091930B882349F483E99BE002
:1079B00040E45DE063E070E00E94A5DD0DC083E976
:1079C0009BE00E94CBDD882339F080EE9BE10E9492
:1079D0000ADB84E08093021C8091021C882321F042
:1079E00080EE9BE10E9418DB8091031C9091041CA7
:1079F00084309105B9F583E99BE00E94F5DD86E0CE
:107A00009CE10E948DDB8091280B882371F086E039
:107A10009CE169E80E94D3DB1092280B8DE698E187
:107A20006AE070E00E94489115C080EE9BE166E03C
:107A30007CE10E949335882369F480EE9BE166E047
:107A40007CE10E942A3B882329F486E09CE165E8DA
:107A50000E94D3DB80EE9BE10E9418DB8CED9BE162
:107A60000E94A2DE8091430B9091440B82309105DD
:107A700041F40E94A33F882321F41092440B1092FA
:107A8000430B0E94283A089580912A0B882309F01D
:107A900056CF8091031C9091041C009709F07BCF76
:107AA0009BCF08951092640B1092450B1092440BDB
:107AB0001092430B08950E944D16882329F00E94CE
:107AC0001C4091E0982701C090E0892F089583E938
:107AD0009BE00E94A1DD84E89BE00E94A1DD85E798
:107AE0009BE00E94A1DD8BE29BE00E94A1DD089556
:107AF00080E090E0EEE2FCE12081253C41F421E2CF
:107B0000EF3FF20709F018F431960196F5CF08958A
:107B1000FF920F931F93CF93DF93CDB7DEB7659797
:107B20000FB6F894DEBF0FBECDBF082FF8940E94A9
:107B3000CC400E943E6F0E9401760E9485160E94F2
:107B40003D990E94127678948DE698E1602F0E940C
:107B50007D9184E790E060E00E94DA99813011F431
:107B600083E002C0823019F480936A00EC9A20917D
:107B7000591B30915A1B3D832C838E81807F8260FC
:107B80008E83CE01049662E040E00E94C39520916E
:107B9000591B30915A1B3A8329838B81807F8260E5
:107BA0008B83CE01019662E00E94D8958093A20B50
:107BB0000023B9F08E01095F1F4FC8010E94A1DDAB
:107BC000C80140EA55E266E270E00E94A5DDF02EB1
:107BD000012F8F2D902F0E94CBDD8823D1F30E949F
:107BE000387C0E94F77A789465960FB6F894DEBFD9
:107BF0000FBECDBFDF91CF911F910F91FF900895E0
:107C0000CF93DF9300D0CDB7DEB781E00E94883DEF
:107C100078940E94477A0E94753C0E94E2238DE688
:107C200098E10E943D940E9454798091591B909153
:107C30005A1B9A8389838B81807F82608B83CE01DC
:107C4000019662E00E94D895182F8091A20B88239C
:107C500039F4112329F00E94523D81E00E94883DB1
:107C60001093A20BD6CF78941F920F920FB60F925B
:107C70000BB60F9211242F933F934F935F936F9303
:107C80007F938F939F93AF93BF93CF93DF93EF93A4
:107C9000FF930E94F77A0E9401760E9485168CED70
:107CA0009BE160E00E94DEDECDE6D8E1CE0167E038
:107CB00070E00E9448918AE890E063E00E94DA99BF
:107CC000282FCE0167E04AE00E946292FF91EF9177
:107CD000DF91CF91BF91AF919F918F917F916F91E4
:107CE0005F914F913F912F910F900BBE0F900FBE60
:107CF0000F901F90189508958F929F92AF92BF9208
:107D0000CF92DF92EF92FF920F931F93CF93DF9367
:107D1000CDB7DEB7FC014083518362837383048354
:107D2000158326833783C086D186E286F3868486D0
:107D30009586A686B78688899989AA89BB89808B0A
:107D4000918BA28BB38BDF91CF911F910F91FF90FD
:107D5000EF90DF90CF90BF90AF909F908F9008955D
:107D6000660F771F660F771F680F791FCB01089585
:107D7000660F771F660F771F680F791FCB01089575
:107D80008091B30B9091B40B009741F00E94D58382
:107D90000E947F8B1092B40B1092B30B08950F9337
:107DA0001F93CF93DF93CDB7DEB7AB970FB6F894A1
:107DB000DEBF0FBECDBFBC018091A70B9091A80B79
:107DC00061157105C9F460E072E0AE014F5F5F4F6D
:107DD0000E94AE888091A70B9091A80BBE016F5FA7
:107DE0007F4F0E949C879093A40B8093A30B0097D6
:107DF00091F485E090E014C00E949C878C0100976C
:107E000069F08091A30B9091A40B0E94D9871093E5
:107E1000A40B0093A30B80E090E002C087E090E009
:107E2000AB960FB6F894DEBF0FBECDBFDF91CF91FA
:107E30001F910F9108950F931F93CF93DF938C01A0
:107E4000EB018091A30B9091A40B0E94398906C08D
:107E5000CE01B8010E9498E5009751F08091A30BE4
:107E60009091A40BBE010E94DF87882389F701C08F
:107E700081E0DF91CF911F910F910895CF93DF9310
:107E8000CDB7DEB7AB970FB6F894DEBF0FBECDBF50
:107E9000BE016F5F7F4F0E941B3F8823F9F089A1CD
:107EA00084FF08C0CE0101960E94CF3E0097B1F436
:107EB0008FEF15C00E94C03E8091A70B9091A80B38
:107EC000BE016F5F7F4F0E949E839C019093B40B15
:107ED0008093B30B81E02115310509F480E0AB9666
:107EE0000FB6F894DEBF0FBECDBFDF91CF910895DE
:107EF000CF93DF93CDB7DEB7AB970FB6F894DEBF65
:107F00000FBECDBF20915003222351F4BE016F5FFD
:107F10007F4F0E941B3F882319F089A184FD0BC06D
:107F200020E0822FAB960FB6F894DEBF0FBECDBF18
:107F3000DF91CF910895CE0101960E94CF3E21E0BE
:107F4000009779F3EDCF8091A90B08958091AA0B4A
:107F50000895CF93DF93EC018091B30B9091B40B14
:107F60000097E1F0BE016E5F7F4F488150E00E94B4
:107F7000F98428818091AB0B9091AC0BA091AD0B53
:107F8000B091AE0B820F911DA11DB11D8093AB0B63
:107F90009093AC0BA093AD0BB093AE0BDF91CF9150
:107FA0000895CF93DF930F92CDB7DEB78983809189
:107FB000B30B9091B40BBE016F5F7F4F41E050E077
:107FC0000E94F9840F90DF91CF9108958091AA0BC0
:107FD000882321F00E94C03E1092AA0B6091AB0B47
:107FE0007091AC0B8091AD0B9091AE0B0895809188
:107FF000B30B9091B40B65EB7BE041E050E00E9445
:10800000E88321E0181619060CF020E02093B60B47
:108010008091AF0B9091B00BA091B10BB091B20BCE
:108020000196A11DB11D8093AF0B9093B00BA0934F
:10803000B10BB093B20B08958091B60B0895CF9316
:10804000DF930F92CDB7DEB78091B50B89830E9485
:10805000F73F89810F90DF91CF910895CF93DF9300
:1080600000D00F92CDB7DEB719821A821B821C8214
:108070008091B30B9091B40BBE016F5F7F4F40E0D6
:108080000E9441871092AB0B1092AC0B1092AD0B7B
:108090001092AE0B1092AF0B1092B00B1092B10B6E
:1080A0001092B20B81E08093A90B0E94F73F0F90D2
:1080B0000F900F900F90DF91CF910895CF92DF92A4
:1080C000EF92FF921F93CF93DF936091AF0B70916C
:1080D000B00B8091B10B9091B20B24E630E040E000
:1080E00050E00E94AAE40E94BCE26B017C01609116
:1080F000B70B7091B80B8091B90B9091BA0B0E949D
:10810000BCE29B01AC01C701B6010E94E3E1162F5E
:10811000C72ED82FC92F9E01862F9C2DA32FB22F9B
:10812000BC01CD0120E030E048EC52E40E94FAE3CB
:108130001816A4F09E01812F9C2DA32FB22FBC01F5
:10814000CD0120E030E040E050E00E94DFE187FF19
:1081500009C010E0CC24D0E0C0E004C010E0CC2482
:10816000D8ECC2E49E01812F9C2DA32FBC2FBC0113
:10817000CD01DF91CF911F91FF90EF90DF90CF90D5
:1081800008958091A90B882331F00E94C03E10927F
:10819000A90B1092B60B08950E94C1400E94E63FC1
:1081A0000E94C03E8091A30B9091A40B009731F0E8
:1081B0000E94D9871092A40B1092A30B8091A70B59
:1081C0009091A80B009731F00E9498831092A80B11
:1081D0001092A70B8091A50B9091A60B009731F000
:1081E0000E94F28A1092A60B1092A50B81E0809358
:1081F000500381E090E090934F0380934E030895E5
:108200000F93CF93DF930E94CC400E948D8C8823E4
:10821000C9F18BE99BE869E37CE848E45DE82EEF6F
:108220003DE800E00E94218A9093A60B8093A50B65
:10823000009779F48BE99BE869E37CE848E45DE822
:108240002EEF3DE80FEF0E94218A9093A60B8093BA
:10825000A50B8091A50B9091A60B0097D1F00E94E1
:10826000F3819093A80B8093A70B0097A9F080E06F
:1082700090E00E94CF3E009791F410925003C0E02E
:10828000D0E018C00E944A8B882361F0C1E0D0E0A2
:108290000BC0C3E0D0E008C0C4E0D0E005C0C5E03A
:1082A000D0E002C0C2E0D0E00E94CC40D0934F03A7
:1082B000C0934E03CE01DF91CF910F9108950F939C
:1082C0001F93CF93DF9300D00F92CDB7DEB78C0111
:1082D00080915003882329F00E940041009709F003
:1082E00050C01092AB0B1092AC0B1092AD0B1092D1
:1082F000AE0B1092AF0B1092B00B1092B10B10920C
:10830000B20BC8010E943E3F8823B1F18F3FB9F103
:1083100081E08093A90B19821A821B821C828091B2
:10832000B30B9091B40BBE016F5F7F4F42E00E9490
:10833000418789819A81AB81BC818093B70B9093EF
:10834000B80BA093B90BB093BA0B19821A821B8297
:108350001C828091B30B9091B40BBE016F5F7F4F75
:1083600040E00E9441878DE698E10E949F900E9424
:10837000F73F80E090E005C087E090E002C089E030
:1083800090E00F900F900F900F90DF91CF911F9181
:108390000F9108950F931F93CF93DF93CDB7DEB75F
:1083A000AB970FB6F894DEBF0FBECDBF8C018091A6
:1083B0005003882329F00E940041009709F043C030
:1083C0000E94668B8823B9F51092AB0B1092AC0B10
:1083D0001092AD0B1092AE0B1092AF0B1092B00B2F
:1083E0001092B10B1092B20BC801BE016F5F7F4FAC
:1083F0000E941B3F882349F08091A70B9091A80B06
:10840000BE016F5F7F4F0E94A3898091A30B909163
:10841000A40BB801AE014F5F5F4F0E9446898823CD
:1084200069F0C8010E943E3F813059F48093AA0B45
:1084300080E090E008C086E090E005C087E090E032
:1084400002C088E090E0AB960FB6F894DEBF0FBE96
:10845000CDBFDF91CF911F910F910895BF92CF9221
:10846000DF92EF92FF920F931F93CF93DF93CDB7DD
:10847000DEB7AB970FB6F894DEBF0FBECDBF7C0161
:10848000D62E8A01FC0110824115510529F0FA010E
:1084900010822EE0B22E02C09EE1B92E80915003D0
:1084A000882389F10E940041009789F52CC08091B2
:1084B000A30B9091A40BBE016F5F7F4F0E94DF87DB
:1084C000882329F189A19B2D9823D1F4998199239F
:1084D000B1F084FF03C081E0F8018083D701FE0181
:1084E000319680E08D1530F49191992319F09D9388
:1084F0008F5FF8CFF701E80FF11D108208C0CA9412
:10850000CC20A9F604C0DA9485E0C82ED0CFAB9673
:108510000FB6F894DEBF0FBECDBFDF91CF911F9194
:108520000F91FF90EF90DF90CF90BF9008958091D2
:108530005003882321F00E940041009741F480916C
:10854000A30B9091A40B0E94398980E090E00895DC
:108550000F931F93CF93DF93CDB7DEB7AB970FB6D3
:10856000F894DEBF0FBECDBF8C010E9497420097EA
:1085700039F4C801BE016F5F7F4F0E941B3F01C0ED
:1085800080E0AB960FB6F894DEBF0FBECDBFDF9193
:10859000CF911F910F9108954F925F926F927F92AA
:1085A0008F929F92AF92BF92CF92DF92EF92FF9203
:1085B0000F931F93CF93DF938091CD0B9091CE0BB0
:1085C000009709F033C49091F10B8091F00B98174C
:1085D000A1F02091F00B30E087E790E0289FF001B8
:1085E000299FF00D389FF00D1124EE50F44FDF015C
:1085F000AC58BF4F81E08C9302C0E0E0F0E0F09314
:10860000CE0BE093CD0B309709F4B3C3808D918DE1
:10861000A28DB38D8093511490935214A093531450
:10862000B0935414848D958DA68DB78D8093551479
:1086300090935614A0935714B093581480A191A10D
:10864000A2A1B3A18093591490935A14A0935B14E0
:10865000B0935C1484A195A1A6A1B7A180935D14E9
:1086600090935E14A0935F14B093601480A591A5BD
:10867000A2A5B3A58093611490936214A093631490
:10868000B093641482AD8093CF0B8091D00B88237C
:10869000E1F18F01C1EDDBE069EC7BE040E050E00F
:1086A000F80184859585A685B7850097A105B10554
:1086B00011F188818823F9F0FA01E953F44F8081A0
:1086C000FA01EE0FFF1FE85BFB4E882349F0808123
:1086D0009181DB012D913C911197821B930B08C076
:1086E00080819181DB012D913C911197820F931F25
:1086F0009183808318824F5F5F4F0C5F1F4F2196DD
:108700006E5F7F4F4230510559F61092D30B109295
:10871000D40B1092D50B1092D60BC091CD0BD091EB
:10872000CE0BFE01E25AFF4F208131813F3460F0D1
:108730003D3930F443E0369527954A95E1F702C07C
:1087400028E833E188E014C0383230F036952795B8
:108750003695279584E00CC0343120F03695279566
:1087600082E006C02032310510F420E230E081E0E2
:108770008093D70B20523040B8E020303B07C8F040
:10878000E32FF0E0EE0FFF1FEE0FFF1FEA58FE4F42
:1087900085919591A591B491AC01BD01AA27279F20
:1087A000C001269F810D9A1F06948A1F9A1F1124CB
:1087B0001AC0F901F695E795EC7FEA58FA4F8591D2
:1087C0009591A591B491AC0130E0277030702A9F4B
:1087D000C0012B9F900D3A9F900D112413E09695A8
:1087E00087951A95E1F7481B590B5093D90B409385
:1087F000D80B8091D70B8093DA0BFE01EE58FF4F18
:108800008081882309F472C0CA59DF4F28813981D9
:108810003093DC0B2093DB0B3F3460F03D3930F4B8
:10882000A3E036952795AA95E1F702C028E833E141
:1088300088E014C0383230F0369527953695279564
:1088400084E00CC0343120F03695279582E006C0D4
:108850002032310510F420E230E081E08093D70B24
:1088600020523040E8E020303E07C8F0E32FF0E02F
:10887000EE0FFF1FEE0FFF1FEA58FE4F85919591F7
:10888000A591B491AC01BD01AA27279FC001269FE5
:10889000810D9A1F06948A1F9A1F11241AC0F9018C
:1088A000F695E795EC7FEA58FA4F85919591A59159
:1088B000B491AC0130E0277030702A9FC0012B9F2B
:1088C000900D3A9F900D112463E0969587956A95D7
:1088D000E1F7481B590BCA01A0E0B0E08093DD0B23
:1088E0009093DE0BA093DF0BB093E00B50939900B5
:1088F00040939800E091CD0BF091CE0B80AD80932A
:10890000E10BEA58FF4F208180914814909149145F
:10891000009719F480915E158111286080914A14A6
:1089200090914B14009719F480915F15811120618B
:1089300080914614281709F442C0E1E6F3E0EF0104
:10894000249640E050E061E070E0CB01042E02C0CC
:10895000880F991F0A94E2F7A82F30914614322706
:10896000382331F1A22390914614AA2389F0982B41
:1089700090934614A081B1813C91CB01088002C044
:10898000880F991F0A94E2F7809583238C9310C077
:108990008095892380934614A081B1813C91CB01BD
:1089A000088002C0880F991F0A94E2F7382B3C9385
:1089B0004F5F5F4FB396A3964530510531F6E09176
:1089C000CD0BF091CE0BDF01AB58BF4FDC9174891A
:1089D000658956894789C091E10B00811181228107
:1089E000338181E0011511052105310509F480E08D
:1089F00080938114882309F444C0872F962FA52FD4
:108A0000B42FEE24E394EC22AC01BD01759567957B
:108A10005795479570956095509541955F4F6F4F6D
:108A20007F4F409382145093831460938414709307
:108A3000851441E0D11140E04093791480937A1479
:108A400090937B14A0937C14B0937D1400938A14AC
:108A500010938B1420938C1430938D14EE2011F00E
:108A60008FEF01C081E080937F1481E08E25809399
:108A70008014109286141092871410928814109209
:108A800089147489658956894789048115812681ED
:108A9000378181E0011511052105310509F480E0D8
:108AA0008093AA14882309F446C0872F962FA52FF8
:108AB000B42FEE24E394C1FFEE24AC01BD01759503
:108AC00067955795479570956095509541955F4F7F
:108AD0006F4F7F4F4093AB145093AC146093AD1421
:108AE0007093AE1441E0D13009F040E04093A214FD
:108AF0008093A3149093A414A093A514B093A614E8
:108B00000093B3141093B4142093B5143093B61497
:108B1000EE2011F08FEF01C081E08093A81481E076
:108B20008E258093A9141092AF141092B014109255
:108B3000B1141092B21474896589568947890085E9
:108B400011852285338581E0011511052105310547
:108B500009F480E08093D314882309F446C0872F5A
:108B6000962FA52FB42FEE24E394C2FFEE24AC0180
:108B7000BD0175956795579547957095609550958A
:108B800041955F4F6F4F7F4F4093D4145093D5144E
:108B90006093D6147093D71441E0D23009F040E0CE
:108BA0004093CB148093CC149093CD14A093CE1407
:108BB000B093CF140093DC141093DD142093DE14D3
:108BC0003093DF14EE2011F08FEF01C081E080932D
:108BD000D11481E08E258093D2141092D814109273
:108BE000D9141092DA141092DB14748965895689AD
:108BF0004789048515852685378581E0011511058E
:108C00002105310509F480E08093FC14882309F4E0
:108C100046C0872F962FA52FB42FEE24E394C3FFD1
:108C2000EE24AC01BD0175956795579547957095F4
:108C30006095509541955F4F6F4F7F4F4093FD1466
:108C40005093FE146093FF147093001541E0D330ED
:108C500009F040E04093F4148093F5149093F614D7
:108C6000A093F714B093F81400930515109306150C
:108C70002093071530930815EE2011F08FEF01C0F7
:108C800081E08093FA1481E08E258093FB1410928A
:108C90000115109202151092031510920415DF01B0
:108CA000AB58BF4FDC91E488058936892789408914
:108CB00051896289738981E041155105610571050A
:108CC00009F480E080932515882309F445C08E2D92
:108CD000902FA32FB22FE1E0C4FFE0E08C019D01B3
:108CE0003595279517950795309520951095019501
:108CF0001F4F2F4F3F4F009326151093271520939A
:108D000028153093291521E0D43009F020E0209374
:108D10001D1580931E1590931F15A0932015B093D9
:108D2000211540932E1550932F1560933015709395
:108D30003115EE2311F08FEF01C081E080932315F0
:108D400081E08E278093241510922A1510922B15FE
:108D500010922C1510922D151092E30B1092E20B2D
:108D60001092BB0B1092BC0B1092BD0B1092BE0B5D
:108D70005DC080ED97E0909399008093980080917A
:108D8000481490914914009709F050C080914A14FA
:108D900090914B14009709F049C02091471480919D
:108DA0004614281709F442C0E1E6F3E0EF012496E7
:108DB00040E050E061E070E0CB01042E02C0880F7B
:108DC000991F0A94E2F7A82F3091461432273823CE
:108DD00031F1A22390914614AA2389F0982B909305
:108DE0004614A081B1813C91CB01088002C0880F5C
:108DF000991F0A94E2F7809583238C9310C0809585
:108E0000892380934614A081B1813C91CB010880D5
:108E100002C0880F991F0A94E2F7382B3C934F5FEA
:108E20005F4FB396A3964530510531F68091D00B34
:108E3000882309F443C06091CD0B7091CE0BA1ED56
:108E4000BBE0C9ECDBE040E050E001E086E7C82E83
:108E5000D12CC60ED71E6115710561F0F601208177
:108E600030E0CA01039602C0359527958A95E2F74E
:108E700020FD1DC08C918823D1F4FA01E953F44FF1
:108E80002081CA01880F991FFC01E85BFB4E80819D
:108E90009181222329F028813981820F931F04C0F8
:108EA00028813981821B930B918380830C934F5FC0
:108EB0005F4F119622964230510569F68091CD0B95
:108EC0009091CE0B009711F40C94BA53D090D70B1D
:108ED000E090E20BF090E30B4090E40B5090E50B38
:108EE0006090E60B7090E70B7094609450944094FF
:108EF000411C511C611C711C452C562C672C77247D
:108F000067FC7A948824C1E0D0E0CC24C39426C6C0
:108F1000E091CD0BF091CE0BDF01AE58BF4F8C919D
:108F2000882309F476C0E114F104F1F002E0E016C0
:108F3000F104A1F586AD97AD909581959F4FAA2735
:108F400097FDA095BA2F4091FD145091FE146091A9
:108F5000FF1470910015840F951FA61FB71F840D75
:108F6000951DA61DB71D12C044AD55AD662757FD12
:108F70006095762F8091FD149091FE14A091FF14BE
:108F8000B0910015840F951FA61FB71F8093FD1485
:108F90009093FE14A093FF14B0930015E114F10414
:108FA00099F444AD55AD662757FD6095762F8091B5
:108FB000261590912715A0912815B0912915840F99
:108FC000951FA61FB71F1DC012E0E116F10409F599
:108FD00086AD97AD909581959F4FAA2797FDA09557
:108FE000BA2F409126155091271560912815709140
:108FF0002915840F951FA61FB71F840D951DA61D4B
:10900000B71D8093261590932715A0932815B0932C
:10901000291580918114882309F414C180918A1440
:1090200090918B14A0918C14B0918D1400918214A6
:10903000109183142091841430918514080F191F06
:109040002A1F3B1F009382141093831420938414CF
:109050003093851410161106120613060CF0F2C098
:1090600040918614509187146091881470918914EE
:10907000481759076A077B070CF0E4C080917A14FF
:1090800090917B14A0917C14B0917D14081B190B56
:109090002A0B3B0B009382141093831420938414A7
:1090A0003093851480917E14882351F1809142146D
:1090B0009091431440917F14242F332727FD30953E
:1090C000820F931F90934314809342148091511404
:1090D00090915214A0915314B0915414552747FD08
:1090E0005095652F752F840F951FA61FB71F80936E
:1090F000511490935214A0935314B09354148FC0EE
:10910000909180148091661481119C25E0915A03FE
:10911000F0915B0380915E032081992349F0AE01B9
:1091200002C0440F551F8A95E2F7242B20830AC002
:10913000BE0102C0660F771F8A95E2F7CB018095CA
:1091400082238083809180148823A1F080916F0313
:1091500090917003009749F1E0917103F0917203CF
:10916000808190E00090730302C0959587950A94E2
:10917000E2F713C080916803909169030097A9F00A
:10918000E0916A03F0916B03808190E000906C03A2
:1091900002C0959587950A94E2F78170907090913E
:1091A0006514981711F00C94CE53E0915303F0918D
:1091B00054032081CE010090570302C0880F991FED
:1091C0000A94E2F7282B2083809151149091521435
:1091D000A0915314B091541440917F14552747FD2A
:1091E0005095652F752F840F951FA61FB71F80936D
:1091F000511490935214A0935314B0935414E091CB
:109200005303F09154032081CE010090570302C014
:10921000880F991F0A94E2F78095822380838091BA
:10922000861490918714A0918814B09189140196A6
:10923000A11DB11D8093861490938714A093881468
:10924000B09389148091AA14882309F414C18091E1
:10925000B3149091B414A091B514B091B6140091C8
:10926000AB141091AC142091AD143091AE14080FD2
:10927000191F2A1F3B1F0093AB141093AC142093AB
:10928000AD143093AE1410161106120613060CF02E
:10929000F2C04091AF145091B0146091B11470912C
:1092A000B214481759076A077B070CF0E4C0809195
:1092B000A3149091A414A091A514B091A614081B16
:1092C000190B2A0B3B0B0093AB141093AC14209397
:1092D000AD143093AE148091A714882351F180917E
:1092E0004414909145144091A814242F332727FD4E
:1092F0003095820F931F909345148093441480916E
:10930000551490915614A0915714B09158145527A4
:1093100047FD5095652F752F840F951FA61FB71F0A
:109320008093551490935614A0935714B0935814E7
:109330008FC09091A91480918F1481119C25E09188
:109340007D03F0917E03809181032081992349F070
:10935000DE0102C0AA0FBB1F8A95E2F72A2B2083E9
:109360000AC08E0102C0000F111F8A95E2F7C801E2
:109370008095822380838091A9148823A1F0809115
:10938000920390919303009749F1E0919403F09137
:109390009503808190E00090960302C09595879593
:1093A0000A94E2F713C080918B0390918C0300978D
:1093B000A9F0E0918D03F0918E03808190E0009000
:1093C0008F0302C0959587950A94E2F7817090709B
:1093D00090918E14981711F00C94D253E09176036B
:1093E000F09177032081CE0100907A0302C0880FAC
:1093F000991F0A94E2F7282B2083809155149091AD
:109400005614A0915714B09158144091A8145527A0
:1094100047FD5095652F752F840F951FA61FB71F09
:109420008093551490935614A0935714B0935814E6
:10943000E0917603F09177032081CE0100907A03CA
:1094400002C0880F991F0A94E2F7809582238083D7
:109450008091AF149091B014A091B114B091B21456
:109460000196A11DB11D8093AF149093B014A093E9
:10947000B114B093B2148091D314882309F414C1A9
:109480008091DC149091DD14A091DE14B091DF1472
:109490000091D4141091D5142091D6143091D71482
:1094A000080F191F2A1F3B1F0093D4141093D514C3
:1094B0002093D6143093D7141016110612061306F3
:1094C0000CF0F2C04091D8145091D9146091DA1484
:1094D0007091DB14481759076A077B070CF0E4C04A
:1094E0008091CC149091CD14A091CE14B091CF1452
:1094F000081B190B2A0B3B0B0093D4141093D514A3
:109500002093D6143093D7148091D014882351F12E
:1095100080914614909147144091D114242F332701
:1095200027FD3095820F931F909347148093461424
:109530008091591490915A14A0915B14B0915C14CD
:10954000552747FD5095652F752F840F951FA61F32
:10955000B71F8093591490935A14A0935B14B0933F
:109560005C148FC09091D2148091B81481119C2505
:10957000E091A003F091A1038091A403208199239D
:1095800049F0AE0102C0440F551F8A95E2F7242B23
:1095900020830AC0BE0102C0660F771F8A95E2F7DA
:1095A000CB018095822380838091D2148823A1F0FF
:1095B0008091B5039091B603009749F1E091B7030C
:1095C000F091B803808190E00090B90302C09595B6
:1095D00087950A94E2F713C08091AE039091AF0390
:1095E0000097A9F0E091B003F091B103808190E081
:1095F0000090B20302C0959587950A94E2F78170B6
:1096000090709091B714981711F00C94D653E09184
:109610009903F0919A032081CE0100909D0302C02E
:10962000880F991F0A94E2F7282B20838091591400
:1096300090915A14A0915B14B0915C144091D11494
:10964000552747FD5095652F752F840F951FA61F31
:10965000B71F8093591490935A14A0935B14B0933E
:109660005C14E0919903F0919A032081CE0100905F
:109670009D0302C0880F991F0A94E2F78095822308
:1096800080838091D8149091D914A091DA14B0916C
:10969000DB140196A11DB11D8093D8149093D914A9
:1096A000A093DA14B093DB148091FC14882309F49E
:1096B00014C18091051590910615A0910715B091E0
:1096C00008150091FD141091FE142091FF143091A3
:1096D0000015080F191F2A1F3B1F0093FD1410933C
:1096E000FE142093FF143093001510161106120675
:1096F00013060CF0F2C040910115509102156091D3
:10970000031570910415481759076A077B070CF079
:10971000E4C08091F5149091F614A091F714B091E3
:10972000F814081B190B2A0B3B0B0093FD14109324
:10973000FE142093FF14309300158091F9148823B0
:1097400051F180914814909149144091FA14242FBA
:10975000332727FD3095820F931F909349148093F0
:10976000481480915D1490915E14A0915F14B091A3
:109770006014552747FD5095652F752F840F951F51
:10978000A61FB71F80935D1490935E14A0935F147F
:10979000B09360148FC09091FB148091E1148111FB
:1097A0009C25E091C303F091C4038091C7032081FD
:1097B000992349F0DE0102C0AA0FBB1F8A95E2F788
:1097C0002A2B20830AC08E0102C0000F111F8A9528
:1097D000E2F7C8018095822380838091FB1488235F
:1097E000A1F08091D8039091D903009749F1E091BD
:1097F000DA03F091DB03808190E00090DC0302C08B
:10980000959587950A94E2F713C08091D1039091C2
:10981000D2030097A9F0E091D303F091D4038081A3
:1098200090E00090D50302C0959587950A94E2F7E1
:10983000817090709091E014981711F00C94DA53A5
:10984000E091BC03F091BD032081CE010090C003E4
:1098500002C0880F991F0A94E2F7282B2083809179
:109860005D1490915E14A0915F14B09160144091CA
:10987000FA14552747FD5095652F752F840F951FB6
:10988000A61FB71F80935D1490935E14A0935F147E
:10989000B0936014E091BC03F091BD032081CE0130
:1098A0000090C00302C0880F991F0A94E2F78095C8
:1098B000822380838091011590910215A091031558
:1098C000B09104150196A11DB11D809301159093CF
:1098D0000215A0930315B0930415809125158823D4
:1098E00009F413C180912E1590912F15A091301578
:1098F000B09131150091261510912715209128154A
:1099000030912915080F191F2A1F3B1F0093261598
:10991000109327152093281530932915101611063A
:10992000120613060CF0F1C040912A1550912B1528
:1099300060912C1570912D15481759076A077B0700
:109940000CF0E3C080911E1590911F15A091201579
:10995000B0912115081B190B2A0B3B0B0093261500
:1099600010932715209328153093291580912215DF
:10997000882351F180914A1490914B144091231502
:10998000242F332727FD3095820F931F90934B147C
:1099900080934A148091611490916214A091631491
:1099A000B0916414552747FD5095652F752F840F8E
:1099B000951FA61FB71F8093611490936214A09304
:1099C0006314B09364148EC09091241580910A158D
:1099D00081119C25E091E603F091E7038091EA0371
:1099E0002081992349F0AE0102C0440F551F8A958A
:1099F000E2F7242B20830AC0BE0102C0660F771F46
:109A00008A95E2F7CB01809582238083809124158B
:109A10008823A1F08091FB039091FC03009741F112
:109A2000E091FD03F091FE03808190E00090FF0340
:109A300002C0959587950A94E2F713C08091F403CC
:109A40009091F5030097A1F0E091F603F091F703F0
:109A5000808190E00090F80302C0959587950A9464
:109A6000E2F78170907090910915981709F0A6C6D9
:109A7000E091DF03F091E0032081CE010090E30349
:109A800002C0880F991F0A94E2F7282B2083809147
:109A9000611490916214A0916314B0916414409188
:109AA0002315552747FD5095652F752F840F951F5A
:109AB000A61FB71F8093611490936214A093631440
:109AC000B0936414E091DF03F091E0032081CE01B4
:109AD0000090E30302C0880F991F0A94E2F7809573
:109AE0008223808380912A1590912B15A0912C15AB
:109AF000B0912D150196A11DB11D80932A1590934B
:109B00002B15A0932C15B0932D158091BB0B909124
:109B1000BC0BA091BD0BB091BE0B0196A11DB11D58
:109B20008093BB0B9093BC0BA093BD0BB093BE0B6B
:109B30008091BB0B9091BC0BA091BD0BB091BE0B63
:109B4000E091CD0BF091CE0B4489558966897789D8
:109B500084179507A607B70720F483948D140CF497
:109B6000D7C94091BB0B5091BC0B6091BD0B70915C
:109B7000BE0BE091CD0BF091CE0B84A595A5A6A5CB
:109B8000B7A584179507A607B70708F4BDC080904E
:109B9000DD0B9090DE0BA090DF0BB090E00B44A9A2
:109BA00055A966A977A995018401AA27059FB12D1A
:109BB000169FE001269FD00D259FC00DD11D069F49
:109BC000B00DC11DDA1F159FB00DC11DDA1F249FF6
:109BD000B00DC11DDA1F149FB10DCA1FDA1FB69553
:109BE000CA1FDA1F1124DF01AA59BF4F8D919C9122
:109BF0008C0F9D1F9093DC0B8093DB0BE25AFF4F81
:109C00004081518162817381A0E0B0E0481759071B
:109C10006A077B0720F45093DC0B4093DB0B8091A9
:109C2000DB0B9091DC0B9F3460F09D3930F4E3E066
:109C300096958795EA95E1F702C088E893E128E0D8
:109C400014C0983230F0969587959695879524E0C4
:109C50000CC0943120F09695879522E006C08032A2
:109C6000910510F480E290E021E02093D70B8097DB
:109C700018E080309107C8F0E92FF0E0EE0FFF1FE9
:109C8000EE0FFF1FEA58FE4F459155916591749173
:109C90006A01AB01AA27859F9001849F210D3A1F7D
:109CA00006942A1F3A1F11241AC0FC01F695E79565
:109CB000EC7FEA58FA4F45915591659174916A018C
:109CC00090E087709070869F9001879F300D969FDF
:109CD000300D112443E0369527954A95E1F7C21AD5
:109CE000D30AD0929900C0929800EE24FF24C80CA9
:109CF000D91CEA1CFB1CC092DD0BD092DE0BE0925B
:109D0000DF0BF092E00B3AC14091BB0B5091BC0BC2
:109D10006091BD0B7091BE0B80A991A9A2A9B3A9B6
:109D20002091E20B3091E30B84179507A607B70744
:109D300008F00FC12115310531F481E090E09093D6
:109D4000E30B8093E20B8091E20B9091E30B813067
:109D5000910571F482E090E09093E30B8093E20B25
:109D60001092E40B1092E50B1092E60B1092E70BA9
:109D7000DF01A05CBF4F4091E40B5091E50B609177
:109D8000E60B7091E70B8D919D910D90BC91A02DEC
:109D9000480F591F6A1F7B1F4093E40B5093E50B3C
:109DA0006093E60B7093E70B8090D30B9090D40BED
:109DB000A090D50BB090D60B44A955A966A977A958
:109DC00095018401AA27059FB12D169FC001269FEA
:109DD000900D259F800D911D069FB00D811D9A1F2E
:109DE000159FB00D811D9A1F249FB00D811D9A1FD4
:109DF000149FB10D8A1F9A1FB6958A1F9A1F1124AE
:109E00009093E90B8093E80B4091DB0B5091DC0BB6
:109E10002091CD0B3091CE0B4817590758F4265995
:109E20003F4FD9018D919C9111979093E90B8093AD
:109E3000E80B1AC0FA01E81BF90BCF01F093E90B0C
:109E4000E093E80B26593F4FD9014D915D916D91FB
:109E50007C91A0E0B0E084179507A607B70720F42F
:109E60005093E90B4093E80B8091E80B9091E90B3C
:109E70009F3460F09D3930F423E0969587952A95BC
:109E8000E1F702C088E893E128E014C0983230F08E
:109E9000969587959695879524E00CC0943120F08F
:109EA0009695879522E006C08032910510F480E2F5
:109EB00090E021E02093D70B8097B8E080309B079B
:109EC000C8F0E92FF0E0EE0FFF1FEE0FFF1FEA587A
:109ED000FE4F45915591659174916A01FB01AA2746
:109EE0008F9F90018E9F210D3A1F06942A1F3A1FC3
:109EF00011241AC0FC01F695E795EC7FEA58FA4F59
:109F000045915591659174916A0190E087709070C8
:109F1000869F9001879F300D969F300D1124C3E0DE
:109F200036952795CA95E1F7C21AD30AD0929900BF
:109F3000C0929800EE24FF24C80CD91CEA1CFB1C1C
:109F4000C092D30BD092D40BE092D50BF092D60BEB
:109F500015C02115310531F481E090E09093E30BB9
:109F60008093E20B8091D80B9091D90B909399003C
:109F7000809398008091DA0B8093D70B4091BB0BB4
:109F80005091BC0B6091BD0B7091BE0BE091CD0B5D
:109F9000F091CE0B84899589A689B789481759070E
:109FA0006A077B0708F4E6C31092CE0B1092CD0B24
:109FB0009091F10B8091F00B981731F08091F00B9C
:109FC0008F5F8F708093F00B9091F10B8091F00B6D
:109FD0009817A1F02091F00B30E087E790E0289FE0
:109FE000F001299FF00D389FF00D1124EE50F44F31
:109FF000DF01AC58BF4F81E08C9302C0E0E0F0E09D
:10A00000F093CE0BE093CD0B309709F4B5C3808D60
:10A01000918DA28DB38D8093511490935214A0937F
:10A020005314B0935414848D958DA68DB78D809361
:10A03000551490935614A0935714B093581480A1BC
:10A0400091A1A2A1B3A18093591490935A14A09303
:10A050005B14B0935C1484A195A1A6A1B7A18093D1
:10A060005D1490935E14A0935F14B093601480A568
:10A0700091A5A2A5B3A58093611490936214A093B7
:10A080006314B093641482AD8093CF0B8091D00B96
:10A090008823E1F18F01C1EDDBE069EC7BE040E07A
:10A0A00050E0F80184859585A685B7850097A105C0
:10A0B000B10511F188818823F9F0FA01E953F44FD1
:10A0C0008081FA01EE0FFF1FE85BFB4E882349F009
:10A0D00080819181DB012D913C911197821B930B23
:10A0E00008C080819181DB012D913C911197820FF5
:10A0F000931F9183808318824F5F5F4F0C5F1F4FC8
:10A1000021966E5F7F4F4230510559F61092D30B66
:10A110001092D40B1092D50B1092D60BC091CD0B90
:10A12000D091CE0BFE01E25AFF4F208131813F34A6
:10A1300060F03D3930F443E0369527954A95E1F7D4
:10A1400002C028E833E188E014C0383230F0369598
:10A1500027953695279584E00CC0343120F036954C
:10A16000279582E006C02032310510F420E230E06D
:10A1700081E08093D70B20523040B8E020303B077D
:10A18000C8F0E32FF0E0EE0FFF1FEE0FFF1FEA58BD
:10A19000FE4F85919591A591B491AC01BD01AA277F
:10A1A000279FC001269F810D9A1F06948A1F9A1F20
:10A1B00011241AC0F901F695E795EC7FEA58FA4F99
:10A1C00085919591A591B491AC0130E027703070E4
:10A1D0002A9FC0012B9F900D3A9F900D112413E0F0
:10A1E000969587951A95E1F7481B590B5093D90B13
:10A1F0004093D80B8091D70B8093DA0BFE01EE5879
:10A20000FF4F8081882309F472C0CA59DF4F28812B
:10A2100039813093DC0B2093DB0B3F3460F03D3908
:10A2200030F4A3E036952795AA95E1F702C028E817
:10A2300033E188E014C0383230F0369527953695F2
:10A24000279584E00CC0343120F03695279582E0C4
:10A2500006C02032310510F420E230E081E0809326
:10A26000D70B20523040E8E020303E07C8F0E32F03
:10A27000F0E0EE0FFF1FEE0FFF1FEA58FE4F859133
:10A280009591A591B491AC01BD01AA27279FC0016A
:10A29000269F810D9A1F06948A1F9A1F11241AC0A7
:10A2A000F901F695E795EC7FEA58FA4F859195917B
:10A2B000A591B491AC0130E0277030702A9FC001A5
:10A2C0002B9F900D3A9F900D112463E096958795F2
:10A2D0006A95E1F7481B590BCA01A0E0B0E08093F2
:10A2E000DD0B9093DE0BA093DF0BB093E00B50934C
:10A2F000990040939800E091CD0BF091CE0B80AD8A
:10A300008093E10BEA58FF4F20818091481490918F
:10A310004914009719F480915E158111286080918D
:10A320004A1490914B14009719F480915F15811194
:10A33000206180914614281709F442C0E1E6F3E059
:10A34000EF01249640E050E061E070E0CB01042E84
:10A3500002C0880F991F0A94E2F7A82F3091461483
:10A360003227382331F1A22390914614AA2389F091
:10A37000982B90934614A081B1813C91CB01088029
:10A3800002C0880F991F0A94E2F7809583238C936B
:10A3900010C08095892380934614A081B1813C919F
:10A3A000CB01088002C0880F991F0A94E2F7382B6E
:10A3B0003C934F5F5F4FB396A3964530510531F6FE
:10A3C000E091CD0BF091CE0BDF01AB58BF4FDC918C
:10A3D0007489658956894789C091E10B0081118193
:10A3E0002281338181E0011511052105310509F430
:10A3F00080E080938114882309F444C0872F962F2E
:10A40000A52FB42FEE24E394EC22AC01BD01759589
:10A4100067955795479570956095509541955F4F15
:10A420006F4F7F4F40938214509383146093841432
:10A430007093851441E0D11140E0409379148093EA
:10A440007A1490937B14A0937C14B0937D140093A2
:10A450008A1410938B1420938C1430938D14EE2057
:10A4600011F08FEF01C081E080937F1481E08E2591
:10A47000809380141092861410928714109288147E
:10A4800010928914748965895689478904811581D8
:10A490002681378181E0011511052105310509F477
:10A4A00080E08093AA14882309F446C0872F962F52
:10A4B000A52FB42FEE24E394C1FFEE24AC01BD011F
:10A4C0007595679557954795709560955095419509
:10A4D0005F4F6F4F7F4F4093AB145093AC1460931A
:10A4E000AD147093AE1441E0D13009F040E04093D8
:10A4F000A2148093A3149093A414A093A514B093D2
:10A50000A6140093B3141093B4142093B51430938D
:10A51000B614EE2011F08FEF01C081E08093A814F3
:10A5200081E08E258093A9141092AF141092B0147C
:10A530001092B1141092B2147489658956894789B2
:10A54000008511852285338581E0011511052105DE
:10A55000310509F480E08093D314882309F446C0C0
:10A56000872F962FA52FB42FEE24E394C2FFEE245D
:10A57000AC01BD01759567955795479570956095A8
:10A58000509541955F4F6F4F7F4F4093D414509338
:10A59000D5146093D6147093D71441E0D23009F0EB
:10A5A00040E04093CB148093CC149093CD14A093AF
:10A5B000CE14B093CF140093DC141093DD142093C9
:10A5C000DE143093DF14EE2011F08FEF01C081E034
:10A5D0008093D11481E08E258093D2141092D814E8
:10A5E0001092D9141092DA141092DB1474896589D0
:10A5F00056894789048515852685378581E00115AB
:10A6000011052105310509F480E08093FC148823AD
:10A6100009F446C0872F962FA52FB42FEE24E3947C
:10A62000C3FFEE24AC01BD0175956795579547951D
:10A6300070956095509541955F4F6F4F7F4F409358
:10A64000FD145093FE146093FF147093001541E0C5
:10A65000D33009F040E04093F4148093F5149093C4
:10A66000F614A093F714B093F81400930515109303
:10A6700006152093071530930815EE2011F08FEF83
:10A6800001C081E08093FA1481E08E258093FB1451
:10A6900010920115109202151092031510920415D4
:10A6A000DF01AB58BF4FDC91E488058936892789E3
:10A6B000408951896289738981E04115510561059D
:10A6C000710509F480E080932515882309F445C0BD
:10A6D0008E2D902FA32FB22FE1E0C4FFE0E08C017C
:10A6E0009D013595279517950795309520951095DF
:10A6F00001951F4F2F4F3F4F00932615109327159D
:10A70000209328153093291521E0D43009F020E05A
:10A7100020931D1580931E1590931F15A09320154F
:10A72000B093211540932E1550932F15609330153B
:10A7300070933115EE2311F08FEF01C081E080930B
:10A74000231581E08E278093241510922A151092EC
:10A750002B1510922C1510922D151092E30B1092C0
:10A76000E20B1092BB0B1092BC0B1092BD0B10921F
:10A77000BE0B02C080E001C081E0DF91CF911F914C
:10A780000F91FF90EF90DF90CF90BF90AF909F9090
:10A790008F907F906F905F904F90089510924C141F
:10A7A0000C94FF4810924D140C94184A10924E14B9
:10A7B0000C94314B10924F140C944A4C109250143C
:10A7C00081C97091EA0B7F5F7093EA0B8091EB0B6C
:10A7D0008F5F8093EB0B5091EC0B6091EE0B40E0A0
:10A7E00081E090E052C02091E114E091C303F09128
:10A7F000C4037081222309F0EDC09C010090C703BF
:10A8000002C0220F331F0A94E2F7209527232083EA
:10A8100020914814309149142F5F3F4F21C020915F
:10A82000481430914914121613066CF52091E11466
:10A83000E091C303F091C4037081222309F0D5C0D5
:10A840009C010090C70302C0220F331F0A94E2F755
:10A85000722B70832091481430914914215030405C
:10A860003093491420934814E091BC03F091BD0348
:10A8700070819C010090C00302C0220F331F0A9414
:10A88000E2F7722B70834F5F70E020914814309193
:10A8900049142115310511F0751760F47093EA0B16
:10A8A0005091ED0B6091EF0B7091EB0B40E081E06C
:10A8B00090E06BC0461791F3E091BC03F091BD03AB
:10A8C00070819C010090C00302C0220F331F0A94C4
:10A8D000E2F72095272320832091481430914914D2
:10A8E00037FF9DCF80CF20910A15E091E603F091CC
:10A8F000E7037081222309F084C09C010090EA03E1
:10A9000002C0220F331F0A94E2F7209527232083E9
:10A9100020914A1430914B142F5F3F4F21C020915A
:10A920004A1430914B14121613066CF520910A1537
:10A93000E091E603F091E7037081222309F06CC0F7
:10A940009C010090EA0302C0220F331F0A94E2F731
:10A95000722B708320914A1430914B142150304057
:10A9600030934B1420934A14E091DF03F091E003FD
:10A9700070819C010090E30302C0220F331F0A94F0
:10A98000E2F7722B70834F5F70E020914A14309190
:10A990004B142115310509F44BC0751708F448C054
:10A9A000461709F445C0E091DF03F091E0037081A0
:10A9B0009C010090E30302C0220F331F0A94E2F7C8
:10A9C00020952723208320914A1430914B1437FF80
:10A9D000A6CF89CF9C010090C70302C0220F331F6E
:10A9E0000A94E2F7722B708313CF9C010090C70387
:10A9F00002C0220F331F0A94E2F7209527232083F9
:10AA000029CF9C010090EA0302C0220F331F0A9451
:10AA1000E2F7722B70837CCF9C010090EA0302C0A6
:10AA2000220F331F0A94E2F720952723208392CF29
:10AA30007093EB0B08952F923F924F925F927F920B
:10AA40008F929F92AF92BF92CF92DF92EF92FF923E
:10AA50000F931F93CF93DF930F920F92CDB7DEB773
:10AA60001092CF0B1FEB412E1BE0512E0AEE202E31
:10AA70000BE0302E8EEEA82E8BE0B82E8CEE9BE0F5
:10AA80009A8389838824992477247394F201C1904E
:10AA9000D190E190F1902F01882D8D5F0E942D6D56
:10AAA0009B01AC01C701B6010E94FEE39B01AC0112
:10AAB00060E070E48CE196E40E94E3E1C62EE72EAC
:10AAC000182F092F9801862F9E2DA32FB22FBC017E
:10AAD000CD0120E030E040E85FE30E94FAE3980116
:10AAE00018166CF48C2D9E2DA32FB22FBC01CD0116
:10AAF0000E94CCE1C62EE72E182F092F12C08C2DF4
:10AB00009E2DA32FB22FBC01CD0120E030E040E804
:10AB10005FE30E94DFE187FF04C0CC24EE2410E055
:10AB200000E098018C2D9E2DA32FB02FBC01CD01EC
:10AB30000E948AE2F62EE981FA816193FA83E98321
:10AB4000F50110826623A1F460E070E080E89FE3E5
:10AB5000412FF02F0C2D1E2D242F3F2FA9019801DE
:10AB60000E94E3E10E94CCE10E948AE2F501608349
:10AB7000F5018081882309F47082F401EE0FFF1F34
:10AB8000E85BFB4E11821082F101F1921F010894E3
:10AB9000811C911C0894A11CB11CF2E08F16910439
:10ABA00009F074CF0F900F90DF91CF911F910F910B
:10ABB000FF90EF90DF90CF90BF90AF909F908F90DD
:10ABC0007F905F904F903F902F9008952091F10BD0
:10ABD0009091F00B81E0291380E00895CF92DF92ED
:10ABE000EF92FF920F931F93CF93DF93E9012FB75B
:10ABF000F894DC01CD90DD90ED90FC90C092511462
:10AC0000D0925214E0925314F0925414FB018081BC
:10AC10009181A281B3818093551490935614A0938F
:10AC20005714B0935814FA0180819181A281B381A5
:10AC30008093591490935A14A0935B14B0935C14AE
:10AC400088819981AA81BB8180935D1490935E1461
:10AC5000A0935F14B0936014F80180819181A28168
:10AC6000B3818093611490936214A0936314B093A2
:10AC700064142FBFDF91CF911F910F91FF90EF9040
:10AC8000DF90CF900895CF92DF92EF92FF920F93D3
:10AC90001F93CF93DF93FB01EA0169012FB7F8946B
:10ACA0004091511450915214609153147091541466
:10ACB000DC014D935D936D937C93139780915514B4
:10ACC00090915614A0915714B09158148083918399
:10ACD000A283B3838091591490915A14A0915B146C
:10ACE000B0915C1488839983AA83BB8380915D149F
:10ACF00090915E14A0915F14B0916014F60180836E
:10AD00009183A283B3838091611490916214A09186
:10AD10006314B0916414F80180839183A283B38398
:10AD20008091CF0BD7018C932FBFDF91CF911F91D3
:10AD30000F91FF90EF90DF90CF9008958091710078
:10AD40008D7F8093710006C08091F00B8F5F8F70B4
:10AD50008093F00B9091F10B8091F00B981709F014
:10AD60005DC01092CE0B1092CD0B2FB7F89480914E
:10AD7000511490915214A0915314B0915414809393
:10AD8000771390937813A0937913B0937A138091EB
:10AD9000551490915614A0915714B0915814809363
:10ADA0007B1390937C13A0937D13B0937E138091BB
:10ADB000591490915A14A0915B14B0915C14809333
:10ADC0007F1390938013A0938113B093821380918B
:10ADD0005D1490915E14A0915F14B0916014809303
:10ADE000831390938413A0938513B093861380915B
:10ADF000611490916214A0916314B09164148093D3
:10AE0000871390938813A0938913B0938A132FBF4D
:10AE10008091710082608093710008959091F10B90
:10AE20008091F00B981709F495CF8ECF8093D00BBB
:10AE300081E08093D10B8093D20B08959C0190EC1C
:10AE400080E4889410F0381710F0381B892B969501
:10AE5000220F331F89279E7FA9F710F0220F830747
:10AE6000891F08952F923F924F925F926F927F9227
:10AE70008F929F92AF92BF92CF92DF92EF92FF920A
:10AE80000F931F93CF93DF93CDB7DEB768970FB6BD
:10AE9000F894DEBF0FBECDBF1C0168017901FC0133
:10AEA000EE58FF4F80818823C1F08A019B01013059
:10AEB00040E0140741E0240740E0340724F000E0BC
:10AEC00010E021E030E051E0C51650E0D50651E039
:10AED000E50650E0F5062CF409C000E010E021E0A2
:10AEE00030E0C12CD12C81E0E82EF12C8EE5882EAB
:10AEF000912C820C931CF40180819181A281B381F9
:10AF000077276627A90198010E943FE0DC01CB0169
:10AF100080509048AF4FBF4F8D01332717FD3095BC
:10AF2000232F09831A832B833C83F4018081918131
:10AF3000A281B38177276627A70196010E943FE08F
:10AF4000DC01CB0180509048AF4FBF4F4D01BB2477
:10AF500097FCB094AB2C8D829E82AF82B88609811B
:10AF60001A812B813C81083711052105310548F4F0
:10AF7000B8E78B2E912CA12CB12C89829A82AB82BE
:10AF8000BC820D811E812F8138850837110521056E
:10AF9000310548F4A8E78A2E912CA12CB12C8D8282
:10AFA0009E82AF82B88669817A818B819C819B0168
:10AFB000AC010E94AAE469877A878B879C876D81A0
:10AFC0007E818F8198859B01AC010E94AAE46D87E8
:10AFD0007E878F87988B910122593F4FD901ED9041
:10AFE000FD900D911C911397ED8AFE8A0F8B188F9F
:10AFF00067017801CC0CDD1CEE1CFF1CF101EE5842
:10B00000FF4F80818823B9F1F101EE59FF4F808015
:10B010009180A280B380C114D104E104F10489F0CD
:10B02000C501B40109851A852B853C85601B710B10
:10B03000820B930BA70196010E941EE529013A019C
:10B0400003C044245524320122273327A9012C1997
:10B050003D094E095F09B9F06D857E858F85988918
:10B06000681979098A099B090E941EE5298B3A8B88
:10B070004B8B5C8B0CC0198A1A8A1B8A1C8A44244D
:10B080005524320104C0198A1A8A1B8A1C8AD101EC
:10B0900054968D909D90AD90BC905797D501C4016A
:10B0A00084199509A609B70909891A892B893C8948
:10B0B000801B910BA20BB30BB7FF40C0C114D1048E
:10B0C000E104F10429F1C701B601A50194010E9430
:10B0D000AAE4DC01CB0109851A852B853C85801B00
:10B0E000910BA20BB30B0D851E852F853889800F20
:10B0F000911FA21FB31FA7019601220F331F441FE8
:10B10000551FBC01CD010E941EE589019A0104C0B2
:10B1100000E010E020E030E02801390137FF03C0F3
:10B12000442455243201481459046A047B0414F061
:10B130002401350180E090E0A0E0B0E0530142013D
:10B14000880E991EAA1EBB1E8D869E86AF86B88A63
:10B15000F10123AD222309F430C10097A105B10507
:10B1600009F07FC0C301B2016F5F7F4F8F4F9F4FC8
:10B1700097FF24C090958095709561957F4F8F4F74
:10B180009F4F2D893E894F89588D0E94AAE4AB01BB
:10B19000BC01440F551F661F771F89849A84AB84B6
:10B1A000BC84481559056A057B0508F051C0D501D6
:10B1B000C401841B950BA60BB70B14C02D893E89C7
:10B1C0004F89588D0E94AAE4DC01CB01880F991F9A
:10B1D000AA1FBB1FE984FA840B851C858E0D9F1D59
:10B1E000A01FB11F803000E8900700E0A00700E03A
:10B1F000B00758F40E941E576C01EE24D7FCE0946F
:10B20000FE2C7601DD24CC2426C000E072E0B69549
:10B21000A795979587957A95D1F70F5F803010E8BD
:10B22000910710E0A10710E0B10780F70E941E57B8
:10B230006C01EE24D7FCE094FE2C7601DD24CC24B6
:10B2400004C0CC0CDD1CEE1CFF1C0A95D2F703C019
:10B25000CC24DD2476016701FF24D7FCF094EF2C89
:10B2600007C0F101E25AFF4FC080D180E280F38035
:10B270001414150416041704E4F46091DC1370919F
:10B28000DD138091DE139091DF1397018601898091
:10B290009A80AB80BC80081919092A093B09A801CA
:10B2A000332722270E943FE0DC01CB014D01B7FF8D
:10B2B00002C0882499244D855E856F8578894F5F0B
:10B2C0005F4F6F4F7F4FF10184899589A689B789B8
:10B2D000481759076A077B070CF078C00091DC1308
:10B2E0001091DD132091DE133091DF1309871A8747
:10B2F0002B873C87970186014D815E816F81788520
:10B30000041B150B260B370BA80133272227698551
:10B310007A858B859C850E943FE0DC01CB016D0125
:10B320006091D8137091D9138091DA139091DB1347
:10B330006115710581059105C9F120E030E044E611
:10B3400050E00E943FE069877A878B879C87F101F4
:10B35000E259FF4F8091510390E001964081518165
:10B360006281738104C075956795579547958A9555
:10B37000D2F7CA0177276627E988FA880B891C89E2
:10B38000A701332722270E94BDE09B01AC016985FC
:10B390007A858B859C850E943FE0DC01CB01CD0145
:10B3A000BB2797FDB095AB2FB7FF04C080E090E0BE
:10B3B000A0E0B0E0D7FE10C00DC080E090E0A0E0BB
:10B3C000B0E0CC24DD248824992406C080E090E0FD
:10B3D000A0E0B0E0CC24DD242FB7F894F101EC58C4
:10B3E000FF4F3081332309F040C0F101EE58FF4F89
:10B3F0003081332369F0F10144A655A666A677A6ED
:10B40000ED84FE840F851889E0AAF1AA02AB13AB84
:10B4100081010A591F4F49815A816B817C81F80152
:10B420004083518362837383810106591F4F4D818D
:10B430005E816F817885F8014083518362837383D5
:10B44000F10195AE84AED7AEC6AEEC5BFF4F118274
:10B450001082F101EA5BFF4F11821082F101E05C82
:10B46000FF4F80839183A283B3832FBF68960FB66B
:10B47000F894DEBF0FBECDBFDF91CF911F910F912A
:10B48000FF90EF90DF90CF90BF90AF909F908F9004
:10B490007F906F905F904F903F902F9008952F92E4
:10B4A0003F924F925F926F927F928F929F92AF9254
:10B4B000BF92CF92DF92EF92FF920F931F93CF93A1
:10B4C000DF9300D000D0CDB7DEB79E838D831B0104
:10B4D000009709F4B2C16115710509F4AEC19C0170
:10B4E000205B3F4FD9018D919D910D90BC91A02D76
:10B4F00089839A83AB83BC836D817E81645B7F4F3C
:10B50000FB0180819181A281B38129813A814B81A4
:10B510005C81281B390B4A0B5B0BDA01C9018130B6
:10B5200030E0930733E0A30730E0B3070CF485C1A4
:10B53000AD81BE81A35ABF4F8C91882309F069C1A8
:10B54000D101AD58BF4F8C91882309F462C1D1015C
:10B55000A45BBF4F8D919D910D90BC91A02D298131
:10B560003A814B815C8182179307A407B5070CF0E1
:10B5700050C19C01AD016CE05595479537952795D5
:10B580006A95D1F7ED81FE81E85AFF4F8080918066
:10B59000A280B380B094A09490948094811C911C5C
:10B5A000A11CB11C76E0B594A794979487947A95E2
:10B5B000D1F7ED81FE81EC5AFF4FC080D180E2804F
:10B5C000F38015E0F594E794D794C7941A95D1F7D2
:10B5D000CA01B9010E943FE02B013C01C701B6013D
:10B5E000A50194010E943FE0DC01CB01A30192017F
:10B5F000281B390B4A0B5B0BDA01C90100E00097ED
:10B60000A105B10509F44BC0AC01BD0140705070FB
:10B610006070707E411551056105710549F432E095
:10B62000880F991FAA1FBB1F3A95D1F70F5FE7CF6D
:10B63000181619061A061B0694F5CD01BB2797FDAF
:10B64000B095AB2F0730A8F00E941E57AC016627BB
:10B6500057FD6095762FBA0155274427802F90E03B
:10B66000069704C075956795579547958A95D2F7C3
:10B670001AC00E941E57AC01662757FD6095762FB1
:10B68000BA015527442786E090E0801B910904C049
:10B69000440F551F661F771F8A95D2F704C040E0FC
:10B6A00050E060E070E089819A81AB81BC818417B1
:10B6B0009507A607B7074CF4ED81FE81E05BFF4FCD
:10B6C00080819181A281B3819FC0F101E45BFF4F32
:10B6D00000811181228133816CE035952795179582
:10B6E00007956A95D1F7ED81FE81E85AFF4F80807A
:10B6F0009180A280B380B094A09490948094811C97
:10B70000911CA11CB11C76E0B594A79497948794E2
:10B710007A95D1F7ED81FE81EC5AFF4FC080D18040
:10B72000E280F380A5E0F594E794D794C794AA95B6
:10B73000D1F7C901B801A90198010E943FE02B018E
:10B740003C01C701B601A50194010E943FE0DC0164
:10B75000CB01A3019201281B390B4A0B5B0BDA01C9
:10B76000C90100E00097A105B10509F449C0AC0189
:10B77000BD01407050706070707E411551056105CB
:10B78000710549F452E0880F991FAA1FBB1F5A95F3
:10B79000D1F70F5FE7CF181619061A061B0684F5B6
:10B7A000CD01BB2797FDB095AB2F0730A0F00E94CD
:10B7B0001E57AA2797FDA095BA2FDC019927882745
:10B7C00010E00650104004C0B595A7959795879551
:10B7D0000A95D2F719C00E941E57AA2797FDA09577
:10B7E000BA2FDC019927882726E030E0201B310999
:10B7F00004C0880F991FAA1FBB1F2A95D2F704C047
:10B8000080E090E0A0E0B0E0ED81FE81E45BFF4FDE
:10B8100005C089819A81AB81BC81FB0180839183C2
:10B82000A283B383ED81FE81ED58FF4F81E08083D9
:10B83000ED81FE81E45AFF4F808326960FB6F8947F
:10B84000DEBF0FBECDBFDF91CF911F910F91FF9053
:10B85000EF90DF90CF90BF90AF909F908F907F90B0
:10B860006F905F904F903F902F900895EF92FF92CE
:10B870000F931F93CF93DF931091F10B8FB7F89431
:10B880000091F00B8FBF60E070E087E7E82EF12CAD
:10B8900013C0112309F410E11150812F90E08E9D07
:10B8A000E0018F9DD00D9E9DD00D1124CE50D44F20
:10B8B000CE010E944F5ABE01101759F7DF91CF9168
:10B8C0001F910F91FF90EF9008952F923F924F920A
:10B8D0005F926F927F928F929F92AF92BF92CF9220
:10B8E000DF92EF92FF920F931F93CF93DF9300D0DD
:10B8F00000D0CDB7DEB79E838D831B01009709F47E
:10B90000C6C1FB01EE58FF4F8081882309F4BFC1F7
:10B91000ED81FE81E35AFF4F8081882309F0B7C192
:10B92000ED81FE81ED58FF4F8081882309F4AFC17E
:10B93000ED81FE81E85BFF4F80819181A281B3811F
:10B94000FB01E85BFF4F4081518162817381841765
:10B950009507A607B707CCF4ED81FE81E45BFF4FA6
:10B9600080819181A281B38181509040AD4FBF4FC2
:10B97000F101E45BFF4F4081518162817381841743
:10B980009507A607B70704F582C1481759076A0744
:10B990007B070CF07CC1ED81FE81E45BFF4F808171
:10B9A0009181A281B38180509040AD4FBF4FF10192
:10B9B000E45BFF4F40815181628173818417950759
:10B9C000A607B7070CF063C19101245B3F4FD90173
:10B9D0008D919D910D90BC91A02D89839A83AB830D
:10B9E000BC83ED81FE81E45BFF4F008111812281E8
:10B9F00033814CE035952795179507954A95D1F7F2
:10BA0000ED81FE81E85AFF4F80809180A280B38053
:10BA100056E0B594A794979487945A95D1F7ED8101
:10BA2000FE81EC5AFF4FC080D180E280F38065E058
:10BA3000F594E794D794C7946A95D1F7C901B801F2
:10BA4000A90198010E943FE02B013C01C701B6010A
:10BA5000A50194010E943FE0DC01CB01840D951DFE
:10BA6000A61DB71D00E00097A105B10509F44BC064
:10BA7000AC01BD01407050706070707E4115510581
:10BA80006105710549F432E0880F991FAA1FBB1F99
:10BA90003A95D1F70F5FE7CF181619061A061B065D
:10BAA00094F5CD01BB2797FDB095AB2F0730A8F0DB
:10BAB0000E941E57AC01662757FD6095762FBA018C
:10BAC00055274427802F90E0069704C07595679509
:10BAD000579547958A95D2F71AC00E941E57AC0118
:10BAE000662757FD6095762FBA015527442786E0D3
:10BAF00090E0801B910904C0440F551F661F771FFB
:10BB00008A95D2F704C040E050E060E070E089819F
:10BB10009A81AB81BC8184179507A607B70744F4C7
:10BB2000F101E45BFF4F408151816281738196C0D6
:10BB3000ED81FE81E45BFF4F008111812281338121
:10BB40006CE035952795179507956A95D1F7ED81A6
:10BB5000FE81E85AFF4F80809180A280B38076E01A
:10BB6000B594A794979487947A95D1F7ED81FE8147
:10BB7000EC5AFF4FC080D180E280F380A5E0F594BD
:10BB8000E794D794C794AA95D1F7C901B801A90140
:10BB900098010E943FE02B013C01C701B601A501BD
:10BBA00094010E943FE0DC01CB01840D951DA61D90
:10BBB000B71D00E00097A105B10509F44BC0AC0129
:10BBC000BD01407050706070707E41155105610577
:10BBD000710549F452E0880F991FAA1FBB1F5A959F
:10BBE000D1F70F5FE7CF181619061A061B0694F552
:10BBF000CD01BB2797FDB095AB2F0730A8F00E9471
:10BC00001E57AC01662757FD6095762FBA01552760
:10BC1000442710E00650104004C07595679557956D
:10BC200047950A95D2F71AC00E941E57AC016627A5
:10BC300057FD6095762FBA015527442786E090E09E
:10BC4000801B910904C0440F551F661F771F8A95FA
:10BC5000D2F704C040E050E060E070E0F101E45B46
:10BC6000FF4F80819181A281B38184179507A60738
:10BC7000B70769F04083518362837383F101E45A0B
:10BC8000FF4F81E08083F101ED58FF4F80832696BE
:10BC90000FB6F894DEBF0FBECDBFDF91CF911F91DD
:10BCA0000F91FF90EF90DF90CF90BF90AF909F905B
:10BCB0008F907F906F905F904F903F902F9008955E
:10BCC000EF92FF920F931F93CF93C091F00B80E000
:10BCD00090E077E7E72EF12C13C02C2F30E02E9D5B
:10BCE00080012F9D100D3E9D100D11240E50144FFC
:10BCF000B8010E94655CCF5FC03109F4C0E0C801A3
:10BD00002091F10BC21749F7CF911F910F91FF902E
:10BD1000EF9008956F927F928F929F92AF92BF9211
:10BD2000CF92DF92FF920F931F93CF93DF93F09008
:10BD3000F00BC0E0D0E0E7E76E2E712C59C08F2DDC
:10BD400090E0869D6001879DD00C969DD00C1124BB
:10BD500082EF9BE0C80ED91E209709F443C0FE0174
:10BD6000EE58FF4F80818823E9F1F601EE58FF4F2E
:10BD700080818823B9F1FE01E45AFF4F8081882336
:10BD800031F4F601E45AFF4F8081882359F1FE0116
:10BD9000E45BFF4F60817181828193818E01085B3A
:10BDA0001F4FF80120813181428153810E94BDE003
:10BDB0004B015C01F601E45BFF4F60817181828180
:10BDC0009381F80120813181428153810E94BDE03D
:10BDD0008B019C01CE01B501A4010E943257C45AC7
:10BDE000DF4F1882F394F0E1FF1609F4FF24E60117
:10BDF0008091F10BF81609F0A2CF2097D1F0FE0147
:10BE0000E45BFF4F6081718182819381FE01E85B79
:10BE1000FF4F20813181428153810E94BDE08B011F
:10BE20009C01CE01B901A8010E943257C45ADF4FCC
:10BE30001882DF91CF911F910F91FF90DF90CF90EB
:10BE4000BF90AF909F908F907F906F9008950E94C9
:10BE5000365C0E94605E0E948A5E08950F93DC014A
:10BE6000CB011092F10B1092F00B10922E14109245
:10BE70002F141092301410923114109277131092E4
:10BE800078131092791310927A1310927B131092F8
:10BE90007C1310927D1310927E1310927F131092D8
:10BEA00080131092811310928213109283131092B8
:10BEB0008413109285131092861310928713109298
:10BEC00088131092891310928A138093DC13909335
:10BED000DD13A093DE13B093DF132093D8133093B8
:10BEE000D9134093DA135093DB130093621381E06C
:10BEF000809352030F9108952F923F924F925F9239
:10BF00006F927F928F929F92AF92BF92CF92DF9269
:10BF1000EF92FF920F931F93CF93DF93CDB7DEB7CE
:10BF2000C354D0400FB6F894DEBF0FBECDBF6F8BA9
:10BF3000788F898F9A8F5CA34BA319018091F4139A
:10BF40009091F513009749F09091F10B8091F00BCF
:10BF5000981719F481E080935203F090F10B1F2D94
:10BF60001F5F1CA7103109F41CA68091F10B90E013
:10BF700027E730E0829FA001839F500D929F500DD4
:10BF800011244E50544F5E8B4D8BFA01EC58FF4FED
:10BF90001082FA01EE58FF4F0083DA01DA96EC9234
:10BFA0008FB7F8940091771310917813209179133B
:10BFB00030917A13ED89FE89008F118F228F338F94
:10BFC00040917B1350917C1360917D1370917E138F
:10BFD0004F8F58A369A37AA3448F558F668F778FAD
:10BFE00040917F135091801360918113709182135F
:10BFF00048A759A76AA77BA740A351A362A373A32D
:10C00000409183135091841360918513709186132E
:10C010004DA75EA76FA778AB44A355A366A377A3EC
:10C0200040918713509188136091891370918A13FE
:10C0300049AB5AAB6BAB7CAB40A751A762A773A7C8
:10C040008FBF4090A7135090A8136090A9137090D1
:10C05000AA13ED89FE8940825182628273824091E7
:10C06000AB135091AC136091AD137091AE134B8F25
:10C070005C8F6D8F7E8F448355836683778380903A
:10C08000AF139090B013A090B113B090B21380860C
:10C090009186A286B386C090B313D090B413E0907B
:10C0A000B513F090B613C486D586E686F786409120
:10C0B000B7135091B8136091B9137091BA13408BB4
:10C0C000518B628B738B8091BC139091BD13A091A7
:10C0D000BE13B091BF13848B958BA68BB78BEB5897
:10C0E000FF4F8091BB13808341145104610471049C
:10C0F000C9F48B8D9C8DAD8DBE8D0097A105B105CA
:10C1000089F481149104A104B10461F4C114D1042F
:10C11000E104F10449F491E09FA341155105610543
:10C12000710521F41FA202C0A1E0AFA3ED89FE8931
:10C1300010AE8091631390916413A0916513B09138
:10C14000661380179107A207B30714F481E080AF4C
:10C150008091671390916813A0916913B0916A134D
:10C160000F8D18A129A13AA180179107A207B30743
:10C1700044F4AD89BE89D8968C91D8978260D896C0
:10C180008C9380916B1390916C13A0916D13B0916F
:10C190006E1308A519A52AA53BA580179107A2072C
:10C1A000B30744F4AD89BE89D8968C91D897846042
:10C1B000D8968C9380916F1390917013A091711306
:10C1C000B09172130DA51EA52FA538A98017910750
:10C1D000A207B30744F4AD89BE89D8968C91D8974D
:10C1E0008860D8968C938091731390917413A0916A
:10C1F0007513B091761309A91AA92BA93CA9801728
:10C200009107A207B3074CF4AD89BE89D8968C91EB
:10C21000D8978061D8968C93D897C114D104E10443
:10C22000F10449F0411551056105710559F4ED8995
:10C23000FE8911AE0EC0411551056105710511F061
:10C2400081E002C0F1018081AD89BE89D9968C93CD
:10C25000D997411451046104710429F08091471465
:10C260008160809347140B8D1C8D2D8D3E8D0115A3
:10C2700011052105310529F08091471482608093D2
:10C28000471481149104A104B10429F0809147144A
:10C29000846080934714C114D104E104F10429F0AF
:10C2A00080914714886080934714411551056105BA
:10C2B000710529F080914714806180934714809123
:10C2C0004714ED89FE89EA58FF4F808390916213ED
:10C2D000992311F0846006C081149104A104B10473
:10C2E00011F48B7F80838091F10B9091F00B891B6F
:10C2F0008F70282F30E03C8F2B8F2115310541F5B1
:10C300001092321410923314109234141092351487
:10C310001092361410923714109238141092391467
:10C3200010923A1410923B1410923C1410923D1447
:10C3300010923E1410923F14109240141092411427
:10C340001092421410924314109244141092451407
:10C35000EBA1FCA180819181A281B381ED89FE894D
:10C36000E25AFF4F80839183A283B3832091F41319
:10C370003091F5132115310509F453C08091520312
:10C38000882349F0EB8CFC8CE216F3060CF449C0D0
:10C390001092520346C00B8D1C8D021713070CF030
:10C3A00040C002301105ECF1C801AA2797FDA09505
:10C3B000BA2F7C01DD24CC24C901AA2797FDA095C2
:10C3C000BA2FAC0133272227C701B6010E94BDE076
:10C3D0006B017C016F89788D898D9A8DA7019601FB
:10C3E0000E943FE06F8B788F898F9A8F0D891E890D
:10C3F000025A1F4FF80180819181A281B381772772
:10C400006627A70196010E943FE0DC01CB01CD0128
:10C41000BB2797FDB095AB2FF80180839183A28352
:10C42000B383EF88F88C098D1A8DE114F1040105AE
:10C43000110509F469C02D893E892C5A3F4FFFA090
:10C44000FF20C9F0AD89BE89D996EC91F0E0EE0FDE
:10C45000FF1FEE0FFF1FE053FC4E80819181A281F0
:10C46000B381B7FF10C0B095A095909581959F4F6F
:10C47000AF4FBF4F08C08091C0139091C113A091DE
:10C48000C213B091C313F90180839183A283B38354
:10C49000ED89FE89EC5AFF4F208131814281538121
:10C4A00060E070E081E090E00E94BDE06F8F78A3D3
:10C4B00089A39AA36F89788D898D9A8D2F8D38A144
:10C4C00049A15AA10E943FE06B017C0114EC812E2E
:10C4D00013E1912E2E010894411C511C05E0D4015A
:10C4E0006D917D918D919D914D01A70196010E94C5
:10C4F0003FE0DC01CB01F20181939193A193B193D1
:10C500002F01015061F704C01F8E18A219A21AA2B0
:10C51000ED89FE89EE58FF4F8081882309F0A3C181
:10C52000EBA1FCA180819181A281B381ED89FE897B
:10C53000E25AFF4F80839183A283B383EF88F88C04
:10C54000098D1A8DE114F1040105110509F4CAC021
:10C550007E010894E11CF11C8AEF282E83E1382E1D
:10C560008701CC24412C512C91E0692E712CAC2CEC
:10C570004701D8013C9111962C91119712969C91EC
:10C58000129713968C9113970C5F1F4FC32ED22EC8
:10C59000E92EF82EF7FE08C0F094E094D094C094F1
:10C5A000C11CD11CE11CF11CF101608171818281EF
:10C5B00093816C157D058E059F05B4F4A701960146
:10C5C0000E94BDE0DC01CB01481659066A067B06D5
:10C5D0005CF0D1016D917D918D919C91A7019601A7
:10C5E0000E94BDE02B013C01A394E4E0F0E02E0E9C
:10C5F0003F1EF5E0AF1609F0BCCF7401EBA1FCA122
:10C6000080819181A281B3810D891E89025A1F4FB9
:10C610008030F0E89F07F0E0AF07F0E0BF0730F1AF
:10C62000F80180819181A281B38124E0B695A7951C
:10C63000979587952A95D1F780839183A283B383B9
:10C6400077276627A30192010E943FE0DC01CB011E
:10C65000CD01BB2797FDB095AB2F689413F8880FD9
:10C66000991FAA1FBB1F1694D1F712C0F801808131
:10C670009181A281B38177276627A30192010E944D
:10C680003FE0DC01CB01CD01BB2797FDB095AB2F7F
:10C69000F80180839183A283B383F0E04F16F0E02A
:10C6A0005F06F1E06F06F0E07F06E1F082E3C82E5E
:10C6B00084E1D82E00E0D7016D917D918D919D91FF
:10C6C0007D01A30192010E943FE0DC01CB01F60154
:10C6D00081939193A193B1936F010F5F053059F747
:10C6E00020E001C021E0AD89BE899C961D921D927B
:10C6F0001D921C929F97FD0184899589A689B7890F
:10C700000196A11DB11D80AB91ABA2ABB3AB2223AF
:10C71000E1F189819A81AB81BC818093321490933D
:10C720003314A0933414B09335148D819E81AF815E
:10C73000B8858093361490933714A0933814B0932F
:10C74000391489859A85AB85BC8580933A1490937A
:10C750003B14A0933C14B0933D148D859E85AF850A
:10C76000B88980933E1490933F14A0934014B093E3
:10C77000411489899A89AB89BC898093421490932A
:10C780004314A0934414B0934514ED89FE89E25AF2
:10C79000FF4F20813181428153810D891E890E59BD
:10C7A0001F4FCA01B9010E94AAE4DC01CB01F801C4
:10C7B00080839183A283B383FCA5F093F10B2FB701
:10C7C000F8948091631390916413A0916513B091D4
:10C7D00066138093771390937813A0937913B09393
:10C7E0007A138091671390916813A0916913B091A7
:10C7F0006A1380937B1390937C13A0937D13B09363
:10C800007E1380916B1390916C13A0916D13B09176
:10C810006E1380937F1390938013A0938113B09332
:10C82000821380916F1390917013A0917113B09146
:10C8300072138093831390938413A0938513B09302
:10C8400086138091731390917413A0917513B09116
:10C8500076138093871390938813A0938913B093D2
:10C860008A132FBF7BC5EFA0EE2009F078C00B8D97
:10C870001C8D0115110509F072C080918B139091E8
:10C880008C13A0918D13B0918E13181619061A06E9
:10C890001B060CF064C00D891E890C5A1F4FD8016D
:10C8A0006D917D918D919C91139716161706180620
:10C8B00019060CF054C02F89388D498D5A8D1216E7
:10C8C0001306140615060CF04AC00E94BDE0DC01F8
:10C8D000CB0120918B1330918C1340918D1350918B
:10C8E0008E1382179307A407B507CCF5D8016D9175
:10C8F0007D918D919C910E94BDE0062FC72E882EC0
:10C90000292EED88FE88EEE5F0E0EE0EFF1EF70121
:10C9100080819181A281B3813C0155244424602F00
:10C920007C2D882D922D2F89388D498D5A8D0E940E
:10C93000BDE09B01AC01C301B2010E943FE0DC01FC
:10C94000CB01CD01BB2797FDB095AB2FF7018083BD
:10C950009183A283B3830F8BC88E898E2A8EED8933
:10C96000FE89E25AFF4F20813181428153810D8936
:10C970001E890E591F4FCA01B9010E94AAE4DC01A9
:10C98000CB01F80180839183A283B383ED89FE8973
:10C99000E85BFF4FEF88F88C098D1A8DE082F182F9
:10C9A00002831383ED89FE8984899589A689B789D5
:10C9B0008030F0E89F07F0E0AF07F0E0BF0778F0C5
:10C9C000B595A79597958795772766272F8D38A1D9
:10C9D00049A15AA1220F331F441F551F06C07727B4
:10C9E00066272F8D38A149A15AA10E943FE06F8B85
:10C9F000788F898F9A8F0D891E8902591F4F2F8931
:10CA0000388D498D5A8DBA01992777FD9095892FD8
:10CA10003FA1332391F020911214309113144091CF
:10CA20001414509115140E94AAE4DC01CB01F80102
:10CA300080839183A283B3830DC12091161430911A
:10CA4000171440911814509119140E94AAE4DC01A3
:10CA5000CB01F80180839183A283B383ED88FE88A4
:10CA6000FCAEEBAE20EE33E138A32F8F4FE853E15D
:10CA70005EAB4DAB1DA619A708A7ABADBCADCD9065
:10CA8000DD90ED90FD90BCAFABAFC114D104E104DB
:10CA9000F10409F4CEC0AD89BE8954960D911D9163
:10CAA0002D913C91579709AB1AAB2BAB3CABEDA941
:10CAB000FEA980819181A281B38180179107A2078D
:10CAC000B30750F1AF8DB8A18D909D90AD90BC9003
:10CAD000E8A5F9A52081318142815381C701B601C2
:10CAE0000E94AAE46B017C01C501B40129A93AA9FD
:10CAF0004BA95CA90E94AAE4DC01CB018C159D0521
:10CB0000AE05BF0508F095C0A8A5B9A58D929D9268
:10CB1000AD92BC9213978DC0AF8DB8A10D911D91B0
:10CB20002D913C910FAB18AF29AF3AAF9701860119
:10CB3000330F000B102F98010BA31CA32DA33EA3B2
:10CB4000E8A5F9A580819181A281B3811C012D0105
:10CB50009601A7016BA1762F862F962F51016201B6
:10CB6000EE24FF2400E010E00E94270C24962FAF53
:10CB700024973BA34DAF5EAF6FAF21967FAF219758
:10CB800022968FAF229723969FAF23972FA938AD78
:10CB900049AD5AAD59016A0149A95AA96BA97CA9A5
:10CBA0001A012B019501A60160E070E080E090E0A1
:10CBB00051016201EE24FF2400E010E00E94270CE6
:10CBC0002396AFAD23979A1748F1A91791F52296AE
:10CBD000BFAD22978B1710F1B81759F52196EFAD1D
:10CBE00021977E17D8F0E71721F5FFAD6F17B0F04A
:10CBF000F617F9F4EEAC5E1588F0E516D1F4FDAC4D
:10CC00004F1560F0F416A9F40BA1301738F0031794
:10CC100081F424961FAD2497211758F42FA938AD1D
:10CC200049AD5AADA8A5B9A52D933D934D935C93FD
:10CC30001397BDA5BF5FBDA7EF8DF8A13496F8A3EC
:10CC4000EF8F0DA91EA90C5F1F4F1EAB0DABB530AA
:10CC500009F013CFED89FE89E259FF4F8081918160
:10CC6000A281B381803010E8910710E0A10710E0A5
:10CC7000B10738F4772766272F89388D498D5A8D6B
:10CC80001CC0803020E0920722E0A20720E0B2071B
:10CC9000E8F4F2E0B595A79597958795FA95D1F7C1
:10CCA000772766272F89388D498D5A8D02E0559553
:10CCB0004795379527950A95D1F70E94BDE0DC018D
:10CCC000CB01ED89FE89E85AFF4F3AC00D891E89D4
:10CCD000085A1F4F803030E0930738E0A30730E058
:10CCE000B307A8F4F4E0B595A79597958795FA95BD
:10CCF000D1F7772766272F89388D498D5A8DE4E043
:10CD00005595479537952795EA95D1F714C025E0B5
:10CD1000B595A795979587952A95D1F77727662793
:10CD20002F89388D498D5A8DE5E055954795379572
:10CD30002795EA95D1F70E94BDE0DC01CB01F8010F
:10CD400080839183A283B383ED89FE89E259FF4FEB
:10CD500080809180A280B3809401A50160E070E0A2
:10CD600080E090E01FEDA12E08E1B02E12E0C12E70
:10CD7000DD24EE24FF2400E010E00E94270C0EE0EA
:10CD80000E94FA0CAD89BE89D4962C93D497D5967F
:10CD90003C93D597D6964C93D697D7965C93D797D6
:10CDA000FD01E85BFF4FEB8CFC8CE114F104D9F43E
:10CDB0006091F6137091F7138091F8139091F91325
:10CDC0006093A3137093A4138093A5139093A61359
:10CDD00020813181428153810E94BDE06F8B788F29
:10CDE000898F9A8FCBC080819181A281B38140913C
:10CDF0000E1450910F146091101470911114481773
:10CE000059076A077B078CF08093A3139093A413B0
:10CE1000A093A513B093A61300E010E021E030E04A
:10CE20000F8B188F298F3A8FA9C08E010F5F1F4F6C
:10CE30001C8F0B8FB2E36B2EB4E17B2E8AEFE82EB2
:10CE400083E1F82E2301180195E0C92E00E010E0DF
:10CE500021E030E00F8B188F298F3A8FAC2C4701DF
:10CE6000D101CD90DD90ED90FD901D01F201419139
:10CE70005191619171912F01D4010D911D912D91CD
:10CE80003D914D01D701C601841B950BA60BB70B35
:10CE9000B7FF07C0B095A095909581959F4FAF4F74
:10CEA000BF4F081719072A073B076CF5C114D104B7
:10CEB000E104F10461F14C155D056E057F052CF46C
:10CEC000400F511F621F731F04C0401B510B620BA8
:10CED000730BCB01BA01A70196010E94BDE0DC01F2
:10CEE000CB01181619061A061B068CF4EF88F88C6D
:10CEF000098D1A8D8E159F05A007B10724F48F8B1D
:10CF0000988FA98FBA8FAA9409F0AACF04C01F8A5C
:10CF1000188E198E1A8EED89FE89E85BFF4F6081AD
:10CF20007181828193812F89388D498D5A8D0E941C
:10CF30003FE0DC01CB018093A3139093A413A09353
:10CF4000A513B093A61300E0AB8DBC8D6D917D91C0
:10CF50008D919D91BC8FAB8F2F89388D498D5A8DC6
:10CF60000E943FE0DC01CB01F30181939193A193F7
:10CF7000B1933F010F5F053039F73CC089819A8139
:10CF8000AB81BC818093321490933314A0933414FA
:10CF9000B09335148D819E81AF81B885809336140E
:10CFA00090933714A0933814B093391489859A85D7
:10CFB000AB85BC8580933A1490933B14A0933C14AA
:10CFC000B0933D148D859E85AF85B88980933E14BE
:10CFD00090933F14A0934014B093411489899A8987
:10CFE000AB89BC898093421490934314A09344145A
:10CFF000B09345140091F6131091F7132091F81394
:10D000003091F9136CE035952795179507956A953A
:10D01000D1F7ED89FE89E85AFF4FC080D180E280C8
:10D02000F38076E0F594E794D794C7947A95D1F796
:10D03000ED89FE89EC5AFF4F80809180A280B380F9
:10D04000A5E0B594A79497948794AA95D1F7C901C0
:10D05000B801A90198010E943FE02B013C01C501E4
:10D06000B401A70196010E943FE0DC01CB01840DD1
:10D07000951DA61DB71D00E00097A105B10509F497
:10D080004BC0AC01BD01407050706070707E4115A6
:10D0900051056105710549F452E0880F991FAA1FD7
:10D0A000BB1F5A95D1F70F5FE7CF181619061A065E
:10D0B0001B0694F5CD01BB2797FDB095AB2F07302C
:10D0C000A8F00E941E57AC01662757FD6095762F89
:10D0D000BA015527442710E00650104004C075954A
:10D0E0006795579547950A95D2F71AC00E941E5723
:10D0F000AC01662757FD6095762FBA015527442766
:10D1000086E090E0801B910904C0440F551F661F04
:10D11000771F8A95D2F704C040E050E060E070E0ED
:10D1200040932E1450932F14609330147093311445
:10D130000091A3131091A4132091A5133091A6136D
:10D140008091F6139091F713A091F813B091F91311
:10D15000ED89FE89E45BFF4FCD88DE880F2EF0E578
:10D16000EF2EFF24F02DCE0CDF1C081719072A071D
:10D170003B0754F480839183A283B383F6018083B9
:10D180009183A283B38317C0B42FA52F962F872F27
:10D19000041715072607370724F4B02FA12F922F65
:10D1A000832FB083A18392838383D6010D931D9334
:10D1B0002D933C931397ED89FE89E85BFF4F8081A7
:10D1C0009181A281B381ED89FE89E35AFF4F48170F
:10D1D00059076A077B071CF081E0808301C0108239
:10D1E000ED89FE89E45AFF4F81E08083ED89FE8955
:10D1F000ED58FF4F1082ED89FE89E05CFF4F1082F1
:10D20000118212821382ED89FE8984859585A68517
:10D21000B7850097A105B10541F480899189A2895C
:10D22000B3890097A105B105D9F0FFA1FF23C1F48F
:10D230008091DC139091DD13A091DE13B091DF1388
:10D240000097A105B10521F58091D8139091D913CC
:10D25000A091DA13B091DB130097A105B105C1F4D9
:10D26000AD89BE89DB961C92DB97DD961C921E92DF
:10D27000DC97DF961C921E92DE97FD01EC5BFF4F60
:10D2800011821082FD01EA5BFF4F1182108204C0FF
:10D2900081E0ED89FE8983AF8D899E894F89588D04
:10D2A000698D7A8D8A019B010E943257FCA5F0930B
:10D2B000F10B2FB7F8948091631390916413A091B0
:10D2C0006513B09166138093771390937813A093AE
:10D2D0007913B0937A138091671390916813A0919A
:10D2E0006913B0916A1380937B1390937C13A0937E
:10D2F0007D13B0937E1380916B1390916C13A0916A
:10D300006D13B0916E1380937F1390938013A0934D
:10D310008113B093821380916F1390917013A09139
:10D320007113B09172138093831390938413A0931D
:10D330008513B09386138091731390917413A09109
:10D340007513B09176138093871390938813A093ED
:10D350008913B0938A132FBF0E94275FCD5BDF4FE5
:10D360000FB6F894DEBF0FBECDBFDF91CF911F91F6
:10D370000F91FF90EF90DF90CF90BF90AF909F9074
:10D380008F907F906F905F904F903F902F90089577
:10D39000FF920F931F93CF93DF93F801FFB6F8949A
:10D3A000EC0188819981AA81BB8180937713909346
:10D3B0007813A0937913B0937A13EB018881998144
:10D3C000AA81BB8180937B1390937C13A0937D13E0
:10D3D000B0937E13EA0188819981AA81BB818093F1
:10D3E0007F1390938013A0938113B0938213E9016C
:10D3F00088819981AA81BB81809383139093841340
:10D40000A0938513B093861380819181A281B3810B
:10D410008093871390938813A0938913B0938A13F2
:10D420008091F10B9091F00B891B8F7061F487E76D
:10D4300093E16BE773E14FE753E123E833E107E85A
:10D4400013E10E94EE55FFBEDF91CF911F910F9126
:10D45000FF9008952F923F924F925F926F927F922A
:10D460008F929F92AF92BF92CF92DF92EF92FF92F4
:10D470000F931F93CF93DF9300D000D0CDB7DEB7CB
:10D480008C017A8369835C834B832091F00B40E0AD
:10D4900050E068EE73E04424552432018824992436
:10D4A0005401CC24DD24760137E7232E312C36C0FD
:10D4B000822F90E0829DF001839DF00D929DF00DF2
:10D4C0001124EE50F44FFE83ED83E45BFF4F808127
:10D4D0009181A281B38184179507A607B70714F439
:10D4E000AC01BD01ED81FE81E85BFF4F8081918140
:10D4F000A281B38188169906AA06BB0614F44C01D2
:10D500005D01480E591E6A1E7B1E2F5F203109F4F3
:10D5100020E00894C11CD11CE11CF11C8091F10B8E
:10D52000281731F6C114D104E104F104A9F1CB01AB
:10D53000BA010E94BCE220E030E040E857E30E94DC
:10D54000FEE3DC01CB01F80180839183A283B383E6
:10D55000C501B4010E94BCE220E030E040E857E39E
:10D560000E94FEE3DC01CB01EB81FC81808391838F
:10D57000A283B383A60133272227C301B2010E94ED
:10D58000BDE00E94BCE220E030E040E857E30E94AA
:10D59000FEE3DC01CB010FC080E090E0A0E0B0E052
:10D5A000F80180839183A283B383EB81FC81808324
:10D5B0009183A283B383E981FA8180839183A283DB
:10D5C000B38326960FB6F894DEBF0FBECDBFDF91B2
:10D5D000CF911F910F91FF90EF90DF90CF90BF9070
:10D5E000AF909F908F907F906F905F904F903F9003
:10D5F0002F9008952F923F924F925F926F927F9259
:10D600008F929F92AF92BF92CF92DF92EF92FF9252
:10D610000F931F93CF93DF93CDB7DEB72A970FB643
:10D62000F894DEBF0FBECDBF782E882369F082E06C
:10D6300090E060E00E94DA99082F83E090E060E0DB
:10D640000E94DA99A82E02C0AA2400E095E6E92EED
:10D6500094E1F92E23E5C22E23E0D22E39E1432EA8
:10D66000512C4C0C5D1CC60142969C838B8340E27E
:10D67000242E312C2C0C3D1C1A821982ABE8B0E010
:10D68000BE83AD8388249924E02FF0E0F887EF83F0
:10D69000662463948A2D90E09A878987B82C772036
:10D6A00009F46CC1A7FE0AC089859A85082C02C0BE
:10D6B000959587950A94E2F7817001C081E0D701C2
:10D6C0008C938F819885082C02C0959587950A9434
:10D6D000E2F78170907011968C938D819E8100ECA1
:10D6E0001DE621ED37E94DE650E060E070E00E9474
:10D6F000E3990E94B6E229EF32E045E150E50E944D
:10D70000E3E1DC01CB01F70182839383A483B5833A
:10D7100089819A81895D9E4F40EC53E060E070E022
:10D720000E943C9A0E94BAE220E030E040E752E4D6
:10D730000E94E3E120E030E040E857E40E94FEE38D
:10D740000E9485E2DC01CB01F70186839783A087E5
:10D75000B18789819A8184549E4F48EE53E060E0FE
:10D7600070E00E943C9A462F572FBC01F2E0BF1692
:10D7700019F1BF1618F084E08B1558F5CB01BA01EA
:10D7800022E030E040E050E00E941EE589019A016D
:10D79000D70150960D931D932D933C935397882753
:10D7A0009927DC01801B910BA20BB30BF701848737
:10D7B0009587A687B78720C0D70150964D935D9374
:10D7C0006D937C935397F7011486158616861786FA
:10D7D00013C0D70150964D935D936D937C935397EF
:10D7E00070956095509541955F4F6F4F7F4FF70152
:10D7F0004487558766877787D6011C96ED91FC9103
:10D800001D97208181E090E01B960C901B9702C031
:10D81000880F991F0A94E2F7282B20831596ED9123
:10D82000FC911697208181E090E014960C9014975B
:10D8300002C0880F991F0A94E2F7282B20831E96B6
:10D84000ED91FC911F97208181E090E0AB81BC813C
:10D850000C9002C0880F991F0A94E2F7282B2083AE
:10D86000D6015396ED91FC915497208181E090E090
:10D87000AB81BC810C9002C0880F991F0A94E2F71B
:10D88000282B2083F601848D958D009791F101A0BE
:10D89000F2A1E02D208181E090E0D1010C9002C046
:10D8A000880F991F0A94E2F7809582238083F701FD
:10D8B0008081D6015C96ED91FC915D972081882353
:10D8C00061F081E090E0D1010C9002C0880F991FB7
:10D8D0000A94E2F7282B20830CC081E090E0D1016C
:10D8E0000C9002C0880F991F0A94E2F7809582235A
:10D8F0008083F60185899689009791F1028CF38DDA
:10D90000E02D208181E090E0D2010C9002C0880FD0
:10D91000991F0A94E2F7809582238083F701808122
:10D92000D6015596ED91FC9156972081882361F0A0
:10D9300081E090E0D2010C9002C0880F991F0A94F8
:10D94000E2F7282B20830CC081E090E0D2010C90FC
:10D9500002C0880F991F0A94E2F780958223808382
:10D96000F401EE0FFF1FEE0FFF1FEF5AFB4E108268
:10D97000118212821382F70112861386F401E45B8E
:10D98000FB4E108281E0F2E0FB1508F080E0D70149
:10D9900059968C935997F701158E168E178E10A2F3
:10D9A000628E138E148A55961D921D921D921C92A2
:10D9B000589711A212A213A214A295961D921D921D
:10D9C0001D921C9298970894811C911CE9E2F0E04A
:10D9D000EE0EFF1E83E290E0C80ED91E480E591EBF
:10D9E000AB81BC819396BC83AB83280E391EED813D
:10D9F000FE813896FE83ED8389819A8104969A830D
:10DA0000898395E08916910409F048CE772021F0AA
:10DA10001092471410924614109249141092481410
:10DA200010924B1410924A142A960FB6F894DEBF47
:10DA30000FBECDBFDF91CF911F910F91FF90EF905F
:10DA4000DF90CF90BF90AF909F908F907F906F901E
:10DA50005F904F903F902F90089590E029E230E042
:10DA6000829FF001839FF00D929FF00D1124EB59DE
:10DA7000FB4EDF011296528111964C91119712962E
:10DA80003C91129713962C91852F942FA32FB22F90
:10DA9000BC01CD0108950F931F93CF93DF930F9295
:10DAA000CDB7DEB749830E94BCE28B019C0149815E
:10DAB00050E089E290E0489FF001499FF00D589FA7
:10DAC000F00D1124EB59FB4EC901B80122813381BD
:10DAD000448155810E94E3E1462F572F682F792F0B
:10DAE000CB01BA010F90DF91CF911F910F91089553
:10DAF0004F925F926F927F928F929F92AF92BF925E
:10DB0000CF92DF92EF92FF920F931F93CF93DF9309
:10DB1000142F20E030E04AE754E40E94FEE30E9424
:10DB20004BE2E901942E852E762E672E582E492E33
:10DB3000212F30E089E290E0289FF001299FF00D2D
:10DB4000389FF00D1124EB59FB4E62817381848163
:10DB500095810E944BE259016A017B018C019E0173
:10DB6000492D582D672D762D852D942D0E94270C3B
:10DB7000A8EEAA2EB3E0BB2ECC24DD24EE24FF2495
:10DB800000E010E00E94680D952FB901842FDF910D
:10DB9000CF911F910F91FF90EF90DF90CF90BF90AA
:10DBA000AF909F908F907F906F905F904F9008956F
:10DBB00080917615882319F480917515089581E078
:10DBC00008958091751508954F925F926F927F929C
:10DBD0008F929F92AF92BF92CF92DF92EF92FF927D
:10DBE0001F93CF93DF931FB7F894C0E0D0E089E490
:10DBF00095E1BE010E94B83EFC01108211821282A2
:10DC0000138285E395E1BE010E94B83EFC011082BB
:10DC10001182128213822196C530D10541F71FBFB0
:10DC20008EEA91E061E00E94DA99823009F00CC13D
:10DC300080E00E942D6D0E9485E24B015C0132E084
:10DC4000880C991CAA1CBB1C3A95D1F780EB91E07B
:10DC500040E050E060E070E00E943C9A6B017C0183
:10DC600084EB91E040E050E060E070E00E943C9A7C
:10DC70002B013C018AEE91E061E00E94DA99882351
:10DC800009F097C0C601D7FE03C0909581959F4FBC
:10DC9000AA2797FDA095BA2F88169906AA06BB0653
:10DCA0001CF580E00E942D6D20E030E044E052E45D
:10DCB0000E94FEE320E030E040E05FE30E9468E184
:10DCC0000E9485E2DC01CB019C01AD012C193D09CC
:10DCD0004E095F0969017A017094609450944094F0
:10DCE000411C511C611C711C1FB7F89489E495E11B
:10DCF00060E070E00E94B83EEC0122E0822E912CA0
:10DD0000A12CB12CC701B601A50194010E941EE50A
:10DD1000288339834A835B8385E395E160E070E083
:10DD20000E94B83EEC0189E495E160E070E00E9459
:10DD3000B83EFC0180819181A281B381B095A0950C
:10DD4000909581959F4FAF4FBF4F88839983AA834A
:10DD5000BB8389E495E161E070E00E94B83EEC018C
:10DD6000C301B201A50194010E941EE528833983F5
:10DD70004A835B8385E395E161E070E00E94B83EF1
:10DD8000EC0189E495E161E070E00E94B83EFC019D
:10DD900080819181A281B381B095A0959095819564
:10DDA0009F4FAF4FBF4F88839983AA83BB831FBF09
:10DDB0004BC0C601D7FE03C0909581959F4FAA27FF
:10DDC00097FDA095BA2F88169906AA06BB061CF1E6
:10DDD00080E00E942D6D20E030E044E052E40E949B
:10DDE000FEE320E030E040E05FE30E9468E10E9453
:10DDF00085E2DC01CB019C01AD012C193D094E09E6
:10DE00005F0969017A017094609450944094411CB8
:10DE1000511C611C711CCFB7F89485E395E160E05B
:10DE200070E00E94B83EFC01C082D182E282F3829F
:10DE300085E395E161E070E00E94B83EFC0140821C
:10DE4000518262827382CFBFDF91CF911F91FF9089
:10DE5000EF90DF90CF90BF90AF909F908F907F908A
:10DE60006F905F904F90089589E890E00E94DE994E
:10DE700091E0863008F090E0892F08951092761591
:10DE80001092751581E00E94FA6A80EB91E04FEFE5
:10DE90005FEF6FEF7FEF0E943C9ADC01CB018F3F79
:10DEA0002FEF92072FEFA2072FEFB20711F40E9476
:10DEB000E03208956F927F928F929F92AF92BF92BD
:10DEC000CF92DF92EF92FF920F931F93CF93DF9346
:10DED000CDB7DEB764970FB6F894DEBF0FBECDBFE7
:10DEE000662EDE011196FC0184E101900D928150B5
:10DEF000E1F740E7E42E44E1F42E00E010E077245F
:10DF00007394F7017082662001F5CE010196B80185
:10DF10000E94B83E6C01FC0180809180A280B38099
:10DF20008091331590913415B8010E94B83EFC01E0
:10DF300080819181A281B381880D991DAA1DBB1D8D
:10DF4000F60180839183A283B3830F5F1F4F89E221
:10DF500090E0E80EF91E0530110599F6CE01019604
:10DF600060E070E00E94B83E7C01CE01019661E065
:10DF700070E00E94B83E4C01CE01019662E070E074
:10DF80000E94B83E6C01CE01019663E070E00E94F1
:10DF9000B83E5C01CE01019664E070E00E94B83E9C
:10DFA0008C01C701B401A60195010E94C86964965D
:10DFB0000FB6F894DEBF0FBECDBFDF91CF911F919A
:10DFC0000F91FF90EF90DF90CF90BF90AF909F9018
:10DFD0008F907F906F9008955F926F927F928F9253
:10DFE0009F92AF92BF92CF92DF92EF92FF920F93E8
:10DFF0001F93CF93DF93CDB7DEB764970FB6F89436
:10E00000DEBF0FBECDBF782E692E0E947B3E5FB66D
:10E01000F89400D00F92409177135091781360914B
:10E02000791370917A1300917B1310917C132091D6
:10E030007D1330917E13C0907F13D0908013E090B9
:10E040008113F09082138090831390908413A0909A
:10E050008513B09086138091871390918813A091B7
:10E060008913B0918A13EDB7FEB781839283A3839E
:10E07000B483CE0101960E947C3EE72DF62DDE0191
:10E08000119684E10D9001928150E1F70F900F906D
:10E090000F900F9000E010E0872D962DB8010E94A0
:10E0A000B83E4C01FC01C080D180E280F3808091B9
:10E0B000331590913415B8010E94B83EFC0180815F
:10E0C0009181A281B381C81AD90AEA0AFB0AF40134
:10E0D000C082D182E282F3820F5F1F4F05301105AB
:10E0E000D9F65FBE872D962D64960FB6F894DEBFE5
:10E0F0000FBECDBFDF91CF911F910F91FF90EF9099
:10E10000DF90CF90BF90AF909F908F907F906F9057
:10E110005F9008954F925F926F927F928F929F923D
:10E12000AF92BF92CF92DF92EF92FF920F931F9325
:10E13000CF93DF93CDB7DEB765970FB6F894DEBF08
:10E140000FBECDBF2C013B01CE010296BE016A5F1E
:10E150007F4FAE01465F5F4F9E01225F3F4F8E01B2
:10E160000E5E1F4F7E010894E11CF11C0E94435675
:10E17000898181708983813029F475E3E72E75E107
:10E18000F72E04C069E4E62E65E1F62E52E0C52EB6
:10E19000D12CCC0EDD1E00E010E0F60180809180D5
:10E1A000A280B380C701B8010E94B83EFC01808103
:10E1B0009181A281B381A5019401281B390B4A0BDF
:10E1C0005B0BF60121933193419351936F010F5FE4
:10E1D0001F4F0530110509F700D00F924A815B816E
:10E1E0006C817D810E811F8128853985CA84DB84FD
:10E1F000EC84FD848E849F84A888B9888A899B8951
:10E20000AC89BD89EDB7FEB781839283A383B483C4
:10E21000C2010E947C3E0F900F900F900F906114EE
:10E22000710419F08981F3018083C20165960FB6EC
:10E23000F894DEBF0FBECDBFDF91CF911F910F913C
:10E24000FF90EF90DF90CF90BF90AF909F908F9016
:10E250007F906F905F904F90089580935D15089523
:10E260002F923F924F925F926F927F928F929F92E6
:10E27000AF92BF92CF92DF92EF92FF920F931F93D4
:10E28000CF93DF9300D00F92CDB7DEB71C012A01E8
:10E290003B01A3E68A2EA3E19A2E540100E010E090
:10E2A000C101B8010E94B03EFC01C080D180E28073
:10E2B000F3808091331590913415B8010E94B83ED7
:10E2C000FC0180819181A281B3818C0D9D1DAE1DC9
:10E2D000BF1DF50181939193A193B1935F010F5FEE
:10E2E0001F4F05301105E1F6E7E72E2EE3E13E2E44
:10E2F000F7EAEF2EF3E1FF2ECC24AA2480E090E091
:10E30000A0E0B0E0F40101911191219131914F0110
:10E31000F10141915191619171911F01041B150B04
:10E32000260B370B37FF07C03095209510950195C8
:10E330001F4F2F4F3F4FF7010193119321933193BB
:10E340007F0180179107A207B3071CF4AC2CD901F9
:10E35000C801C394F5E0CF16A9F6A092BB13809331
:10E36000BC139093BD13A093BE13B093BF1300973B
:10E37000A105B10551F160E472E48FE090E0A301E2
:10E3800092010E941EE529833A834B835C8360E0FF
:10E3900070E080E090E0AE014F5F5F4F22E335E137
:10E3A00000E0E09032150E947C5F8091F10B90912B
:10E3B000F00B891B8F7090917415891720F081E004
:10E3C0008093761502C0109276150F900F900F90E3
:10E3D0000F90DF91CF911F910F91FF90EF90DF9001
:10E3E000CF90BF90AF909F908F907F906F905F90F5
:10E3F0004F903F902F9008952F923F924F925F92AF
:10E400006F927F928F929F92AF92BF92CF92DF9244
:10E41000EF92FF920F931F93CF93DF93CDB7DEB7A9
:10E420002A970FB6F894DEBF0FBECDBF9E838D83B3
:10E430004F83588769877A8713E6412E13E1512E5F
:10E4400007E7602E03E1702E6301720100E010E027
:10E45000222E33248D819E81B8010E94B03EDC01C2
:10E460008D909D90AD90BC90809133159091341516
:10E47000B8010E94B83EFC014081518162817381E4
:10E48000480D591D6A1D7B1DD7014D935D936D93FA
:10E490007C931397C101002E02C0959587950A942D
:10E4A000E2F780FF0EC0F60180819181A281B381E5
:10E4B000840F951FA61FB71FF70180839183A28346
:10E4C000B3830F5F1F4F84E090E0E80EF91EC80E83
:10E4D000D91E0530110509F0BDCFB7EA8B2EB3E187
:10E4E0009B2EEE24CC2400E010E020E030E0D201AE
:10E4F0004D915D916D917D912D01F30181919191EE
:10E50000A191B1913F01481B590B6A0B7B0B77FF1F
:10E5100007C070956095509541955F4F6F4F7F4F45
:10E52000D4014D935D936D937D934D0104171507B1
:10E53000260737071CF4CE2C8A019B01E394B5E033
:10E54000EB16A9F6C092BB130093BC131093BD1336
:10E550002093BE133093BF1301151105210531051A
:10E5600081F16F81788589859A85A90198010E943A
:10E570001EE560E472E48FE090E00E941EE52983CE
:10E580003A834B835C8360E070E080E090E0AE0112
:10E590004F5F5F4F22E335E100E0E09032150E94CB
:10E5A0007C5F8091F10B9091F00B891B8F709091A3
:10E5B0007415891720F081E08093761502C01092BF
:10E5C00076152A960FB6F894DEBF0FBECDBFDF9149
:10E5D000CF911F910F91FF90EF90DF90CF90BF9060
:10E5E000AF909F908F907F906F905F904F903F90F3
:10E5F0002F9008952F923F924F925F926F927F9249
:10E600008F929F92AF92BF92CF92DF92EF92FF9242
:10E610000F931F93CF93DF93CDB7DEB766970FB6F7
:10E62000F894DEBF0FBECDBF1C01498B5A8B6B8B9C
:10E630007C8BED86FE860F87188BDE8ACD8A43E6BB
:10E6400053E15A87498767E773E17C876B877B01D2
:10E650008A01CC24DD24422E5524C101B6010E943A
:10E66000B03EFC0180809180A280B3808091331500
:10E6700090913415B6010E94B83EFC014081518151
:10E6800062817381480D591D6A1D7B1DF80140830D
:10E69000518362837383C2010C2C02C095958795C8
:10E6A0000A94E2F780FF0EC0F70180819181A28178
:10E6B000B381840F951FA61FB71FF8018083918334
:10E6C000A283B3830894C11CD11C0C5F1F4F44E08C
:10E6D00050E0E40EF51E55E0C516D10409F0BDCF9B
:10E6E0001092BB13F7EA2F2EF3E13F2E60E675E19F
:10E6F0007E836D8384EC93E198878F8300E0882488
:10E7000099245401E985FA85419151916191719162
:10E71000FA87E987EB85FC8581919191A191B1916F
:10E72000FC87EB87481B590B6A0B7B0BF10140837D
:10E730005183628373836A017B0177FF07C0CC2416
:10E74000DD247601C41AD50AE60AF70AF0E0CF16EE
:10E75000F0E8DF06F0E0EF06F0E0FF0664F4CA013F
:10E7600077276627ED81FE812081318142815381A7
:10E770000E943FE022C0CB01BA010E94BCE22B0103
:10E780003C01ED81FE8160817181828193810E94D3
:10E79000BCE220E030E040E857E30E94FEE39B014A
:10E7A000AC01C301B2010E94FEE320E030E040E88A
:10E7B00057E40E94FEE30E9485E2DC01CB01EF8179
:10E7C000F88580839183A283B383F101C082D182D3
:10E7D000E282F3828C149D04AE04BF0424F40093FF
:10E7E000BB134601570144E050E0240E351E0F5F75
:10E7F0006D817E816C5F7F4F7E836D838F81988575
:10E80000049698878F83053009F07CCF8092BC13E3
:10E810009092BD13A092BE13B092BF1381149104C5
:10E82000A104B10409F463C06D857E858F85988944
:10E8300020E030E040E050E00E94DFE1882309F46E
:10E8400056C06D857E858F85988920E030E040E850
:10E8500057E40E94FEE30E9485E2DC01CB01809335
:10E86000C0139093C113A093C213B093C31320910C
:10E870000204222379F0ED89FE89CF01AA2797FDB2
:10E88000A095BA2F3AE0880F991FAA1FBB1F3A958F
:10E89000D1F704C080E090E0A0E0B0E049895A8957
:10E8A0006B897C8949835A836B837C83222319F08B
:10E8B0000091030401C000E0BC01CD01AE014F5F37
:10E8C0005F4F22E335E1E09032150E947C5F80913A
:10E8D000F10B9091F00B891B8F7090917415891733
:10E8E00020F081E08093761502C01092761566962E
:10E8F0000FB6F894DEBF0FBECDBFDF91CF911F9151
:10E900000F91FF90EF90DF90CF90BF90AF909F90CE
:10E910008F907F906F905F904F903F902F900895D1
:10E920002F923F924F925F926F927F928F929F921F
:10E93000AF92BF92CF92DF92EF92FF920F931F930D
:10E94000CF93DF93CDB7DEB764970FB6F894DEBFF1
:10E950000FBECDBF882E162F29013A011092030455
:10E960006E010894C11CD11CC60160E070E00E94D9
:10E970008A70BFE6AB2EB4E1BB2EEE24FF24212E1D
:10E9800033249C2C0D2D11E0C1010E2C02C0959555
:10E9900087950A94E2F7ACE4CA2EA4E1DA2ECE0CF5
:10E9A000DF1C80FD03C0F601108219C0892D902F55
:10E9B000B7010E94B83EFC01882029F08FEF9FEF3D
:10E9C000AFEFBFE304C080E090E0A0E0B0EC808354
:10E9D0009183A283B383F6011083F5011083089419
:10E9E000E11CF11C89E290E0A80EB91E95E0E91641
:10E9F000F10451F6CE010196B301A2010E943071DB
:10EA000081E08093751564960FB6F894DEBF0FBE53
:10EA1000CDBFDF91CF911F910F91FF90EF90DF90CD
:10EA2000CF90BF90AF909F908F907F906F905F90AE
:10EA30004F903F902F900895853098F4909147140F
:10EA400021E030E002C0220F331F8A95E2F76623EF
:10EA500021F0922B90934714089520952923209319
:10EA600047140895809303040895817080933215AC
:10EA7000813019F485E395E102C089E495E1909332
:10EA800034158093331508958091B5039091B603A2
:10EA90000097A1F0E091B703F091B803808190E076
:10EAA0000090B90302C0959587950A94E2F78170AA
:10EAB000907091E02091B714281709F490E0292F65
:10EAC0002295220F207E8091AE039091AF03009794
:10EAD000A1F0E091B003F091B103808190E000904B
:10EAE000B20302C0959587950A94E2F78170907001
:10EAF00031E09091B714981709F430E03295307FE7
:10EB0000322B80919203909193030097A1F0E091B2
:10EB10009403F0919503808190E00090960302C0E9
:10EB2000959587950A94E2F78170907021E0909115
:10EB30008E14981709F420E0220F220F220F232BA6
:10EB400080918B0390918C030097A1F0E0918D034D
:10EB5000F0918E03808190E000908F0302C0959524
:10EB600087950A94E2F78170907041E090918E143D
:10EB7000981709F440E0440F440F422B80916F0333
:10EB8000909170030097A1F0E0917103F0917203EE
:10EB9000208130E00090730302C0359527950A94D8
:10EBA000E2F72170307081E090916514921709F4BA
:10EBB00080E0880F842B2091680330916903211530
:10EBC0003105A1F0E0916A03F0916B03208130E000
:10EBD00000906C0302C0359527950A94E2F72170E6
:10EBE000307091E030916514321709F490E0892B70
:10EBF000089590910204992309F480E00E94165729
:10EC000008950E949E56109276151092751580E018
:10EC10000E94FA6A809102048093030481E00E94BA
:10EC2000F97508952F923F924F925F926F927F9263
:10EC30008F929F92AF92BF92CF92DF92EF92FF920C
:10EC40000F931F93CF93DF930E94346F882311F4A7
:10EC50000E94403380E00E94FA6A0E94E46D80E0E6
:10EC60000E94357586E291E061E00E94DA99817038
:10EC7000809302048093030481E00E94F97500E60A
:10EC800015E1C0E08C2F0E942D6D9B01AC0160E06E
:10EC900070E080E89FE30E94E3E120E030E040E89C
:10ECA00057E40E94FEE30E9485E2DC01CB01F801FB
:10ECB00081939193A193B1938F01CF5FC53011F7E9
:10ECC0008BE391E044EF51E060E070E00E943C9AF9
:10ECD000DC01CB0180931A1490931B14A0931C1495
:10ECE000B0931D148FE391E044EF51E060E070E0D9
:10ECF0000E943C9ADC01CB0180931E1490931F1458
:10ED0000A0932014B093211483E491E046E950E0ED
:10ED100060E070E00E943C9ADC01CB0180932214F9
:10ED200090932314A0932414B093251487E491E0C6
:10ED300040E157E260E070E00E943C9ADC01CB01C8
:10ED40008093261490932714A0932814B093291429
:10ED500086EA91E040E157E260E070E00E943C9A70
:10ED6000DC01CB0180932A1490932B14A0932C14D4
:10ED7000B0932D140AE114E1C0EE6C2EC3E17C2E99
:10ED8000DFE84D2ED3E15D2EC0E088248A94982CD4
:10ED900054011801F801C080D180E280F3808C2FEB
:10EDA0000E942D6D9B01AC0160EF7FEF8FE799E42E
:10EDB0000E94E3E10E948AE2DC01CB018C159D05F3
:10EDC000AE05BF05A0F48C2F0E942D6D9B01AC01F8
:10EDD00060EF7FEF8FE799E40E94E3E10E948AE20F
:10EDE000DC01CB01F80180839183A283B3830C5FA4
:10EDF0001F4FF10160817181828193810E94BAE28B
:10EE00006B017C018C2F0E942D6D9B01AC01C70111
:10EE1000B6010E94FEE30E948AE29B01AC01F3016D
:10EE200061937193819391933F01C501B4010E9455
:10EE3000FCE4F20121933193419351932F01CF5F71
:10EE4000C53009F0A6CF8BE491E040ED57E060E0DB
:10EE500070E00E943C9ADC01CB01809316149093E1
:10EE60001714A0931814B09319148131F7E29F0777
:10EE7000F0E0AF07F0E0BF0760F080E197E2A0E0CC
:10EE8000B0E08093161490931714A0931814B093C5
:10EE900019148FE491E040EA5FE060E070E00E94C6
:10EEA0003C9ADC01CB018093121490931314A0932D
:10EEB0001414B0931514813127E2920720E0A207C1
:10EEC00020E0B20760F080E197E2A0E0B0E080933C
:10EED000121490931314A0931414B093151485E88E
:10EEE00091E048E050E060E070E00E943C9ADC0174
:10EEF000CB019093CA0B8093C90B8AEA91E048E05A
:10EF000050E060E070E00E943C9ADC01CB019093FD
:10EF1000CC0B8093CB0B82E991E04CE251E060E0B6
:10EF200070E00E943C9A0E94BAE220E030E040E2A9
:10EF300051E40E94E3E120E030E040E857E40E9421
:10EF4000FEE30E9485E2DC01CB018093FA139093EB
:10EF5000FB13A093FC13B093FD1386E991E04CE200
:10EF600051E060E070E00E943C9A0E94BAE220E02A
:10EF700030E040E251E40E94E3E120E030E040E88C
:10EF800057E40E94FEE30E9485E2DC01CB018093FE
:10EF9000FE139093FF13A0930014B09301148AE919
:10EFA00091E044E650E060E070E00E943C9A0E94EC
:10EFB000BAE220E030E040E251E40E94E3E120E0E8
:10EFC00030E040E857E40E94FEE30E9485E2DC0165
:10EFD000CB018093021490930314A0930414B09374
:10EFE00005148EE991E04CE251E060E070E00E948F
:10EFF0003C9A0E94BAE220E030E040E251E40E94F4
:10F00000E3E120E030E040E857E40E94FEE30E94A4
:10F0100085E2DC01CB018093061490930714A09342
:10F020000814B093091482EA91E04CE251E060E0E8
:10F0300070E00E943C9A0E94BAE220E030E040E298
:10F0400051E40E94E3E120E030E040E857E40E9410
:10F05000FEE30E9485E2DC01CB0180930A149093C9
:10F060000B14A0930C14B0930D1480910214909182
:10F070000314A0910414B0910514EAEFF3E120E029
:10F080004191519161917191481759076A077B0726
:10F0900014F4DB01CA012F5F253091F780930E1421
:10F0A00090930F14A0931014B093111487E691E07D
:10F0B0004CEB52E060E070E00E943C9A0E94BAE2A1
:10F0C00020E030E543EC57E40E94E3E120E030E04B
:10F0D00040E857E40E94FEE30E9485E2062FC72F16
:10F0E000D82FC92E8FE591E040E951E060E070E053
:10F0F0000E943C9A0E94BAE220E030E543EC57E4DB
:10F100000E94E3E120E030E040E857E40E94FEE3A3
:10F110000E9485E2162FF72EE82ED92E8EE195E07B
:10F12000A0E0B0E080938B1390938C13A0938D1389
:10F13000B0938E1380E090E0A2E0B0E08093F613ED
:10F140009093F713A093F813B093F91389E891E023
:10F1500061E00E94DA99882339F084E090E090938E
:10F16000F5138093F41304C01092F5131092F41366
:10F1700081E08093C70B8093C80B6091E614709177
:10F18000E7148091E8149091E9140E94BCE220E019
:10F1900030E040E857E30E94FEE3DC01CB018093BE
:10F1A000BF0B9093C00BA093C10BB093C20B6091A7
:10F1B0000F157091101580911115909112150E94E4
:10F1C000BCE220E030E040E857E30E94FEE3DC01CF
:10F1D000CB018093C30B9093C40BA093C50BB0934A
:10F1E000C60B89EE91E060E00E94DA9991E08823F5
:10F1F00009F490E090935E1590935F1583E00E9470
:10F200002D6D20E030E048E452E40E94E3E120E08C
:10F2100030E040E05FE30E9468E10E9485E26530F3
:10F2200071056CF463307105A4F46130710569F007
:10F230006230710564F46115710529F00EC0693002
:10F2400071055CF408C082E009C083E007C084E077
:10F2500005C085E003C086E001C087E080935103CC
:10F260008FE080937415602F7C2F8D2F9C2D212F84
:10F270003F2D4E2D5D2D00915D150E942E5F0E9449
:10F280001B55DF91CF911F910F91FF90EF90DF9071
:10F29000CF90BF90AF909F908F907F906F905F9036
:10F2A0004F903F902F900895CF93DF9300D000D0E0
:10F2B000CDB7DEB78091571B9091581B9D838C83EF
:10F2C0008E81807F8E8380910304882319F0409182
:10F2D000020401C040E0CE01049660E00E94E59582
:10F2E0008091671B9091681B9A8389838B81807FB3
:10F2F0008B838091F10B9091F00B891B8F7041E013
:10F30000833008F440E0CE01019660E00E94E5956C
:10F3100026960FB6F894DEBF0FBECDBFDF91CF911A
:10F3200008950E94CC42882311F0109276158091A6
:10F330007515882351F110927515209175158091DE
:10F340004C1490E030E0822B932B80937515209124
:10F35000751580914D1490E030E0822B932B8093B3
:10F3600075152091751580914E1490E030E0822B38
:10F37000932B8093751580917515882331F40E9425
:10F380009E56809102048093030408950E94E153E5
:10F39000089589E495E10E947B3E85E395E10E9412
:10F3A0007B3E089580E99BE1089586EB9BE10895FB
:10F3B00080919815882351F480919715882321F422
:10F3C00081E080939715089580E0089580E0089586
:10F3D000109297150895FF920F931F93CF93DF9389
:10F3E000CDB7DEB72F970FB6F894DEBF0FBECDBFF7
:10F3F0008091831590918415A0918515B091861503
:10F400000196A11DB11D8093831590938415A0933F
:10F410008515B09386158E010F5F1F4FC8010E949E
:10F42000A1DDC80144EF51E060E070E00E94A5DD7D
:10F43000F02E012F8F2D902F0E94CBDD8823D1F34A
:10F4400081E08093981588E895E140E553EC60E011
:10F4500070E00E94A5DD85E08093040480E99BE1D3
:10F460000E9418DB8CE89BE10E94A2DE2F960FB66B
:10F47000F894DEBF0FBECDBFDF91CF911F910F91EA
:10F48000FF9008959091981581E0892708958091C3
:10F490009815882309F4AAC08091B31B9091B41BDE
:10F4A0008430910519F41092981508958091B21B3B
:10F4B0008823E1F18091B21B8130C1F480917715EE
:10F4C00090917815A0917915B0917A150196A11DAA
:10F4D000B11D8093771590937815A0937915B0930B
:10F4E0007A1580E99BE10E9418DB089520910404BD
:10F4F000222339F580917F1590918015A091811577
:10F50000B09182150196A11DB11D80937F15909336
:10F510008015A0938115B0938215109298158DE6F1
:10F5200098E163E070E00E944891089588E895E1D1
:10F530000E94CBDD882309F459C0209104042223C2
:10F5400079F180917B1590917C15A0917D15B091FA
:10F550007E150196A11DB11D80937B1590937C159E
:10F56000A0937D15B0937E1521502093040488E864
:10F5700095E140E553EC60E070E00E94A5DD86EB8C
:10F580009BE10E9495DB80E99BE10E9418DB8CE8FF
:10F590009BE10E9444DF8CE89BE10E94A2DE08957B
:10F5A00080917F1590918015A0918115B091821561
:10F5B0000196A11DB11D80937F1590938015A09396
:10F5C0008115B093821580E99BE10E940ADB84E0FB
:10F5D0008093B21B8CE89BE10E9444DF1092981547
:10F5E0008DE698E161E070E00E9448910895FF92F5
:10F5F0000F931F93CF93DF93CDB7DEB72F970FB63F
:10F60000F894DEBF0FBECDBF8E010F5F1F4FC80144
:10F610000E94A1DDC80140EA56E861E070E00E9466
:10F62000A5DDF02E012F12C08F2D902F0E94CBDD73
:10F63000882361F081E080939715109298158DE6EC
:10F6400098E162E070E00E94489104C00E94D8797D
:10F65000882351F386EB9BE10E948DDB86EB9BE1D7
:10F660006FE70E94D3DB86EB9BE161E00E94D3DB76
:10F670000E94EB7988E895E140EA56E861E070E0A5
:10F680000E94A5DD1092971502C00E94477A8091D2
:10F6900098158823D1F72091B31B3091B41B81E0DA
:10F6A0002430310509F080E02F960FB6F894DEBFC4
:10F6B0000FBECDBFDF91CF911F910F91FF900895A5
:10F6C000FF920F931F93CF93DF93CDB7DEB72F97A2
:10F6D0000FB6F894DEBF0FBECDBF8E010F5F1F4F78
:10F6E000C8010E94A1DDC80140EA56E861E070E06F
:10F6F0000E94A5DDF02E012F12C08F2D902F0E94A9
:10F70000CBDD882361F081E08093971510929815E6
:10F710008DE698E162E070E00E94489104C00E948A
:10F72000D879882351F386EB9BE10E948DDB86EB31
:10F730009BE160E00E94D3DB86EB9BE168E20E94E4
:10F74000D3DB0E94EB7988E895E140EA56E861E076
:10F7500070E00E94A5DD1092971502C00E94477AC2
:10F76000809198158823D1F72F960FB6F894DEBFB5
:10F770000FBECDBFDF91CF911F910F91FF900895E4
:10F78000FF920F931F93CF93DF93CDB7DEB72F97E1
:10F790000FB6F894DEBF0FBECDBF8E010F5F1F4FB7
:10F7A000C8010E94A1DDC80140EA56E861E070E0AE
:10F7B0000E94A5DDF02E012F12C08F2D902F0E94E8
:10F7C000CBDD882361F081E0809397151092981526
:10F7D0008DE698E162E070E00E94489104C00E94CA
:10F7E000D879882351F386EB9BE10E948DDB86EB71
:10F7F0009BE160E00E94D3DB86EB9BE160E00E942E
:10F80000D3DB86EB9BE160E00E94D3DB86EB9BE1E0
:10F8100060E00E94D3DB0E94EB7988E895E140EA42
:10F8200056E861E070E00E94A5DD1092971502C0D5
:10F830000E94477A809198158823D1F78091B21B56
:10F84000843041F080E99BE160E00E946DDB91E053
:10F85000813009F090E0892F2F960FB6F894DEBF23
:10F860000FBECDBFDF91CF911F910F91FF900895F3
:10F870001F93CF93DF930F92CDB7DEB7109283150E
:10F8800010928415109285151092861510927F158E
:10F8900010928015109281151092821510927B158E
:10F8A00010927C1510927D1510927E15109277158E
:10F8B000109278151092791510927A1510E002C006
:10F8C000882379F00E94C07B1F5F1038C9F709C0F8
:10F8D00089830E94607B89810F90DF91CF911F9176
:10F8E000089581E040917B1550917C1560917D15C4
:10F8F00070917E15411551056105710549F380E050
:10F90000EBCF80938715089580918715089588E837
:10F9100095E10E94A1DD08954F925F926F927F92D0
:10F92000AF92BF92CF92DF92EF92FF920F931F930D
:10F93000CF93DF930F920F92CDB7DEB75C018B01AF
:10F94000009709F449C06230710508F445C0DC0134
:10F9500016964D905D906D907C901997000F111F39
:10F960006801EE24FF24C40CD51CE61CF71CD5014D
:10F97000ED91FC910190F081E02DC701B601AE013F
:10F980004F5F5F4F22E030E01995882329F109810C
:10F990001A8101151105F1F0C801409688309105D2
:10F9A000D8F0BFEF083F1B0710F000E010E01A820C
:10F9B0001982D501ED91FC910480F581E02DC701FC
:10F9C000B601AE014F5F5F4F22E030E0199501159F
:10F9D000110521F681E001C080E00F900F90DF91CA
:10F9E000CF911F910F91FF90EF90DF90CF90BF903C
:10F9F000AF907F906F905F904F9008952F923F92BD
:10FA00004F925F926F927F928F929F92AF92BF922E
:10FA1000CF92DF92EF92FF920F931F93CF93DF93DA
:10FA2000CDB7DEB72C970FB6F894DEBF0FBECDBFB3
:10FA30004C017A876987009709F4ABC0DC01ED912E
:10FA4000FC911197208131813C872B87848195819E
:10FA50009C838B8316968D919D910D90BC91A02DCA
:10FA60008D839E83AF83B887F401A28CB38C82858B
:10FA70009385A485B585B695A795979587951C011F
:10FA8000138E128E3A014424552400E010E0C80180
:10FA900085015C0151C00230110518F002151305F3
:10FAA00010F002E010E06801CC0CDD1CEE24FF2415
:10FAB0002D813E814F815885C20ED31EE41EF51E56
:10FAC000C701B601AE014F5F5F4F22E030E0AB856A
:10FAD000BC85FD011995882309F45BC089819A8151
:10FAE000009729F56114710439F4C50158018C019E
:10FAF000F401B38EA28E28C0A114B10429F42FEF13
:10FB00003FEF3A83298302C0BA82A982C701B601B6
:10FB1000AE014F5F5F4F22E030E0AB81BC81FD0161
:10FB20001995882389F108946108710858010F5FBD
:10FB30001F4F0894411C511C2414350409F0ABCF0D
:10FB400085016114710409F5E985FA85E230F10552
:10FB500010F109831A83BF01660F771F80E090E0E0
:10FB60002D813E814F815885620F731F841F951F21
:10FB7000AE014F5F5F4F22E030E0AB81BC81FD0101
:10FB80001995882311F007C08501C401B8010E94AE
:10FB90008C7C00E010E0C8012C960FB6F894DEBF14
:10FBA0000FBECDBFDF91CF911F910F91FF90EF90CE
:10FBB000DF90CF90BF90AF909F908F907F906F908D
:10FBC0005F904F903F902F90089580E190E00895CE
:10FBD0000F931F93CF93DF93EC010097C1F0623036
:10FBE0007105A8F06250704080E090E02889398962
:10FBF00040E050E00E94AAE48B019C018A899B8925
:10FC0000AC89BD89080F191F2A1F3B1F04C000E0E3
:10FC100010E020E030E0B801C901DF91CF911F91E1
:10FC20000F910895AF92BF92CF92DF92EF92FF9221
:10FC30000F931F93CF93DF93CDB7DEB72D970FB6FA
:10FC4000F894DEBF0FBECDBF8C016A017B01D901E4
:10FC50004D915C91119712968D919C91139780967E
:10FC600013969C938E931297F8018081853E11F034
:10FC7000882329F4D90114961C921497DDC0F80149
:10FC800093859F3009F04AC0D90114968C9114973E
:10FC9000882319F09585891789F08BE2FA01119272
:10FCA0008A95E9F7D8011D968C91F9018483DA01D0
:10FCB0009796CD92DD92ED92FC929A97F801808111
:10FCC00090E08F73907001972DE030E0829FB0013B
:10FCD000839F700D929F700D1124FE013196A2E05A
:10FCE000B2E08DE00D9001928150E1F7DE011196B6
:10FCF00020E06F31710508F09FC03D91CA01860F69
:10FD0000971FF801E30FF11D3081FC0130832F5F55
:10FD10006F5F7F4F2D3009F48FC0EBCFDA019C91DC
:10FD20009923B9F0F901A481F801319661E090E0DE
:10FD300071915C01B694BA2CAA24B794A7949595B6
:10FD400087958A29870F6F5F6B3089F7A81709F4A9
:10FD500057C08BE2DA011D928A95E9F7FA01C7A232
:10FD6000D0A6E1A6F2A66801DA0180E0F601908152
:10FD70009032A1F09C93F801648563FF08C0F601FE
:10FD80006081613420F06B3510F4905E9C938F5F3E
:10FD90000894C11CD11C1196883041F7DA019C915E
:10FDA000953011F495EE9C93F8019085903221F1F5
:10FDB000FA01E80FF11D9EE29083F8013896782F42
:10FDC0007C5F8F5F90819032B9F06A01C80ED11CC0
:10FDD000D6019C93D8011C966C911C9764FF08C0B7
:10FDE0006081613428F06B3518F4905ED6019C93E5
:10FDF0008F5F3196871731F7FA01E80FF11D1082F6
:10FE0000F8018385DA0190968C939097828D938D7B
:10FE100092969C938E939197848D958DA68DB78D98
:10FE2000FA0183A394A3A5A3B6A381E0D9011596F3
:10FE30008C93159780E001C081E02D960FB6F89461
:10FE4000DEBF0FBECDBFDF91CF911F910F91FF900D
:10FE5000EF90DF90CF90BF90AF9008954F925F9258
:10FE60006F927F928F929F92AF92BF92CF92DF92CA
:10FE7000EF92FF920F931F93CF93DF93CDB7DEB72F
:10FE8000A0970FB6F894DEBF0FBECDBF6B010097F1
:10FE900009F42BC16115710509F427C1DC01ED914D
:10FEA000FC9184809580FB0147A050A461A472A4BA
:10FEB000F62E1D2DDB010D900020E9F711970A2F7A
:10FEC000061B802F90E00C966DE070E00E94E9E444
:10FED000E62ECE01019660E270E04BE050E00E9419
:10FEE00086E5C6016EE270E00E94BEE50097E1F093
:10FEF000DC0111962C9111972223B1F0BC016F5FA8
:10FF00007F4FDB010D900020E9F71197A61BB70B7F
:10FF10008A2F8095080FCE0109964A2FA43008F049
:10FF200043E050E00E947DE5093098F4CE0101964F
:10FF30006F2D712F402F50E00E947DE5F6018081EA
:10FF40008E3259F581818E3209F48281882321F124
:10FF500024C0DE011196EF2DF12F88E001900D9263
:10FF60008150E1F7D60191962C919197822F90E0E4
:10FF700004E0959587950A95E1F7203A10F4805DA5
:10FF800001C08F598F83822F8F708A3010F4805D6B
:10FF900001C08F59888701C0EE248981853E11F404
:10FFA00085E0898385E1FE013C96DF011D928A95FB
:10FFB000E9F7F60180A18C8781A192A19C8F8B8F9C
:10FFC00083A194A1A5A1B6A18D8F9E8FAF8FB8A359
:10FFD0006E2D70E015E0660F771F1A95E1F780E04F
:10FFE00090E0640D751D861D971D8E010F5F1F4FDC
:10FFF000A80120E230E0F4011995882309F475C0C6
:020000021000EC
:10000000F98020E030E08F2D90E0AC015695542F20
:1000100044275795479595958795F42EF82AF8012A
:10002000E20FF31F8181F80E2F5F3F4F2A30310519
:1000300051F70E2D1DE0A12EB12C1FE051C0CE01B5
:1000400001966FEF70E040E250E00E9486E5802F5D
:1000500090E001978A9DD0018B9DB00D9A9DB00DC7
:100060001124AC0DBD1D81E0E1E0F0E0EC0FFD1FBF
:10007000E80FF11D9C919083982F9F5FE1E0F0E0E5
:10008000EC0FFD1FE90FF11D10828E5F8B3019F010
:100090008A3121F402C08EE001C08CE19D91992348
:1000A00011F08F3108F309830E1519F4802F806445
:1000B00089831C87FE861D861B8E1C8EC301B201A0
:1000C000AE014F5F5F4F20E230E0F401199580E20E
:1000D00090E0A0E0B0E0480E591E6A1E7B1E015061
:1000E000002309F0ACCF81E001C080E0A0960FB6FC
:1000F000F894DEBF0FBECDBFDF91CF911F910F915E
:10010000FF90EF90DF90CF90BF90AF909F908F9037
:100110007F906F905F904F9008950F931F93CF93B0
:10012000DF930F920F92CDB7DEB7FC01009769F114
:100130006230710550F1A081B181660F771F80E0B8
:1001400090E00681178120853185600F711F821F25
:10015000931FED91FC91AE014F5F5F4F22E030E0C5
:100160001995882391F089819A81009781F02FEF6A
:10017000873F920751F09C01205F3F4F27303105A8
:1001800020F02FEF883F920710F080E090E00F9072
:100190000F90DF91CF911F910F910895EF92FF92F1
:1001A0000F931F93CF93DF93CDB7DEB760970FB652
:1001B000F894DEBF0FBECDBF8C010E94E87DAE017A
:1001C0004F5F5F4F20E1DA011D922A95E9F7D801D0
:1001D000ED91FC91119750962D913C91519706808D
:1001E000F781E02D05EE1DE7EE24FF2419956096BA
:1001F0000FB6F894DEBF0FBECDBFDF91CF911F9138
:100200000F91FF90EF9008952F923F924F925F923F
:100210006F927F928F929F92AF92BF92CF92DF9216
:10022000EF92FF920F931F93CF93DF9300D0CDB740
:10023000DEB79B838A839B01009709F4B9C04115FF
:10024000510509F4B5C0DA010D900020E9F7CD01A0
:10025000841B950B0B966DE070E00E94D5E4062F91
:100260000F5FF901208031802114310479F4AA81D3
:10027000BB8156968D909D90AD90BC9059975296AB
:100280004D905D906D907C90559706C04424552408
:1002900032018824992454017501640110E084140A
:1002A0009504A604B70409F055C02114310409F4DB
:1002B0007FC081149104A104B104A9F18A819B81BA
:1002C000B1010E948D80009769F58A819B81B101FF
:1002D00041E050E00E94FE7C8C01009709F468C068
:1002E000BC016250704080E090E0EA81FB8120898F
:1002F000318940E050E00E94AAE46B017C01EA8170
:10030000FB8182899389A489B589C80ED91EEA1E0A
:10031000FB1E0230110508F44EC0CF01B8010E9447
:10032000CE8049C01C018A819B81B1010E94E87D79
:100330004B015C01AA81BB8150968D919C91519794
:100340002C0166247724480C591C6A1C7B1C7501FF
:10035000640110E0AA81BB81ED91FC910190F081D4
:10036000E02DC501B401AE014F5F5F4F21E030E0E9
:1003700019958823E9F08981853E11F0882361F47D
:100380001F5F1017C0F480E290E0A0E0B0E0880E9C
:10039000991EAA1EBB1E83CF90E2C92ED12CE12C40
:1003A000F12CC80CD91CEA1CFB1C4601570176CF66
:1003B000CC24DD247601B601C7010F900F900F9079
:1003C000DF91CF911F910F91FF90EF90DF90CF9031
:1003D000BF90AF909F908F907F906F905F904F9065
:1003E0003F902F9008952F923F924F925F926F927D
:1003F0007F928F929F92AF92BF92CF92DF92EF92B5
:10040000FF920F931F93CF93DF93CDB7DEB7AC97D7
:100410000FB6F894DEBF0FBECDBF8C01009709F474
:1004200065C1DC0114968D919C911597009709F494
:100430005DC116968D919C911797009709F071C137
:1004400055C1E9E9F5E18CE1DF011D928A95E9F7F3
:1004500010939A1500939915D8011996CD90DD90B7
:10046000ED90FC901C9789E0CC0CDD1CEE1CFF1C71
:100470008A95D1F7CA8EDB8EEC8EFD8EC701B60150
:10048000655F7F4F8F4F9F4FED91FC91AE014F5FA6
:100490005F4F29E130E01995882309F423C12980B1
:1004A0003A804C815D81CB80CAA26E81EF80F88456
:1004B000FCA2EBA289859A852C853D85CE88DF88B4
:1004C000E88CF98CCE8EDF8EE8A2F9A2C114D1049B
:1004D000E104F10451F4009709F404C16C01EE2425
:1004E000FF24CE8EDF8EE8A2F9A22115310509F492
:1004F000F9C06A01EE24FF24CDA2DEA2EFA2F8A685
:1005000070E080E090E040E050E00E94AAE469A73B
:100510007AA78BA79CA7CE8CDF8CE8A0F9A08DA131
:100520009EA1AFA1B8A5C81AD90AEA0AFB0A89A5F3
:100530009AA5ABA5BCA5C81AD90AEA0AFB0AC1014B
:1005400001972BA13CA1F5E0220F331FFA95E1F7AB
:10055000820F931FB1010E94D5E4CB01A0E0B0E06F
:10056000C81AD90AEA0AFB0A9AA1292F30E040E00A
:1005700050E0C701B6010E94FCE449015A01253F41
:10058000AFE03A07A0E04A07A0E05A0708F4AAC083
:10059000253FBFEF3B07B0E04B07B0E05B0720F41F
:1005A00086E0F801808704C08BE0D80118968C9310
:1005B00088E1EBE9F5E1DF011D928A95E9F7210178
:1005C000662477246E8D7F8D88A199A1A301920165
:1005D0000E94AAE4DC01CB0180939B1590939C15AB
:1005E000A0939D15B0939E15C301B2012DA13EA10C
:1005F0004FA158A50E94AAE46B017C018A8D9B8DB6
:10060000AC8DBD8DC80ED91EEA1EFB1EC0929F1573
:10061000D092A015E092A115F092A215A501940127
:100620002E5F3F4F4F4F5F4FD80118968C91189710
:10063000863029F462E070E080E090E004C064E07D
:1006400070E080E090E00E94AAE4DC01CB0180939E
:10065000A3159093A415A093A515B093A615309259
:10066000A8152092A715BAA12B2F30E0229DC0011A
:10067000239D900D329D900D11249093AA15809387
:10068000A91569A57AA58BA59CA5A30192010E9435
:10069000AAE4DC01CB018C0D9D1DAE1DBF1D809316
:1006A000AF159093B015A093B115B093B215CBA030
:1006B000DCA0A60160E070E0E5E0440F551F661F76
:1006C000771FEA95D1F7480F591F6A1F7B1F409388
:1006D000AB155093AC156093AD157093AE1589E9C9
:1006E00095E106C010929A151092991580E090E05D
:1006F000AC960FB6F894DEBF0FBECDBFDF91CF91A1
:100700001F910F91FF90EF90DF90CF90BF90AF902F
:100710009F908F907F906F905F904F903F902F9021
:1007200008958091991590919A150097F9F689CEC0
:10073000009719F0FC01118210820895CF93DF9386
:10074000FB01009729F1309719F120A124FF25C062
:100750001FC0A7EBB5E1EF012BE209900D922150EC
:10076000E1F79093B6158093B5151092E2151092AB
:10077000E3151092E4151092E51581A192A19093D2
:10078000E7158093E6151092E81585EB95E102C018
:1007900080E090E0DF91CF9108952091B5153091E0
:1007A000B61521153105A1F7D4CFCF93DF93EC0116
:1007B000009759F08BA9813031F4FE01819191911C
:1007C000BF010E942E7F19821882DF91CF91089578
:1007D0002F923F924F925F926F927F928F929F9251
:1007E000AF92BF92CF92DF92EF92FF920F931F933F
:1007F000CF93DF9300D000D0CDB7DEB78C017C83E0
:100800006B831A01009709F4D9C06115710509F4C9
:10081000D5C04115510509F4D1C0DC019D968D90DC
:100820009D90AD90BC90D09795964D915D916D91B6
:100830007C919897C101A0E0B0E0880D991DAA1D98
:10084000BB1D481759076A077B0728F41A012818A7
:10085000390809F4B0C0D801ED91FC9111972089B5
:1008600031893A832983D1968D919C91D2979E8329
:100870008D83009789F593960D90BC91A02DBE8332
:10088000AD83109739F481149104A104B10409F4E3
:1008900092C094C081149104A104B10489F41CC0D5
:1008A000C418D508E608F708F801808191816D81A8
:1008B0007E810E948D809E838D83009741F47EC04F
:1008C0007501640129813A81290166247724C414C1
:1008D000D504E604F70420F749805A8008944108BB
:1008E0005108482059204101D801ED90FC90C701E2
:1008F0006D817E810E94E87DAB01BC01C980DA80F8
:10090000C418D5088C149D0408F46401D701ED9136
:10091000FC91C201A0E0B0E0840F951FA61FB71F95
:100920000190F081E02DBC01CD014B815C819601ED
:100930001995882379F1EB81FC81EC0DFD1DFC8379
:10094000EB838C189D08A60160E070E0F80185A596
:1009500096A5A7A5B0A9840F951FA61FB71F85A7A9
:1009600096A7A7A7B0ABC601840D951D29813A8132
:1009700082179307A8F0808191816D817E810E940A
:100980008D809E838D83009749F4D801D2961C9266
:100990001E92D197C1018819990912C04424552487
:1009A0002D813E81F80132AB21AB8114910409F015
:1009B0009BCFC10105C080E090E002C08FEF9FEFA8
:1009C00026960FB6F894DEBF0FBECDBFDF91CF9154
:1009D0001F910F91FF90EF90DF90CF90BF90AF905D
:1009E0009F908F907F906F905F904F903F902F904F
:1009F00008952F923F924F925F926F927F928F92C3
:100A00009F92AF92BF92CF92DF92EF92FF920F939D
:100A10001F93CF93DF9300D000D0CDB7DEB79E8376
:100A20008D837A8369835C834B83009709F406C1C5
:100A30006115710509F402C14115510509F4FEC0A3
:100A4000DC019D964D905D906D907C90D097FC015F
:100A500085A196A1A7A1B0A584159505A605B70502
:100A600008F4ECC080819181DC0150962D903C907F
:100A7000519701A912A90115110509F050C003A150
:100A800014A101151105A1F441145104610471046C
:100A900009F0D4C060E070E041E050E00E94FE7CCC
:100AA0008C01ED81FE8194A383A3009709F4C6C055
:100AB000AD81BE819D96CD90DD90ED90FC90D0975C
:100AC000C114D104E104F10451F121C0C818D908BE
:100AD000EA08FB08ED81FE8180819181B8010E94C6
:100AE0008D80009791F4C114D104E104F10409F060
:100AF000A5C0AD81BE818D919C91B80141E050E0CF
:100B00000E94FE7C009709F499C08C0103C041014A
:100B1000AA24BB24C814D904EA04FB04B8F6710162
:100B20000894E108F108E420F5208B809C80ED8199
:100B3000FE8140805180C201B8010E94E87DAB0176
:100B4000BC016101CE18DF088C149D0408F4640117
:100B5000D201ED91FC91C701A0E0B0E0840F951F98
:100B6000A61FB71F0480F581E02DBC01CD0149818E
:100B70005A8196011995882309F446C0E981FA81C2
:100B8000EC0DFD1DFA83E9838C189D08A60160E039
:100B900070E0ED81FE8185A596A5A7A5B0A9840F7B
:100BA000951FA61FB71F85A796A7A7A7B0ABC6011D
:100BB0008E0D9F1D82159305E8F080819181B8010B
:100BC0000E948D80009799F48114910459F0AD81B1
:100BD000BE818D919C91B80141E050E00E94FE7C65
:100BE000009729F4ED81FE8112AA11AA0DC08C0193
:100BF000EE24FF24AD81BE81D2961C930E93D19733
:100C00008114910409F093CFED81FE8145A556A58D
:100C100067A570A985A196A1A7A1B0A5841795077E
:100C2000A607B70730F481E083AB45A356A367A3BB
:100C300070A78B819C818819990902C08FEF9FEF63
:100C400026960FB6F894DEBF0FBECDBFDF91CF91D1
:100C50001F910F91FF90EF90DF90CF90BF90AF90DA
:100C60009F908F907F906F905F904F903F902F90CC
:100C700008954F925F926F927F92AF92BF92CF9200
:100C8000DF92EF92FF920F931F93CF93DF9300D0E9
:100C900000D0CDB7DEB75C014B835C836D837E8370
:100CA000009709F4D6C0DC0193960D911C9194979E
:100CB000ED91FC911197C088D1880115110539F08B
:100CC0004B805C806D807E80EE24FF2418C02B81D9
:100CD0003C814D815E81211531054105510509F4A5
:100CE000A3C0EECFD5018D919C91B8010E948D805B
:100CF000009769F04C185D086E087F088C01C414D9
:100D0000D504E604F70470F30115110511F5D701B8
:100D1000C601840D951DA61DB71D0197A109B10936
:100D2000BC01CD01A70196010E94FCE4F501808180
:100D30009181B801A9010E94FE7C009709F489C045
:100D40000115110531F4D50194969C938E939397D8
:100D50008C012B813C814D815E81D50195962D932F
:100D60003D934D935C9398972115310541055105AD
:100D700021F494961C921E929397F5018191919182
:100D8000BF010E942E7F882309F463C02B813C8120
:100D90004D815E81211531054105510531F4D501A3
:100DA0008D919C911197B8013DC0C414D504E604FF
:100DB000F704D0F1F501C080D180C114D104A1F1B4
:100DC0000230110588F1C601B8010E948D802C0106
:100DD0008FEF9FEF9A838983D6014D915C91119794
:100DE000000F111F20E030E016968D919D910D901F
:100DF000BC91A02D080F191F2A1F3B1FDA01149662
:100E0000ED91FC911597C901B801AE014F5F5F4F9D
:100E100022E030E01995882339F04114510421F083
:100E2000C601B2010E948C7CF50185A596A5A7A5F7
:100E3000B0A92B813C814D815E81281739074A0773
:100E40005B0748F425A736A747A750AB12AA11AAFB
:100E500002C080E001C081E026960FB6F894DEBFA4
:100E60000FBECDBFDF91CF911F910F91FF90EF90FB
:100E7000DF90CF90BF90AF907F906F905F904F903A
:100E80000895CF92DF92EF92FF920F931F93CF932B
:100E9000DF93EC018B010097C1F161157105A9F198
:100EA0008DA59EA5AFA5B8A9413059F0413018F0E5
:100EB000423059F50CC0FB01C080D180E280F38044
:100EC00013C0FB01C080D180E280F38009C0FB0128
:100ED000C080D180E280F3808DA19EA1AFA1B8A592
:100EE000C80ED91EEA1EFB1E8DA19EA1AFA1B8A5FA
:100EF0008C159D05AE05BF0590F4CE01B701A60186
:100F00000E943986882359F401C080E0DF91CF9197
:100F10001F910F91FF90EF90DF90CF900895CDA695
:100F2000DEA6EFA6F8AA1AAA19AAF801C082D182F1
:100F3000E282F38281E0EACFCF93DF939C01EB0161
:100F4000009789F1209779F188A184FF2CC08091C6
:100F5000E9159091EA15009749F080911A16909141
:100F60001B16009701F5AAE1B6E102C0A9EEB5E1B2
:100F7000BD016E5F7F4FCE014BE2FC010190CF01BE
:100F8000FB010192BF014150C1F711963C932E9392
:100F900089A19AA19E969C938E939D97D0961C9220
:100FA0001E929F9702C0A0E0B0E0CD01DF91CF91EB
:100FB0000895009719F0FC011182108208952F9274
:100FC0003F924F925F926F927F928F929F92AF92D9
:100FD000BF92CF92DF92EF92FF920F931F93CF9326
:100FE000DF93CDB7DEB7A8970FB6F894DEBF0FBE7C
:100FF000CDBF5C01009709F497C06115710509F434
:1010000093C0DC016D907C901197F30120883188AA
:101010009D964D905C909E979F968D909C90D097BA
:101020008214930408F066C0FE01319686E0DF0169
:101030001D928A95E9F78BE2FB0111928A95E9F7F7
:101040007A8369834114510409F063C0D301529635
:101050002D903C90539756968D919C915797281AB6
:10106000390A57C08101081919096401EE24FF24C7
:101070004114510431F4F30186899789A08DB18D13
:1010800006C0C301B2010E94E87DDC01CB018C0DDA
:101090009D1DAE1DBF1D1C821B82F301208131816D
:1010A000F9010280F381E02DBC01CD01AE01495F61
:1010B0005F4F20E230E00F2EF2E1EF2EFEE7FF2E31
:1010C000F02D6E010894C11CD11C1995882361F183
:1010D0008B819C81880E991E82149304D0F0C301E9
:1010E000B2010E948D802C01009789F48E818823A3
:1010F000A1F4D50193968D919C9194979E969C9383
:101100008E939D97D0961C921E929F970DC0882417
:1011100099248E81882309F4A5CFF50156A645A60A
:1011200090AA87A68E8101C080E0A8960FB6F89499
:10113000DEBF0FBECDBFDF91CF911F910F91FF900A
:10114000EF90DF90CF90BF90AF909F908F907F9067
:101150006F905F904F903F902F9008958F929F9245
:10116000AF92BF92CF92DF92EF92FF920F931F93B5
:10117000CF93DF934C01EB018A01009709F465C01E
:10118000209709F462C08881882309F45EC0411564
:10119000510509F45AC08F3209F421968BE2F80107
:1011A00011928A95E9F780E1F80180A301C0E50179
:1011B0008881882309F44BC0C401B8010E949C8730
:1011C0006C01009709F441C0CE016FE270E00E940B
:1011D0008DE5009739F0E82FEC1B5C010894A11C09
:1011E000B11C2AC0AC2FBD2FFD0101900020E9F7F2
:1011F0003197EC1B5E01AE0EB11C1EC0F8010190D0
:101200000020E9F73197E01BF10BEE15FF05B1F473
:10121000CE01B801A7010E94A1E5009779F4F6017B
:1012200011821082CE0DDF1D8881882381F0F801A4
:1012300080A184FDBCCF09C0EE2EFF24C601B801F9
:101240000E94DF878823D1F610C080E001C081E0D2
:10125000DF91CF911F910F91FF90EF90DF90CF9092
:10126000BF90AF909F908F900895F60111821082E9
:101270009FCFFC01009741F083A194A196A785A779
:1012800010AA17A681E0089580E00895CF92DF921A
:10129000EF92FF920F931F93CF93DF938C017B010B
:1012A000EA01009709F444C06115710509F440C0D2
:1012B000FB0180818823E1F12097D1F1C801BE01B3
:1012C0000E94DF87882371F0C701BE010E9498E564
:1012D0000097A1F7F80183A194A196A785A710AA6A
:1012E00017A626C0F801C080D1808BE2FE011192C2
:1012F0008A95E9F7CE01B7014FE150E00E94AFE5D2
:10130000B8016D5D7F4FC601AE010E940481DC0112
:10131000CB018FA398A7A9A7BAA70097A105B105EC
:1013200039F0C601BE010E942E7F91E0882309F4A6
:1013300090E0892FDF91CF911F910F91FF90EF9057
:10134000DF90CF9008959F92AF92BF92CF92DF929D
:10135000EF92FF920F931F93CF93DF93CDB7DEB73A
:101360002C970FB6F894DEBF0FBECDBF8C015B018A
:10137000009709F453C06115710509F44FC0DB01F2
:101380009796CD90DD90ED90FC909A97C114D10482
:10139000E104F10409F442C085EE982ED801ED91E4
:1013A000FC910190F081E02DC701B601AE014F5FC5
:1013B0005F4F2CE030E01995882381F19982D801A4
:1013C000ED91FC910480F581E02DC701B601AE01DD
:1013D0004F5F5F4F2CE030E019958823F9F08C8542
:1013E0008F3049F480E290E0A0E0B0E0C80ED91E52
:1013F000EA1EFB1ED3CFD50191966D917C919297F9
:101400006115710541F0C8010E948C7C91E0882330
:1014100019F490E001C091E0892F01C080E02C9682
:101420000FB6F894DEBF0FBECDBFDF91CF911F91F5
:101430000F91FF90EF90DF90CF90BF90AF909F9073
:1014400008958F929F92AF92BF92CF92DF92EF92C8
:10145000FF920F93CF93DF93CDB7DEB760970FB6B0
:10146000F894DEBF0FBECDBF7C016B015A0149016C
:10147000009709F4A2C06115710509F49EC00430FB
:101480000CF09BC007FD1DC0602F772767FD70958E
:1014900084E0660F771F8A95E1F762547E4F8827B4
:1014A00077FD8095982FAE014F5F5F4F20E130E0D0
:1014B000F7011995882309F480C08D81882309F4E8
:1014C0007CC080915316882309F077C0EBE4F6E1E5
:1014D00081E1DF011D928A95E9F7F0924C16E092C6
:1014E0004B16D0924E16C0924D16B0925016A09246
:1014F0004F16909252168092511607FD5AC08D8158
:10150000809353168A8590E0A0E0B0E0BA2FA92F0F
:10151000982F88274B8550E060E070E0BA0155278E
:101520004427842B952BA62BB72B498550E060E0F0
:1015300070E0842B952BA62BB72B4C8550E060E0F8
:1015400070E0742F662755274427842B952BA62BF4
:10155000B72B81879287A387B4878E8590E0A0E020
:10156000B0E0BA2FA92F982F88274F8550E060E070
:1015700070E0BA0155274427842B952BA62BB72B57
:101580004D8550E060E070E0842B952BA62BB72BA7
:10159000488950E060E070E0742F662755274427A3
:1015A000842B952BA62BB72B85879687A787B08B87
:1015B00006C08FEF8093531602C0E0E0F0E0CF0149
:1015C00060960FB6F894DEBF0FBECDBFDF91CF910E
:1015D0000F91FF90EF90DF90CF90BF90AF909F90D2
:1015E0008F900895009721F0FC01108681E0089506
:1015F00080E008958EBD0DB407FEFDCF8DB58F77C9
:101600008DBD08958FEF8EBD0DB407FEFDCF8DB556
:101610008F778DBD8EB508951F93CF93DF9300D044
:101620000F92CDB7DEB7182F4C835B836A83798323
:101630000E94028B812F80640E94FA8A7981872F11
:101640000E94FA8A6A81862F0E94FA8A5B81852F1E
:101650000E94FA8A4C81842F0E94FA8A112319F081
:10166000183041F405C085E90E94FA8A1AE004C0E6
:1016700087E8FACF8FEFF8CF0E94028B8F3F11F4EB
:101680001150D1F70F900F900F900F90DF91CF91E5
:101690001F910895CF93DF9300D0CDB7DEB780912F
:1016A000651B9091661B9A8389838B81807F816003
:1016B0008B83CE01019661E00E94D89591E0892745
:1016C0000F900F900F90DF91CF910895CF93DF93FC
:1016D00000D0CDB7DEB78091651B9091661B9A83D1
:1016E00089838B81807F8B83CE01019660E00E948D
:1016F000D8950F900F900F90DF91CF910895809122
:1017000061168823B1F460915D1670915E16809128
:101710005F169091601642E656E120E032E00E94AA
:10172000488D882321F081E080936116089580E040
:10173000089581E008952F923F924F925F926F92A9
:101740007F928F929F92AF92BF92CF92DF92EF9251
:10175000FF920F931F93CF93DF932B013C015A010C
:1017600019016DC08FEF882E81E0982E842095207E
:10177000C401A0E0B0E073016201C81AD90AEA0A04
:10178000FB0AC0E0D2E0C819D9092C163D0608F4BE
:10179000E10180915D1690915E16A0915F16B09167
:1017A0006016C816D906EA06FB06B9F10E947F8BBF
:1017B000882309F44AC0289881E1B701A6010E9454
:1017C0000C8B882311F0289A40C00E94028B8E3F18
:1017D000E1F702E616E10E94028BF80181938F0186
:1017E000F8E102361F07B9F7C0925D16D0925E1677
:1017F000E0925F16F0926016B4016E59794EC50101
:10180000AE010E947DE5AC0EBD1E0E94028B0E94BF
:10181000028B289A0E94028B09C0B4016E59794E3E
:10182000C501AE010E947DE5AC0EBD1E2C1A3D0A1D
:10183000CE01A0E0B0E0480E591E6A1E7B1E2114A6
:10184000310409F08FCF81E001C080E0DF91CF91BA
:101850001F910F91FF90EF90DF90CF90BF90AF90CE
:101860009F908F907F906F905F904F903F902F90C0
:1018700008952F923F924F925F926F927F928F9234
:101880009F92AF92BF92CF92DF92EF92FF920F930F
:101890001F93CF93DF932B013C011A01E9014115FE
:1018A000510529F1209719F10217130700F1E114EE
:1018B000F104E9F04901AA24BB24C301B201A1014A
:1018C0009E010E949B8B882391F0C101B301A2016C
:1018D0009601F7011995882361F0480C591C6A1C80
:1018E0007B1C0C1B1D0B0C171D0738F702C080E07A
:1018F00001C081E0DF91CF911F910F91FF90EF9098
:10190000DF90CF90BF90AF909F908F907F906F901F
:101910005F904F903F902F9008950F931F93CF9318
:10192000DF9300D000D0CDB7DEB78091651B9091DA
:10193000661B9D838C838E81807F81608E83CE0128
:10194000049661E040E00E94C3958091651B9091F0
:10195000661B9A8389838B81807F8B83CE0101965E
:1019600060E040E00E94C395229A219A209A239831
:10197000289A83E58CBD8DB58E7F8DBD10925C1647
:101980000E944A8B882309F476C00AE00E94028BE9
:101990000150E1F7289800E012E080E040E050E0DC
:1019A00060E070E00E940C8B813021F0015010400B
:1019B000A1F733C087E340E050E060E070E00E94B0
:1019C0000C8B89E240E050E060E070E00E940C8BFC
:1019D00082FD05C080915C16816080935C1600E0FA
:1019E00010E880915C1690E083709070009749F049
:1019F00087E340E050E060E070E00E940C8B89E2F9
:101A000001C081E040E050E060E070E00E940C8B9B
:101A100080FF05C00150104021F7289A2CC080E1BA
:101A200040E052E060E070E00E940C8B289A88232E
:101A300011F58CB58C7F8CBD8DB581608DBD8FEF20
:101A40009FEFAFEFBFEF80935D1690935E16A0936C
:101A50005F16B093601681E08093611660E070E0DD
:101A600080E090E042E656E120E032E00E949B8B6D
:101A700091E0882309F490E0892F26960FB6F89418
:101A8000DEBF0FBECDBFDF91CF911F910F910895A3
:101A90003F924F925F926F927F928F929F92AF92FE
:101AA000BF92CF92DF92EF92FF920F931F93CF934B
:101AB000DF932B013C014A0159010E94668B882368
:101AC00009F481C088C0E201D170CE01A0E0B0E08D
:101AD00073016201C81AD90AEA0AFB0A00E012E09F
:101AE0000C1B1D0BA016B10608F4850180915D1634
:101AF00090915E16A0915F16B0916016C816D90637
:101B0000EA06FB06F1F00E947F8B882309F463C08C
:101B1000209721F482E00030180758F4C701B6017D
:101B200042E656E120E032E00E949B8B882309F4D4
:101B300052C0C0925D16D0925E16E0925F16F0928F
:101B4000601682E6881686E1980661F0CE018E590D
:101B5000994EB401A8010E947DE510926116A0166D
:101B6000B106B9F1289888E1B701A6010E940C8B53
:101B7000882311F0289A2FC08EEF0E94FA8AC2E6BD
:101B8000D6E189910E94FA8A88E1C236D807C9F75E
:101B90008FEF0E94FA8A8FEF0E94FA8A0E94028BCE
:101BA0008F3FE1F70E94028B289A800E911EC80198
:101BB000A0E0B0E0480E591E6A1E7B1EA01AB10AB2
:101BC0003092611602C033243394A114B10409F099
:101BD0007ACF81E001C080E0DF91CF911F910F911A
:101BE000FF90EF90DF90CF90BF90AF909F908F903D
:101BF0007F906F905F904F903F9008954F925F92CB
:101C00006F927F928F929F92AF92BF92CF92DF920C
